
IBM(R) Linker for OS/2(R), Version 5.0 
Copyright (C) IBM Corporation 1988, 2003.
Copyright (C) Microsoft Corp. 1988, 1989.
All rights reserved.

Current option settings:
	PDD	CODE:RX	DATA:RWS
	Alignfile:0x00000010	ALIGNAddr:0x00010000	NOBASe
	BRowse	NODBgpack	DEbug:none	NODEFaultlibrarysearch
	NOEXEPACK	NOEXTdictionary	NOFIxed	FReeformat	NOIGnorecase
	Linenumbers	NOLOgo	MAP:bin\Debug.ACP\uniaud32.map
	OCache:0x1d1d0000	OLDcpp	NOOPTFunc	PACKCode:0xffffffff
	PACKData:0xffffffff	PMTYPE:VIO	SEGMENTS:256 	NOSEGOrder
	NOSTRictwarnings	NONOSTRictwarnings	NOSTUB	NOVERBose
	VERSION:00.00


ILink : warning LNK4019: device driver can not have a stack

 UNIAUD32

 Start         Length     Name                   Class
 0001:00000000 00000048BH DATA16                 DATA16 16-bit
	at offset 00000000 0048BH bytes from F:\src\os2\uniaud32t\drv32\bin\Debug.ACP\startup.obj (startup.asm)

 0002:00000000 0000006DBH CODE16                 CODE 16-bit
	at offset 00000000 006DBH bytes from F:\src\os2\uniaud32t\drv32\bin\Debug.ACP\startup.obj (startup.asm)

 0003:00000000 000000000H FIRSTCODE32            CODE 32-bit

 0003:00000000 0000DE07FH CODE32                 CODE 32-bit
	at offset 00000000 004DDH bytes from F:\src\os2\uniaud32t\drv32\bin\Debug.ACP\startup.obj (startup.asm)
	at offset 000004DD 001FBH bytes from F:\src\os2\uniaud32t\drv32\bin\Debug.ACP\strategy.obj (F:\src\os2\uniaud32t\drv32\strategy.c)
	at offset 000006D8 00176H bytes from F:\src\os2\uniaud32t\drv32\bin\Debug.ACP\read.obj (F:\src\os2\uniaud32t\drv32\read.cpp)
	at offset 0000084E 005CFH bytes from F:\src\os2\uniaud32t\drv32\bin\Debug.ACP\init.obj (F:\src\os2\uniaud32t\drv32\init.c)
	at offset 00000E1D 00807H bytes from F:\src\os2\uniaud32t\drv32\bin\Debug.ACP\parse.obj (F:\src\os2\uniaud32t\drv32\parse.c)
	at offset 00001624 0004EH bytes from F:\src\os2\uniaud32t\drv32\bin\Debug.ACP\devhlp.obj (devhlp.asm)
	at offset 00001672 00641H bytes from F:\src\os2\uniaud32t\drv32\bin\Debug.ACP\idc.obj (F:\src\os2\uniaud32t\drv32\idc.c)
	at offset 00001CB3 00C39H bytes from F:\src\os2\uniaud32t\drv32\bin\Debug.ACP\dispatch.obj (F:\src\os2\uniaud32t\drv32\dispatch.c)
	at offset 000028EC 00A3AH bytes from F:\src\os2\uniaud32t\drv32\bin\Debug.ACP\rmhelp.obj (F:\src\os2\uniaud32t\drv32\rmhelp.cpp)
	at offset 00003326 0018EH bytes from F:\src\os2\uniaud32t\drv32\bin\Debug.ACP\irq.obj (F:\src\os2\uniaud32t\drv32\irq.cpp)
	at offset 000034B4 00194H bytes from F:\src\os2\uniaud32t\drv32\bin\Debug.ACP\util.obj (F:\src\os2\uniaud32t\drv32\util.cpp)
	at offset 00003648 00724H bytes from F:\src\os2\uniaud32t\lib\Debug.ACP\linuxlib.lib (F:\src\os2\uniaud32t\lib32\vsprintf.c)
	at offset 00003D6C 00204H bytes from F:\src\os2\uniaud32t\lib\Debug.ACP\linuxlib.lib (F:\src\os2\uniaud32t\lib32\timer.c)
	at offset 00003F70 000CCH bytes from F:\src\os2\uniaud32t\lib\Debug.ACP\linuxlib.lib (F:\src\os2\uniaud32t\lib32\strncmp.c)
	at offset 0000403C 000AEH bytes from F:\src\os2\uniaud32t\lib\Debug.ACP\linuxlib.lib (F:\src\os2\uniaud32t\lib32\task.c)
	at offset 000040EA 008F5H bytes from F:\src\os2\uniaud32t\lib\Debug.ACP\linuxlib.lib (F:\src\os2\uniaud32t\lib32\misc.c)
	at offset 000049DF 004DBH bytes from F:\src\os2\uniaud32t\lib\Debug.ACP\linuxlib.lib (F:\src\os2\uniaud32t\lib32\ossidc.cpp)
	at offset 00004EBA 00966H bytes from F:\src\os2\uniaud32t\lib\Debug.ACP\linuxlib.lib (F:\src\os2\uniaud32t\lib32\soundmidi.c)
	at offset 00005820 017B1H bytes from F:\src\os2\uniaud32t\lib\Debug.ACP\linuxlib.lib (F:\src\os2\uniaud32t\lib32\soundmixer.c)
	at offset 00006FD1 02654H bytes from F:\src\os2\uniaud32t\lib\Debug.ACP\linuxlib.lib (F:\src\os2\uniaud32t\lib32\sound.c)
	at offset 00009625 00806H bytes from F:\src\os2\uniaud32t\lib\Debug.ACP\linuxlib.lib (F:\src\os2\uniaud32t\lib32\debug.c)
	at offset 00009E2B 00B85H bytes from F:\src\os2\uniaud32t\lib\Debug.ACP\linuxlib.lib (F:\src\os2\uniaud32t\lib32\memory.cpp)
	at offset 0000A9B0 01C82H bytes from F:\src\os2\uniaud32t\lib\Debug.ACP\linuxlib.lib (F:\src\os2\uniaud32t\lib32\ioctl.c)
	at offset 0000C632 0050DH bytes from F:\src\os2\uniaud32t\lib\Debug.ACP\linuxlib.lib (F:\src\os2\uniaud32t\lib32\irq.c)
	at offset 0000CB3F 02C25H bytes from F:\src\os2\uniaud32t\lib\Debug.ACP\linuxlib.lib (F:\src\os2\uniaud32t\lib32\pci.c)
	at offset 0000F764 0092FH bytes from F:\src\os2\uniaud32t\lib\Debug.ACP\linuxlib.lib (F:\src\os2\uniaud32t\lib32\malloc.cpp)
	at offset 00010093 00067H bytes from F:\src\os2\uniaud32t\lib\Debug.ACP\linuxlib.lib (F:\src\os2\uniaud32t\lib32\strncpy.c)
	at offset 000100FA 0013FH bytes from F:\src\os2\uniaud32t\lib\Debug.ACP\linuxlib.lib (F:\src\os2\uniaud32t\lib32\waitqueue.c)
	at offset 00010239 000B6H bytes from F:\src\os2\uniaud32t\lib\Debug.ACP\linuxlib.lib (F:\src\os2\uniaud32t\lib32\spinlock.c)
	at offset 000102EF 01019H bytes from F:\src\os2\uniaud32t\lib\Debug.ACP\core.lib (F:\src\os2\uniaud32t\alsa-kernel\core\hwdep.c)
	at offset 00011308 03FA1H bytes from F:\src\os2\uniaud32t\lib\Debug.ACP\core.lib (F:\src\os2\uniaud32t\alsa-kernel\core\timer.c)
	at offset 000152A9 031B5H bytes from F:\src\os2\uniaud32t\lib\Debug.ACP\core.lib (F:\src\os2\uniaud32t\alsa-kernel\core\rawmidi.c)
	at offset 0001845E 005BCH bytes from F:\src\os2\uniaud32t\lib\Debug.ACP\core.lib (F:\src\os2\uniaud32t\alsa-kernel\core\pcm_misc.c)
	at offset 00018A1A 04C2BH bytes from F:\src\os2\uniaud32t\lib\Debug.ACP\core.lib (F:\src\os2\uniaud32t\alsa-kernel\core\pcm_lib.c)
	at offset 0001D645 01677H bytes from F:\src\os2\uniaud32t\lib\Debug.ACP\core.lib (F:\src\os2\uniaud32t\alsa-kernel\core\pcm.c)
	at offset 0001ECBC 007D2H bytes from F:\src\os2\uniaud32t\lib\Debug.ACP\core.lib (F:\src\os2\uniaud32t\alsa-kernel\core\sound.c)
	at offset 0001F48E 017FAH bytes from F:\src\os2\uniaud32t\lib\Debug.ACP\core.lib (F:\src\os2\uniaud32t\alsa-kernel\core\info.c)
	at offset 00020C88 00667H bytes from F:\src\os2\uniaud32t\lib\Debug.ACP\core.lib (F:\src\os2\uniaud32t\alsa-kernel\core\pcm_memory.c)
	at offset 000212EF 003D0H bytes from F:\src\os2\uniaud32t\lib\Debug.ACP\core.lib (F:\src\os2\uniaud32t\alsa-kernel\core\pcm_timer.c)
	at offset 000216BF 069C1H bytes from F:\src\os2\uniaud32t\lib\Debug.ACP\core.lib (F:\src\os2\uniaud32t\alsa-kernel\core\pcm_native.c)
	at offset 00028080 0034DH bytes from F:\src\os2\uniaud32t\lib\Debug.ACP\core.lib (F:\src\os2\uniaud32t\alsa-kernel\core\info_oss.c)
	at offset 000283CD 00698H bytes from F:\src\os2\uniaud32t\lib\Debug.ACP\core.lib (F:\src\os2\uniaud32t\alsa-kernel\core\sound_oss.c)
	at offset 00028A65 005C9H bytes from F:\src\os2\uniaud32t\lib\Debug.ACP\core.lib (F:\src\os2\uniaud32t\alsa-kernel\core\device.c)
	at offset 0002902E 02F35H bytes from F:\src\os2\uniaud32t\lib\Debug.ACP\core.lib (F:\src\os2\uniaud32t\alsa-kernel\core\control.c)
	at offset 0002BF63 00714H bytes from F:\src\os2\uniaud32t\lib\Debug.ACP\core.lib (F:\src\os2\uniaud32t\alsa-kernel\core\memalloc.c)
	at offset 0002C677 01530H bytes from F:\src\os2\uniaud32t\lib\Debug.ACP\core.lib (F:\src\os2\uniaud32t\alsa-kernel\core\init.c)
	at offset 0002DBA7 002DEH bytes from F:\src\os2\uniaud32t\lib\Debug.ACP\core.lib (F:\src\os2\uniaud32t\alsa-kernel\core\sgbuf.c)
	at offset 0002DE85 019B9H bytes from F:\src\os2\uniaud32t\lib\Debug.ACP\pci.lib (F:\src\os2\uniaud32t\alsa-kernel\pci\bt87x.c)
	at offset 0002F83E 0143EH bytes from F:\src\os2\uniaud32t\lib\Debug.ACP\pci.lib (F:\src\os2\uniaud32t\alsa-kernel\pci\als4000.c)
	at offset 00030C7C 050A4H bytes from F:\src\os2\uniaud32t\lib\Debug.ACP\pci.lib (F:\src\os2\uniaud32t\alsa-kernel\pci\cmipci.c)
	at offset 00035D20 02745H bytes from F:\src\os2\uniaud32t\lib\Debug.ACP\pci.lib (F:\src\os2\uniaud32t\alsa-kernel\pci\atiixp.c)
	at offset 00038465 02074H bytes from F:\src\os2\uniaud32t\lib\Debug.ACP\pci.lib (F:\src\os2\uniaud32t\alsa-kernel\pci\fm801.c)
	at offset 0003A4D9 03BDDH bytes from F:\src\os2\uniaud32t\lib\Debug.ACP\pci.lib (F:\src\os2\uniaud32t\alsa-kernel\pci\via82xx.c)
	at offset 0003E0B6 0309AH bytes from F:\src\os2\uniaud32t\lib\Debug.ACP\pci.lib (F:\src\os2\uniaud32t\alsa-kernel\pci\maestro3.c)
	at offset 00041150 04EA8H bytes from F:\src\os2\uniaud32t\lib\Debug.ACP\pci.lib (F:\src\os2\uniaud32t\alsa-kernel\pci\intel8x0.c)
	at offset 00045FF8 0429AH bytes from F:\src\os2\uniaud32t\lib\Debug.ACP\pci.lib (F:\src\os2\uniaud32t\alsa-kernel\pci\es1968.c)
	at offset 0004A292 02C2AH bytes from F:\src\os2\uniaud32t\lib\Debug.ACP\pci.lib (F:\src\os2\uniaud32t\alsa-kernel\pci\es1938.c)
	at offset 0004CEBC 0357AH bytes from F:\src\os2\uniaud32t\lib\Debug.ACP\pci.lib (F:\src\os2\uniaud32t\alsa-kernel\pci\cs4281.c)
	at offset 00050436 031D8H bytes from F:\src\os2\uniaud32t\lib\Debug.ACP\pci.lib (F:\src\os2\uniaud32t\alsa-kernel\pci\ens1371.c)
	at offset 0005360E 0046DH bytes from F:\src\os2\uniaud32t\lib\Debug.ACP\pci.lib (F:\src\os2\uniaud32t\alsa-kernel\pci\pci_iomap_compat.c)
	at offset 00053A7B 02958H bytes from F:\src\os2\uniaud32t\lib\Debug.ACP\ca0106.lib (F:\src\os2\uniaud32t\alsa-kernel\pci\ca0106\ca0106_main.c)
	at offset 000563D3 00899H bytes from F:\src\os2\uniaud32t\lib\Debug.ACP\ca0106.lib (F:\src\os2\uniaud32t\alsa-kernel\pci\ca0106\ca_midi.c)
	at offset 00056C6C 015E3H bytes from F:\src\os2\uniaud32t\lib\Debug.ACP\ca0106.lib (F:\src\os2\uniaud32t\alsa-kernel\pci\ca0106\ca0106_mixer.c)
	at offset 0005824F 00DDCH bytes from F:\src\os2\uniaud32t\lib\Debug.ACP\ca0106.lib (F:\src\os2\uniaud32t\alsa-kernel\pci\ca0106\ca0106_proc.c)
	at offset 0005902B 048CDH bytes from F:\src\os2\uniaud32t\lib\Debug.ACP\hda.lib (F:\src\os2\uniaud32t\alsa-kernel\pci\hda\patch_via.c)
	at offset 0005D8F8 01EC3H bytes from F:\src\os2\uniaud32t\lib\Debug.ACP\hda.lib (F:\src\os2\uniaud32t\alsa-kernel\pci\hda\patch_conexant.c)
	at offset 0005F7BB 003FFH bytes from F:\src\os2\uniaud32t\lib\Debug.ACP\hda.lib (F:\src\os2\uniaud32t\alsa-kernel\pci\hda\patch_atihdmi.c)
	at offset 0005FBBA 07E77H bytes from F:\src\os2\uniaud32t\lib\Debug.ACP\hda.lib (F:\src\os2\uniaud32t\alsa-kernel\pci\hda\patch_sigmatel.c)
	at offset 00067A31 03A23H bytes from F:\src\os2\uniaud32t\lib\Debug.ACP\hda.lib (F:\src\os2\uniaud32t\alsa-kernel\pci\hda\patch_analog.c)
	at offset 0006B454 00D0FH bytes from F:\src\os2\uniaud32t\lib\Debug.ACP\hda.lib (F:\src\os2\uniaud32t\alsa-kernel\pci\hda\patch_cmedia.c)
	at offset 0006C163 0BBB7H bytes from F:\src\os2\uniaud32t\lib\Debug.ACP\hda.lib (F:\src\os2\uniaud32t\alsa-kernel\pci\hda\patch_realtek.c)
	at offset 00077D1A 03C29H bytes from F:\src\os2\uniaud32t\lib\Debug.ACP\hda.lib (F:\src\os2\uniaud32t\alsa-kernel\pci\hda\hda_intel.c)
	at offset 0007B943 06C02H bytes from F:\src\os2\uniaud32t\lib\Debug.ACP\hda.lib (F:\src\os2\uniaud32t\alsa-kernel\pci\hda\hda_codec.c)
	at offset 00082545 00463H bytes from F:\src\os2\uniaud32t\lib\Debug.ACP\hda.lib (F:\src\os2\uniaud32t\alsa-kernel\pci\hda\hda_hwdep.c)
	at offset 000829A8 01F73H bytes from F:\src\os2\uniaud32t\lib\Debug.ACP\hda.lib (F:\src\os2\uniaud32t\alsa-kernel\pci\hda\hda_generic.c)
	at offset 0008491B 01819H bytes from F:\src\os2\uniaud32t\lib\Debug.ACP\hda.lib (F:\src\os2\uniaud32t\alsa-kernel\pci\hda\hda_proc.c)
	at offset 00086134 000AEH bytes from F:\src\os2\uniaud32t\lib\Debug.ACP\sequencer.lib (F:\src\os2\uniaud32t\alsa-kernel\core\seq\seq.c)
	at offset 000861E2 00BA2H bytes from F:\src\os2\uniaud32t\lib\Debug.ACP\sequencer.lib (F:\src\os2\uniaud32t\alsa-kernel\core\seq\seq_device.c)
	at offset 00086D84 00117H bytes from F:\src\os2\uniaud32t\lib\Debug.ACP\sequencer.lib (F:\src\os2\uniaud32t\alsa-kernel\core\seq\seq_info.c)
	at offset 00086E9B 00317H bytes from F:\src\os2\uniaud32t\lib\Debug.ACP\sequencer.lib (F:\src\os2\uniaud32t\alsa-kernel\core\seq\seq_system.c)
	at offset 000871B2 01427H bytes from F:\src\os2\uniaud32t\lib\Debug.ACP\sequencer.lib (F:\src\os2\uniaud32t\alsa-kernel\core\seq\seq_queue.c)
	at offset 000885D9 00CF0H bytes from F:\src\os2\uniaud32t\lib\Debug.ACP\sequencer.lib (F:\src\os2\uniaud32t\alsa-kernel\core\seq\seq_memory.c)
	at offset 000892C9 03EBAH bytes from F:\src\os2\uniaud32t\lib\Debug.ACP\sequencer.lib (F:\src\os2\uniaud32t\alsa-kernel\core\seq\seq_clientmgr.c)
	at offset 0008D183 01515H bytes from F:\src\os2\uniaud32t\lib\Debug.ACP\sequencer.lib (F:\src\os2\uniaud32t\alsa-kernel\core\seq\seq_ports.c)
	at offset 0008E698 00CC8H bytes from F:\src\os2\uniaud32t\lib\Debug.ACP\sequencer.lib (F:\src\os2\uniaud32t\alsa-kernel\core\seq\seq_timer.c)
	at offset 0008F360 00A34H bytes from F:\src\os2\uniaud32t\lib\Debug.ACP\sequencer.lib (F:\src\os2\uniaud32t\alsa-kernel\core\seq\seq_prioq.c)
	at offset 0008FD94 0061FH bytes from F:\src\os2\uniaud32t\lib\Debug.ACP\sequencer.lib (F:\src\os2\uniaud32t\alsa-kernel\core\seq\seq_fifo.c)
	at offset 000903B3 006F7H bytes from F:\src\os2\uniaud32t\lib\Debug.ACP\opl3.lib (F:\src\os2\uniaud32t\alsa-kernel\drivers\opl3\opl3_seq.c)
	at offset 00090AAA 00D69H bytes from F:\src\os2\uniaud32t\lib\Debug.ACP\opl3.lib (F:\src\os2\uniaud32t\alsa-kernel\drivers\opl3\opl3_lib.c)
	at offset 00091813 003D2H bytes from F:\src\os2\uniaud32t\lib\Debug.ACP\opl3.lib (F:\src\os2\uniaud32t\alsa-kernel\drivers\opl3\opl3_drums.c)
	at offset 00091BE5 01237H bytes from F:\src\os2\uniaud32t\lib\Debug.ACP\opl3.lib (F:\src\os2\uniaud32t\alsa-kernel\drivers\opl3\opl3_midi.c)
	at offset 00092E1C 00D57H bytes from F:\src\os2\uniaud32t\lib\Debug.ACP\opl3.lib (F:\src\os2\uniaud32t\alsa-kernel\drivers\opl3\opl3_synth.c)
	at offset 00093B73 00F18H bytes from F:\src\os2\uniaud32t\lib\Debug.ACP\mpu401.lib (F:\src\os2\uniaud32t\alsa-kernel\drivers\mpu401\mpu401_uart.c)
	at offset 00094A8B 002D4H bytes from F:\src\os2\uniaud32t\lib\Debug.ACP\cs46xx.lib (F:\src\os2\uniaud32t\alsa-kernel\pci\cs46xx\cs46xx.c)
	at offset 00094D5F 04659H bytes from F:\src\os2\uniaud32t\lib\Debug.ACP\cs46xx.lib (F:\src\os2\uniaud32t\alsa-kernel\pci\cs46xx\cs46xx_lib.c)
	at offset 000993B8 00956H bytes from F:\src\os2\uniaud32t\lib\Debug.ACP\cs5535audio.lib (F:\src\os2\uniaud32t\alsa-kernel\pci\cs5535audio\cs5535audio.c)
	at offset 00099D0E 002B3H bytes from F:\src\os2\uniaud32t\lib\Debug.ACP\cs5535audio.lib (F:\src\os2\uniaud32t\alsa-kernel\pci\cs5535audio\cs5535audio_pm.c)
	at offset 00099FC1 00B55H bytes from F:\src\os2\uniaud32t\lib\Debug.ACP\cs5535audio.lib (F:\src\os2\uniaud32t\alsa-kernel\pci\cs5535audio\cs5535audio_pcm.c)
	at offset 0009AB16 0068EH bytes from F:\src\os2\uniaud32t\lib\Debug.ACP\emu10k1.lib (F:\src\os2\uniaud32t\alsa-kernel\pci\emu10k1\emu10k1.c)
	at offset 0009B1A4 015ABH bytes from F:\src\os2\uniaud32t\lib\Debug.ACP\emu10k1.lib (F:\src\os2\uniaud32t\alsa-kernel\pci\emu10k1\p16v.c)
	at offset 0009C74F 001E4H bytes from F:\src\os2\uniaud32t\lib\Debug.ACP\emu10k1.lib (F:\src\os2\uniaud32t\alsa-kernel\pci\emu10k1\timer.c)
	at offset 0009C933 082E8H bytes from F:\src\os2\uniaud32t\lib\Debug.ACP\emu10k1.lib (F:\src\os2\uniaud32t\alsa-kernel\pci\emu10k1\emufx.c)
	at offset 000A4C1B 03247H bytes from F:\src\os2\uniaud32t\lib\Debug.ACP\emu10k1.lib (F:\src\os2\uniaud32t\alsa-kernel\pci\emu10k1\emumixer.c)
	at offset 000A7E62 03D6CH bytes from F:\src\os2\uniaud32t\lib\Debug.ACP\emu10k1.lib (F:\src\os2\uniaud32t\alsa-kernel\pci\emu10k1\emupcm.c)
	at offset 000ABBCE 00B31H bytes from F:\src\os2\uniaud32t\lib\Debug.ACP\emu10k1.lib (F:\src\os2\uniaud32t\alsa-kernel\pci\emu10k1\emumpu401.c)
	at offset 000AC6FF 02999H bytes from F:\src\os2\uniaud32t\lib\Debug.ACP\emu10k1.lib (F:\src\os2\uniaud32t\alsa-kernel\pci\emu10k1\emu10k1_main.c)
	at offset 000AF098 00FB4H bytes from F:\src\os2\uniaud32t\lib\Debug.ACP\emu10k1.lib (F:\src\os2\uniaud32t\alsa-kernel\pci\emu10k1\emuproc.c)
	at offset 000B004C 00F59H bytes from F:\src\os2\uniaud32t\lib\Debug.ACP\emu10k1.lib (F:\src\os2\uniaud32t\alsa-kernel\pci\emu10k1\io.c)
	at offset 000B0FA5 00431H bytes from F:\src\os2\uniaud32t\lib\Debug.ACP\emu10k1.lib (F:\src\os2\uniaud32t\alsa-kernel\pci\emu10k1\voice.c)
	at offset 000B13D6 00F44H bytes from F:\src\os2\uniaud32t\lib\Debug.ACP\emu10k1.lib (F:\src\os2\uniaud32t\alsa-kernel\pci\emu10k1\memory.c)
	at offset 000B231A 00551H bytes from F:\src\os2\uniaud32t\lib\Debug.ACP\emu10k1.lib (F:\src\os2\uniaud32t\alsa-kernel\pci\emu10k1\irq.c)
	at offset 000B286B 0088FH bytes from F:\src\os2\uniaud32t\lib\Debug.ACP\ymfpci.lib (F:\src\os2\uniaud32t\alsa-kernel\pci\ymfpci\ymfpci.c)
	at offset 000B30FA 059D0H bytes from F:\src\os2\uniaud32t\lib\Debug.ACP\ymfpci.lib (F:\src\os2\uniaud32t\alsa-kernel\pci\ymfpci\ymfpci_main.c)
	at offset 000B8ACA 036E7H bytes from F:\src\os2\uniaud32t\lib\Debug.ACP\ali5451.lib (F:\src\os2\uniaud32t\alsa-kernel\pci\ali5451\ali5451.c)
	at offset 000BC1B1 00408H bytes from F:\src\os2\uniaud32t\lib\Debug.ACP\trident.lib (F:\src\os2\uniaud32t\alsa-kernel\pci\trident\trident.c)
	at offset 000BC5B9 05EE0H bytes from F:\src\os2\uniaud32t\lib\Debug.ACP\trident.lib (F:\src\os2\uniaud32t\alsa-kernel\pci\trident\trident_main.c)
	at offset 000C2499 00636H bytes from F:\src\os2\uniaud32t\lib\Debug.ACP\trident.lib (F:\src\os2\uniaud32t\alsa-kernel\pci\trident\trident_memory.c)
	at offset 000C2ACF 02924H bytes from F:\src\os2\uniaud32t\lib\Debug.ACP\nm256.lib (F:\src\os2\uniaud32t\alsa-kernel\pci\nm256\nm256.c)
	at offset 000C53F3 01473H bytes from F:\src\os2\uniaud32t\lib\Debug.ACP\sb.lib (F:\src\os2\uniaud32t\alsa-kernel\isa\sb\sb_mixer.c)
	at offset 000C6866 006C8H bytes from F:\src\os2\uniaud32t\lib\Debug.ACP\sb.lib (F:\src\os2\uniaud32t\alsa-kernel\isa\sb\sb_common.c)
	at offset 000C6F2E 068BBH bytes from F:\src\os2\uniaud32t\lib\Debug.ACP\core_oss.lib (F:\src\os2\uniaud32t\alsa-kernel\core\oss\pcm_oss.c)
	at offset 000CD800 00140H bytes from F:\acpi\lib\acpidrv.lib (acpi)
	at offset 000CD940 002BCH bytes from F:\acpi\lib\acpidrv.lib (FindAddress)
	at offset 000CDBFC 0010CH bytes from F:\src\os2\uniaud32t\lib\Debug.ACP\linuxlib.lib (F:\src\os2\uniaud32t\lib32\semaphore.c)
	at offset 000CDD08 00A73H bytes from F:\src\os2\uniaud32t\lib\Debug.ACP\core.lib (F:\src\os2\uniaud32t\alsa-kernel\core\vmaster.c)
	at offset 000CE77B 000B9H bytes from F:\src\os2\uniaud32t\lib\Debug.ACP\core.lib (F:\src\os2\uniaud32t\alsa-kernel\core\misc.c)
	at offset 000CE834 00160H bytes from F:\src\os2\uniaud32t\lib\Debug.ACP\core.lib (F:\src\os2\uniaud32t\alsa-kernel\core\memory.c)
	at offset 000CE994 0136CH bytes from F:\src\os2\uniaud32t\lib\Debug.ACP\ac97.lib (F:\src\os2\uniaud32t\alsa-kernel\pci\ac97\ac97_pcm.c)
	at offset 000CFD00 0B499H bytes from F:\src\os2\uniaud32t\lib\Debug.ACP\ac97.lib (F:\src\os2\uniaud32t\alsa-kernel\pci\ac97\ac97_codec.c)
	at offset 000DB199 019D7H bytes from F:\src\os2\uniaud32t\lib\Debug.ACP\ac97.lib (F:\src\os2\uniaud32t\alsa-kernel\pci\ac97\ac97_proc.c)
	at offset 000DCB70 010BDH bytes from F:\src\os2\uniaud32t\lib\Debug.ACP\sequencer.lib (F:\src\os2\uniaud32t\alsa-kernel\core\seq\seq_midi_emul.c)
	at offset 000DDC2D 00452H bytes from F:\src\os2\uniaud32t\lib\Debug.ACP\synth.lib (F:\src\os2\uniaud32t\alsa-kernel\synth\util_mem.c)

 0003:000DE080 0000029A6H _TEXT                  CODE 32-bit
	at offset 00000000 0004FH bytes from E:\watcom\lib386\os2\clib3r.lib (i8s)
	at offset 00000050 0001CH bytes from E:\watcom\lib386\os2\clib3r.lib (i8m)
	at offset 00000070 000ADH bytes from E:\watcom\lib386\os2\clib3r.lib (strstr.c)
	at offset 00000120 00041H bytes from E:\watcom\lib386\os2\clib3r.lib (strlcpy.c)
	at offset 00000170 00091H bytes from E:\watcom\lib386\os2\clib3r.lib (sscanf.c)
	at offset 00000210 000C7H bytes from E:\watcom\lib386\os2\clib3r.lib (snprintf.c)
	at offset 000002E0 00018H bytes from E:\watcom\lib386\os2\clib3r.lib (memset.c)
	at offset 00000300 00053H bytes from E:\watcom\lib386\os2\clib3r.lib (memmove.c)
	at offset 00000360 0023DH bytes from E:\watcom\lib386\os2\clib3r.lib (strtol.c)
	at offset 000005A0 00101H bytes from E:\watcom\lib386\os2\clib3r.lib (istable.c)
	at offset 000006B0 000A3H bytes from E:\watcom\lib386\os2\clib3r.lib (__stos)
	at offset 00000760 00DCBH bytes from E:\watcom\lib386\os2\clib3r.lib (scnf.c)
	at offset 00001530 00CE4H bytes from E:\watcom\lib386\os2\clib3r.lib (prtf.c)
	at offset 00002214 0004BH bytes from E:\watcom\lib386\os2\clib3r.lib (seterrno.c)
	at offset 00002260 0000EH bytes from E:\watcom\lib386\os2\clib3r.lib (tolower.c)
	at offset 00002270 0004CH bytes from E:\watcom\lib386\os2\clib3r.lib (fdfs386)
	at offset 000022C0 00020H bytes from E:\watcom\lib386\os2\clib3r.lib (strupr.c)
	at offset 000022E0 00008H bytes from E:\watcom\lib386\os2\clib3r.lib (bits.c)
	at offset 000022F0 00042H bytes from E:\watcom\lib386\os2\clib3r.lib (noefgfmt.c)
	at offset 00002332 00128H bytes from E:\watcom\lib386\os2\clib3r.lib (maino32.c)
	at offset 00002460 0002EH bytes from E:\watcom\lib386\os2\clib3r.lib (wctomb.c)
	at offset 00002490 000BCH bytes from E:\watcom\lib386\os2\clib3r.lib (mbtowc.c)
	at offset 00002550 00017H bytes from E:\watcom\lib386\os2\clib3r.lib (mbislead.c)
	at offset 00002570 00074H bytes from E:\watcom\lib386\os2\clib3r.lib (ltoa.c)
	at offset 000025F0 00099H bytes from E:\watcom\lib386\os2\clib3r.lib (lltoa.c)
	at offset 00002690 00074H bytes from E:\watcom\lib386\os2\clib3r.lib (itoa.c)
	at offset 00002710 00070H bytes from E:\watcom\lib386\os2\clib3r.lib (xmsgo32.c)
	at offset 00002780 000B3H bytes from E:\watcom\lib386\os2\clib3r.lib (initrtns.c)
	at offset 00002833 00001H bytes from E:\watcom\lib386\os2\clib3r.lib (crwdata)
	at offset 00002840 0000BH bytes from E:\watcom\lib386\os2\clib3r.lib (cinit.c)
	at offset 0000284B 00132H bytes from E:\watcom\lib386\os2\clib3r.lib (mbinit.c)
	at offset 00002980 00026H bytes from E:\watcom\lib386\os2\clib3r.lib (enterdb.c)

 0003:000E0A28 000000000H LASTCODE32             CODE 32-bit

 0004:00000000 000000007H BEGTEXT                CODE 32-bit
	at offset 00000000 00007H bytes from E:\watcom\lib386\os2\clib3r.lib (segdefns)

 0005:00000000 000000030H BSS32                  BSS 32-bit
	at offset 00000000 00004H bytes from F:\src\os2\uniaud32t\drv32\bin\Debug.ACP\begin.obj (begin.asm)
	at offset 00000004 0002CH bytes from F:\acpi\lib\acpidrv.lib (acpi)

 0005:00000030 000001728H _BSS                   BSS 32-bit
	at offset 00000000 00008H bytes from F:\src\os2\uniaud32t\drv32\bin\Debug.ACP\strategy.obj (F:\src\os2\uniaud32t\drv32\strategy.c)
	at offset 00000008 0000CH bytes from F:\src\os2\uniaud32t\drv32\bin\Debug.ACP\read.obj (F:\src\os2\uniaud32t\drv32\read.cpp)
	at offset 00000014 00008H bytes from F:\src\os2\uniaud32t\drv32\bin\Debug.ACP\parse.obj (F:\src\os2\uniaud32t\drv32\parse.c)
	at offset 0000001C 00006H bytes from F:\src\os2\uniaud32t\drv32\bin\Debug.ACP\idc.obj (F:\src\os2\uniaud32t\drv32\idc.c)
	at offset 00000024 0005CH bytes from F:\src\os2\uniaud32t\drv32\bin\Debug.ACP\rmhelp.obj (F:\src\os2\uniaud32t\drv32\rmhelp.cpp)
	at offset 00000080 00028H bytes from F:\src\os2\uniaud32t\lib\Debug.ACP\linuxlib.lib (F:\src\os2\uniaud32t\lib32\ossidc.cpp)
	at offset 000000A8 00028H bytes from F:\src\os2\uniaud32t\lib\Debug.ACP\linuxlib.lib (F:\src\os2\uniaud32t\lib32\debug.c)
	at offset 000000D0 00008H bytes from F:\src\os2\uniaud32t\lib\Debug.ACP\linuxlib.lib (F:\src\os2\uniaud32t\lib32\memory.cpp)
	at offset 000000D8 00440H bytes from F:\src\os2\uniaud32t\lib\Debug.ACP\linuxlib.lib (F:\src\os2\uniaud32t\lib32\pci.c)
	at offset 00000518 0002CH bytes from F:\src\os2\uniaud32t\lib\Debug.ACP\linuxlib.lib (F:\src\os2\uniaud32t\lib32\malloc.cpp)
	at offset 00000544 00004H bytes from F:\src\os2\uniaud32t\lib\Debug.ACP\core.lib (F:\src\os2\uniaud32t\alsa-kernel\core\hwdep.c)
	at offset 00000548 00004H bytes from F:\src\os2\uniaud32t\lib\Debug.ACP\core.lib (F:\src\os2\uniaud32t\alsa-kernel\core\timer.c)
	at offset 0000054C 00020H bytes from F:\src\os2\uniaud32t\lib\Debug.ACP\core.lib (F:\src\os2\uniaud32t\alsa-kernel\core\rawmidi.c)
	at offset 0000056C 00104H bytes from F:\src\os2\uniaud32t\lib\Debug.ACP\core.lib (F:\src\os2\uniaud32t\alsa-kernel\core\pcm.c)
	at offset 00000670 0040CH bytes from F:\src\os2\uniaud32t\lib\Debug.ACP\core.lib (F:\src\os2\uniaud32t\alsa-kernel\core\sound.c)
	at offset 00000A7C 00010H bytes from F:\src\os2\uniaud32t\lib\Debug.ACP\core.lib (F:\src\os2\uniaud32t\alsa-kernel\core\info.c)
	at offset 00000A8C 000C4H bytes from F:\src\os2\uniaud32t\lib\Debug.ACP\core.lib (F:\src\os2\uniaud32t\alsa-kernel\core\info_oss.c)
	at offset 00000B50 00204H bytes from F:\src\os2\uniaud32t\lib\Debug.ACP\core.lib (F:\src\os2\uniaud32t\alsa-kernel\core\sound_oss.c)
	at offset 00000D54 00004H bytes from F:\src\os2\uniaud32t\lib\Debug.ACP\core.lib (F:\src\os2\uniaud32t\alsa-kernel\core\memalloc.c)
	at offset 00000D58 0004CH bytes from F:\src\os2\uniaud32t\lib\Debug.ACP\core.lib (F:\src\os2\uniaud32t\alsa-kernel\core\init.c)
	at offset 00000DA4 00028H bytes from F:\src\os2\uniaud32t\lib\Debug.ACP\pci.lib (F:\src\os2\uniaud32t\alsa-kernel\pci\bt87x.c)
	at offset 00000DCC 00004H bytes from F:\src\os2\uniaud32t\lib\Debug.ACP\pci.lib (F:\src\os2\uniaud32t\alsa-kernel\pci\als4000.c)
	at offset 00000DD0 00024H bytes from F:\src\os2\uniaud32t\lib\Debug.ACP\pci.lib (F:\src\os2\uniaud32t\alsa-kernel\pci\cmipci.c)
	at offset 00000DF4 00008H bytes from F:\src\os2\uniaud32t\lib\Debug.ACP\pci.lib (F:\src\os2\uniaud32t\alsa-kernel\pci\atiixp.c)
	at offset 00000DFC 00024H bytes from F:\src\os2\uniaud32t\lib\Debug.ACP\pci.lib (F:\src\os2\uniaud32t\alsa-kernel\pci\fm801.c)
	at offset 00000E20 00014H bytes from F:\src\os2\uniaud32t\lib\Debug.ACP\pci.lib (F:\src\os2\uniaud32t\alsa-kernel\pci\via82xx.c)
	at offset 00000E34 00004H bytes from F:\src\os2\uniaud32t\lib\Debug.ACP\pci.lib (F:\src\os2\uniaud32t\alsa-kernel\pci\maestro3.c)
	at offset 00000E38 00018H bytes from F:\src\os2\uniaud32t\lib\Debug.ACP\pci.lib (F:\src\os2\uniaud32t\alsa-kernel\pci\intel8x0.c)
	at offset 00000E50 00024H bytes from F:\src\os2\uniaud32t\lib\Debug.ACP\pci.lib (F:\src\os2\uniaud32t\alsa-kernel\pci\es1968.c)
	at offset 00000E74 00004H bytes from F:\src\os2\uniaud32t\lib\Debug.ACP\pci.lib (F:\src\os2\uniaud32t\alsa-kernel\pci\es1938.c)
	at offset 00000E78 00024H bytes from F:\src\os2\uniaud32t\lib\Debug.ACP\pci.lib (F:\src\os2\uniaud32t\alsa-kernel\pci\cs4281.c)
	at offset 00000E9C 00044H bytes from F:\src\os2\uniaud32t\lib\Debug.ACP\pci.lib (F:\src\os2\uniaud32t\alsa-kernel\pci\ens1371.c)
	at offset 00000EE0 00024H bytes from F:\src\os2\uniaud32t\lib\Debug.ACP\ca0106.lib (F:\src\os2\uniaud32t\alsa-kernel\pci\ca0106\ca0106_main.c)
	at offset 00000F04 00008H bytes from F:\src\os2\uniaud32t\lib\Debug.ACP\hda.lib (F:\src\os2\uniaud32t\alsa-kernel\pci\hda\patch_sigmatel.c)
	at offset 00000F0C 0006CH bytes from F:\src\os2\uniaud32t\lib\Debug.ACP\hda.lib (F:\src\os2\uniaud32t\alsa-kernel\pci\hda\hda_intel.c)
	at offset 00000F78 00008H bytes from F:\src\os2\uniaud32t\lib\Debug.ACP\sequencer.lib (F:\src\os2\uniaud32t\alsa-kernel\core\seq\seq_device.c)
	at offset 00000F80 0000CH bytes from F:\src\os2\uniaud32t\lib\Debug.ACP\sequencer.lib (F:\src\os2\uniaud32t\alsa-kernel\core\seq\seq_info.c)
	at offset 00000F8C 00024H bytes from F:\src\os2\uniaud32t\lib\Debug.ACP\sequencer.lib (F:\src\os2\uniaud32t\alsa-kernel\core\seq\seq_queue.c)
	at offset 00000FB0 003C8H bytes from F:\src\os2\uniaud32t\lib\Debug.ACP\sequencer.lib (F:\src\os2\uniaud32t\alsa-kernel\core\seq\seq_clientmgr.c)
	at offset 00001378 00044H bytes from F:\src\os2\uniaud32t\lib\Debug.ACP\cs46xx.lib (F:\src\os2\uniaud32t\alsa-kernel\pci\cs46xx\cs46xx.c)
	at offset 000013BC 00008H bytes from F:\src\os2\uniaud32t\lib\Debug.ACP\cs5535audio.lib (F:\src\os2\uniaud32t\alsa-kernel\pci\cs5535audio\cs5535audio.c)
	at offset 000013C4 00084H bytes from F:\src\os2\uniaud32t\lib\Debug.ACP\emu10k1.lib (F:\src\os2\uniaud32t\alsa-kernel\pci\emu10k1\emu10k1.c)
	at offset 00001448 00064H bytes from F:\src\os2\uniaud32t\lib\Debug.ACP\ymfpci.lib (F:\src\os2\uniaud32t\alsa-kernel\pci\ymfpci\ymfpci.c)
	at offset 000014AC 00008H bytes from F:\src\os2\uniaud32t\lib\Debug.ACP\ali5451.lib (F:\src\os2\uniaud32t\alsa-kernel\pci\ali5451\ali5451.c)
	at offset 000014B4 00004H bytes from F:\src\os2\uniaud32t\lib\Debug.ACP\trident.lib (F:\src\os2\uniaud32t\alsa-kernel\pci\trident\trident.c)
	at offset 000014B8 0001CH bytes from F:\src\os2\uniaud32t\lib\Debug.ACP\nm256.lib (F:\src\os2\uniaud32t\alsa-kernel\pci\nm256\nm256.c)
	at offset 000014D4 00020H bytes from F:\src\os2\uniaud32t\lib\Debug.ACP\core_oss.lib (F:\src\os2\uniaud32t\alsa-kernel\core\oss\pcm_oss.c)
	at offset 000014F4 00106H bytes from E:\watcom\lib386\os2\clib3r.lib (maino32.c)
	at offset 000015FC 00101H bytes from E:\watcom\lib386\os2\clib3r.lib (mbislead.c)
	at offset 00001700 00004H bytes from E:\watcom\lib386\os2\clib3r.lib (mbisdbcs.c)
	at offset 00001704 00004H bytes from E:\watcom\lib386\os2\clib3r.lib (cinit.c)
	at offset 00001708 00020H bytes from F:\src\os2\uniaud32t\lib\Debug.ACP\ac97.lib (F:\src\os2\uniaud32t\alsa-kernel\pci\ac97\ac97_codec.c)

 0005:00001758 000000000H C_COMMON               DATA 32-bit

 0005:00001758 000000010H c_common               DATA 32-bit
	at offset 00000000 00010H bytes from F:\acpi\lib\acpidrv.lib (acpi)

 0005:00001768 000000098H DATA32                 DATA 32-bit
	at offset 00000000 0008AH bytes from F:\src\os2\uniaud32t\drv32\bin\Debug.ACP\startup.obj (startup.asm)
	at offset 0000008C 0000CH bytes from F:\src\os2\uniaud32t\drv32\bin\Debug.ACP\devhlp.obj (devhlp.asm)

 0005:00001800 00005EF4CH _DATA                  DATA 32-bit
	at offset 00000000 00080H bytes from F:\src\os2\uniaud32t\drv32\bin\Debug.ACP\strategy.obj (F:\src\os2\uniaud32t\drv32\strategy.c)
	at offset 00000080 00018H bytes from F:\src\os2\uniaud32t\drv32\bin\Debug.ACP\parse.obj (F:\src\os2\uniaud32t\drv32\parse.c)
	at offset 00000098 00004H bytes from F:\src\os2\uniaud32t\drv32\bin\Debug.ACP\rmhelp.obj (F:\src\os2\uniaud32t\drv32\rmhelp.cpp)
	at offset 0000009C 00020H bytes from F:\src\os2\uniaud32t\drv32\bin\Debug.ACP\irq.obj (F:\src\os2\uniaud32t\drv32\irq.cpp)
	at offset 000000BC 0000CH bytes from F:\src\os2\uniaud32t\lib\Debug.ACP\linuxlib.lib (F:\src\os2\uniaud32t\lib32\timer.c)
	at offset 000000C8 00028H bytes from F:\src\os2\uniaud32t\lib\Debug.ACP\linuxlib.lib (F:\src\os2\uniaud32t\lib32\task.c)
	at offset 000000F0 00414H bytes from F:\src\os2\uniaud32t\lib\Debug.ACP\linuxlib.lib (F:\src\os2\uniaud32t\lib32\misc.c)
	at offset 00000504 00108H bytes from F:\src\os2\uniaud32t\lib\Debug.ACP\linuxlib.lib (F:\src\os2\uniaud32t\lib32\ossidc.cpp)
	at offset 0000060C 00004H bytes from F:\src\os2\uniaud32t\lib\Debug.ACP\linuxlib.lib (F:\src\os2\uniaud32t\lib32\soundmidi.c)
	at offset 00000610 001F1H bytes from F:\src\os2\uniaud32t\lib\Debug.ACP\linuxlib.lib (F:\src\os2\uniaud32t\lib32\soundmixer.c)
	at offset 00000804 061D8H bytes from F:\src\os2\uniaud32t\lib\Debug.ACP\linuxlib.lib (F:\src\os2\uniaud32t\lib32\sound.c)
	at offset 000069DC 00013H bytes from F:\src\os2\uniaud32t\lib\Debug.ACP\linuxlib.lib (F:\src\os2\uniaud32t\lib32\debug.c)
	at offset 000069F0 0202CH bytes from F:\src\os2\uniaud32t\lib\Debug.ACP\linuxlib.lib (F:\src\os2\uniaud32t\lib32\ioctl.c)
	at offset 00008A1C 00880H bytes from F:\src\os2\uniaud32t\lib\Debug.ACP\linuxlib.lib (F:\src\os2\uniaud32t\lib32\irq.c)
	at offset 0000929C 03F44H bytes from F:\src\os2\uniaud32t\lib\Debug.ACP\linuxlib.lib (F:\src\os2\uniaud32t\lib32\pci.c)
	at offset 0000D1E0 00004H bytes from F:\src\os2\uniaud32t\lib\Debug.ACP\linuxlib.lib (F:\src\os2\uniaud32t\lib32\malloc.cpp)
	at offset 0000D1E4 00068H bytes from F:\src\os2\uniaud32t\lib\Debug.ACP\core.lib (F:\src\os2\uniaud32t\alsa-kernel\core\hwdep.c)
	at offset 0000D24C 000ACH bytes from F:\src\os2\uniaud32t\lib\Debug.ACP\core.lib (F:\src\os2\uniaud32t\alsa-kernel\core\timer.c)
	at offset 0000D2F8 00090H bytes from F:\src\os2\uniaud32t\lib\Debug.ACP\core.lib (F:\src\os2\uniaud32t\alsa-kernel\core\rawmidi.c)
	at offset 0000D388 00210H bytes from F:\src\os2\uniaud32t\lib\Debug.ACP\core.lib (F:\src\os2\uniaud32t\alsa-kernel\core\pcm_misc.c)
	at offset 0000D598 000A0H bytes from F:\src\os2\uniaud32t\lib\Debug.ACP\core.lib (F:\src\os2\uniaud32t\alsa-kernel\core\pcm_lib.c)
	at offset 0000D638 00030H bytes from F:\src\os2\uniaud32t\lib\Debug.ACP\core.lib (F:\src\os2\uniaud32t\alsa-kernel\core\pcm.c)
	at offset 0000D668 0005CH bytes from F:\src\os2\uniaud32t\lib\Debug.ACP\core.lib (F:\src\os2\uniaud32t\alsa-kernel\core\sound.c)
	at offset 0000D6C4 00048H bytes from F:\src\os2\uniaud32t\lib\Debug.ACP\core.lib (F:\src\os2\uniaud32t\alsa-kernel\core\info.c)
	at offset 0000D70C 00008H bytes from F:\src\os2\uniaud32t\lib\Debug.ACP\core.lib (F:\src\os2\uniaud32t\alsa-kernel\core\pcm_memory.c)
	at offset 0000D714 00030H bytes from F:\src\os2\uniaud32t\lib\Debug.ACP\core.lib (F:\src\os2\uniaud32t\alsa-kernel\core\pcm_timer.c)
	at offset 0000D744 00144H bytes from F:\src\os2\uniaud32t\lib\Debug.ACP\core.lib (F:\src\os2\uniaud32t\alsa-kernel\core\pcm_native.c)
	at offset 0000D888 0000CH bytes from F:\src\os2\uniaud32t\lib\Debug.ACP\core.lib (F:\src\os2\uniaud32t\alsa-kernel\core\info_oss.c)
	at offset 0000D894 0000CH bytes from F:\src\os2\uniaud32t\lib\Debug.ACP\core.lib (F:\src\os2\uniaud32t\alsa-kernel\core\sound_oss.c)
	at offset 0000D8A0 00060H bytes from F:\src\os2\uniaud32t\lib\Debug.ACP\core.lib (F:\src\os2\uniaud32t\alsa-kernel\core\control.c)
	at offset 0000D900 0001CH bytes from F:\src\os2\uniaud32t\lib\Debug.ACP\core.lib (F:\src\os2\uniaud32t\alsa-kernel\core\memalloc.c)
	at offset 0000D91C 00058H bytes from F:\src\os2\uniaud32t\lib\Debug.ACP\core.lib (F:\src\os2\uniaud32t\alsa-kernel\core\init.c)
	at offset 0000D974 00408H bytes from F:\src\os2\uniaud32t\lib\Debug.ACP\pci.lib (F:\src\os2\uniaud32t\alsa-kernel\pci\bt87x.c)
	at offset 0000DD7C 0019CH bytes from F:\src\os2\uniaud32t\lib\Debug.ACP\pci.lib (F:\src\os2\uniaud32t\alsa-kernel\pci\als4000.c)
	at offset 0000DF18 00E61H bytes from F:\src\os2\uniaud32t\lib\Debug.ACP\pci.lib (F:\src\os2\uniaud32t\alsa-kernel\pci\cmipci.c)
	at offset 0000ED7C 003A8H bytes from F:\src\os2\uniaud32t\lib\Debug.ACP\pci.lib (F:\src\os2\uniaud32t\alsa-kernel\pci\atiixp.c)
	at offset 0000F124 004C0H bytes from F:\src\os2\uniaud32t\lib\Debug.ACP\pci.lib (F:\src\os2\uniaud32t\alsa-kernel\pci\fm801.c)
	at offset 0000F5E4 006B8H bytes from F:\src\os2\uniaud32t\lib\Debug.ACP\pci.lib (F:\src\os2\uniaud32t\alsa-kernel\pci\via82xx.c)
	at offset 0000FC9C 00744H bytes from F:\src\os2\uniaud32t\lib\Debug.ACP\pci.lib (F:\src\os2\uniaud32t\alsa-kernel\pci\maestro3.c)
	at offset 000103E0 00F94H bytes from F:\src\os2\uniaud32t\lib\Debug.ACP\pci.lib (F:\src\os2\uniaud32t\alsa-kernel\pci\intel8x0.c)
	at offset 00011374 002B4H bytes from F:\src\os2\uniaud32t\lib\Debug.ACP\pci.lib (F:\src\os2\uniaud32t\alsa-kernel\pci\es1968.c)
	at offset 00011628 00899H bytes from F:\src\os2\uniaud32t\lib\Debug.ACP\pci.lib (F:\src\os2\uniaud32t\alsa-kernel\pci\es1938.c)
	at offset 00011EC4 002D0H bytes from F:\src\os2\uniaud32t\lib\Debug.ACP\pci.lib (F:\src\os2\uniaud32t\alsa-kernel\pci\cs4281.c)
	at offset 00012194 0049CH bytes from F:\src\os2\uniaud32t\lib\Debug.ACP\pci.lib (F:\src\os2\uniaud32t\alsa-kernel\pci\ens1371.c)
	at offset 00012630 004ECH bytes from F:\src\os2\uniaud32t\lib\Debug.ACP\ca0106.lib (F:\src\os2\uniaud32t\alsa-kernel\pci\ca0106\ca0106_main.c)
	at offset 00012B1C 00020H bytes from F:\src\os2\uniaud32t\lib\Debug.ACP\ca0106.lib (F:\src\os2\uniaud32t\alsa-kernel\pci\ca0106\ca_midi.c)
	at offset 00012B3C 00634H bytes from F:\src\os2\uniaud32t\lib\Debug.ACP\ca0106.lib (F:\src\os2\uniaud32t\alsa-kernel\pci\ca0106\ca0106_mixer.c)
	at offset 00013170 00058H bytes from F:\src\os2\uniaud32t\lib\Debug.ACP\ca0106.lib (F:\src\os2\uniaud32t\alsa-kernel\pci\ca0106\ca0106_proc.c)
	at offset 000131C8 01668H bytes from F:\src\os2\uniaud32t\lib\Debug.ACP\hda.lib (F:\src\os2\uniaud32t\alsa-kernel\pci\hda\patch_via.c)
	at offset 00014830 01E88H bytes from F:\src\os2\uniaud32t\lib\Debug.ACP\hda.lib (F:\src\os2\uniaud32t\alsa-kernel\pci\hda\patch_conexant.c)
	at offset 000166B8 0015CH bytes from F:\src\os2\uniaud32t\lib\Debug.ACP\hda.lib (F:\src\os2\uniaud32t\alsa-kernel\pci\hda\patch_atihdmi.c)
	at offset 00016814 03166H bytes from F:\src\os2\uniaud32t\lib\Debug.ACP\hda.lib (F:\src\os2\uniaud32t\alsa-kernel\pci\hda\patch_sigmatel.c)
	at offset 0001997C 075E4H bytes from F:\src\os2\uniaud32t\lib\Debug.ACP\hda.lib (F:\src\os2\uniaud32t\alsa-kernel\pci\hda\patch_analog.c)
	at offset 00020F60 007A0H bytes from F:\src\os2\uniaud32t\lib\Debug.ACP\hda.lib (F:\src\os2\uniaud32t\alsa-kernel\pci\hda\patch_cmedia.c)
	at offset 00021700 1D0D1H bytes from F:\src\os2\uniaud32t\lib\Debug.ACP\hda.lib (F:\src\os2\uniaud32t\alsa-kernel\pci\hda\patch_realtek.c)
	at offset 0003E7D4 00664H bytes from F:\src\os2\uniaud32t\lib\Debug.ACP\hda.lib (F:\src\os2\uniaud32t\alsa-kernel\pci\hda\hda_intel.c)
	at offset 0003EE38 00447H bytes from F:\src\os2\uniaud32t\lib\Debug.ACP\hda.lib (F:\src\os2\uniaud32t\alsa-kernel\pci\hda\hda_codec.c)
	at offset 0003F280 0008CH bytes from F:\src\os2\uniaud32t\lib\Debug.ACP\hda.lib (F:\src\os2\uniaud32t\alsa-kernel\pci\hda\hda_generic.c)
	at offset 0003F30C 000E0H bytes from F:\src\os2\uniaud32t\lib\Debug.ACP\hda.lib (F:\src\os2\uniaud32t\alsa-kernel\pci\hda\hda_proc.c)
	at offset 0003F3EC 0005CH bytes from F:\src\os2\uniaud32t\lib\Debug.ACP\sequencer.lib (F:\src\os2\uniaud32t\alsa-kernel\core\seq\seq.c)
	at offset 0003F448 00028H bytes from F:\src\os2\uniaud32t\lib\Debug.ACP\sequencer.lib (F:\src\os2\uniaud32t\alsa-kernel\core\seq\seq_device.c)
	at offset 0003F470 00008H bytes from F:\src\os2\uniaud32t\lib\Debug.ACP\sequencer.lib (F:\src\os2\uniaud32t\alsa-kernel\core\seq\seq_system.c)
	at offset 0003F478 00004H bytes from F:\src\os2\uniaud32t\lib\Debug.ACP\sequencer.lib (F:\src\os2\uniaud32t\alsa-kernel\core\seq\seq_queue.c)
	at offset 0003F47C 00140H bytes from F:\src\os2\uniaud32t\lib\Debug.ACP\sequencer.lib (F:\src\os2\uniaud32t\alsa-kernel\core\seq\seq_clientmgr.c)
	at offset 0003F5BC 00030H bytes from F:\src\os2\uniaud32t\lib\Debug.ACP\opl3.lib (F:\src\os2\uniaud32t\alsa-kernel\drivers\opl3\opl3_seq.c)
	at offset 0003F5EC 00074H bytes from F:\src\os2\uniaud32t\lib\Debug.ACP\opl3.lib (F:\src\os2\uniaud32t\alsa-kernel\drivers\opl3\opl3_lib.c)
	at offset 0003F660 000A7H bytes from F:\src\os2\uniaud32t\lib\Debug.ACP\opl3.lib (F:\src\os2\uniaud32t\alsa-kernel\drivers\opl3\opl3_drums.c)
	at offset 0003F708 000E8H bytes from F:\src\os2\uniaud32t\lib\Debug.ACP\opl3.lib (F:\src\os2\uniaud32t\alsa-kernel\drivers\opl3\opl3_midi.c)
	at offset 0003F7F0 00024H bytes from F:\src\os2\uniaud32t\lib\Debug.ACP\opl3.lib (F:\src\os2\uniaud32t\alsa-kernel\drivers\opl3\opl3_synth.c)
	at offset 0003F814 00028H bytes from F:\src\os2\uniaud32t\lib\Debug.ACP\mpu401.lib (F:\src\os2\uniaud32t\alsa-kernel\drivers\mpu401\mpu401_uart.c)
	at offset 0003F83C 0011CH bytes from F:\src\os2\uniaud32t\lib\Debug.ACP\cs46xx.lib (F:\src\os2\uniaud32t\alsa-kernel\pci\cs46xx\cs46xx.c)
	at offset 0003F958 0DBC8H bytes from F:\src\os2\uniaud32t\lib\Debug.ACP\cs46xx.lib (F:\src\os2\uniaud32t\alsa-kernel\pci\cs46xx\cs46xx_lib.c)
	at offset 0004D520 00118H bytes from F:\src\os2\uniaud32t\lib\Debug.ACP\cs5535audio.lib (F:\src\os2\uniaud32t\alsa-kernel\pci\cs5535audio\cs5535audio.c)
	at offset 0004D638 00110H bytes from F:\src\os2\uniaud32t\lib\Debug.ACP\cs5535audio.lib (F:\src\os2\uniaud32t\alsa-kernel\pci\cs5535audio\cs5535audio_pcm.c)
	at offset 0004D748 0015CH bytes from F:\src\os2\uniaud32t\lib\Debug.ACP\emu10k1.lib (F:\src\os2\uniaud32t\alsa-kernel\pci\emu10k1\emu10k1.c)
	at offset 0004D8A4 002E8H bytes from F:\src\os2\uniaud32t\lib\Debug.ACP\emu10k1.lib (F:\src\os2\uniaud32t\alsa-kernel\pci\emu10k1\p16v.c)
	at offset 0004DB8C 00030H bytes from F:\src\os2\uniaud32t\lib\Debug.ACP\emu10k1.lib (F:\src\os2\uniaud32t\alsa-kernel\pci\emu10k1\timer.c)
	at offset 0004DBBC 001C0H bytes from F:\src\os2\uniaud32t\lib\Debug.ACP\emu10k1.lib (F:\src\os2\uniaud32t\alsa-kernel\pci\emu10k1\emufx.c)
	at offset 0004DD7C 0169CH bytes from F:\src\os2\uniaud32t\lib\Debug.ACP\emu10k1.lib (F:\src\os2\uniaud32t\alsa-kernel\pci\emu10k1\emumixer.c)
	at offset 0004F418 00334H bytes from F:\src\os2\uniaud32t\lib\Debug.ACP\emu10k1.lib (F:\src\os2\uniaud32t\alsa-kernel\pci\emu10k1\emupcm.c)
	at offset 0004F74C 00020H bytes from F:\src\os2\uniaud32t\lib\Debug.ACP\emu10k1.lib (F:\src\os2\uniaud32t\alsa-kernel\pci\emu10k1\emumpu401.c)
	at offset 0004F76C 00894H bytes from F:\src\os2\uniaud32t\lib\Debug.ACP\emu10k1.lib (F:\src\os2\uniaud32t\alsa-kernel\pci\emu10k1\emu10k1_main.c)
	at offset 00050000 00270H bytes from F:\src\os2\uniaud32t\lib\Debug.ACP\emu10k1.lib (F:\src\os2\uniaud32t\alsa-kernel\pci\emu10k1\emuproc.c)
	at offset 00050270 00280H bytes from F:\src\os2\uniaud32t\lib\Debug.ACP\emu10k1.lib (F:\src\os2\uniaud32t\alsa-kernel\pci\emu10k1\io.c)
	at offset 000504F0 00150H bytes from F:\src\os2\uniaud32t\lib\Debug.ACP\ymfpci.lib (F:\src\os2\uniaud32t\alsa-kernel\pci\ymfpci\ymfpci.c)
	at offset 00050640 006D8H bytes from F:\src\os2\uniaud32t\lib\Debug.ACP\ymfpci.lib (F:\src\os2\uniaud32t\alsa-kernel\pci\ymfpci\ymfpci_main.c)
	at offset 00050D18 002E8H bytes from F:\src\os2\uniaud32t\lib\Debug.ACP\ali5451.lib (F:\src\os2\uniaud32t\alsa-kernel\pci\ali5451\ali5451.c)
	at offset 00051000 0013CH bytes from F:\src\os2\uniaud32t\lib\Debug.ACP\trident.lib (F:\src\os2\uniaud32t\alsa-kernel\pci\trident\trident.c)
	at offset 0005113C 004ECH bytes from F:\src\os2\uniaud32t\lib\Debug.ACP\trident.lib (F:\src\os2\uniaud32t\alsa-kernel\pci\trident\trident_main.c)
	at offset 00051628 0C81CH bytes from F:\src\os2\uniaud32t\lib\Debug.ACP\nm256.lib (F:\src\os2\uniaud32t\alsa-kernel\pci\nm256\nm256.c)
	at offset 0005DE44 005B0H bytes from F:\src\os2\uniaud32t\lib\Debug.ACP\sb.lib (F:\src\os2\uniaud32t\alsa-kernel\isa\sb\sb_mixer.c)
	at offset 0005E3F4 00014H bytes from F:\src\os2\uniaud32t\lib\Debug.ACP\sb.lib (F:\src\os2\uniaud32t\alsa-kernel\isa\sb\sb_common.c)
	at offset 0005E408 00080H bytes from F:\src\os2\uniaud32t\lib\Debug.ACP\core_oss.lib (F:\src\os2\uniaud32t\alsa-kernel\core\oss\pcm_oss.c)
	at offset 0005E488 0008CH bytes from E:\watcom\lib386\os2\clib3r.lib (strtol.c)
	at offset 0005E514 00008H bytes from E:\watcom\lib386\os2\clib3r.lib (noefgfmt.c)
	at offset 0005E51C 00040H bytes from E:\watcom\lib386\os2\clib3r.lib (maino32.c)
	at offset 0005E55C 0004AH bytes from E:\watcom\lib386\os2\clib3r.lib (crwdata)
	at offset 0005E5A8 00004H bytes from E:\watcom\lib386\os2\clib3r.lib (mbinit.c)
	at offset 0005E5AC 00001H bytes from E:\watcom\lib386\os2\clib3r.lib (enterdb.c)
	at offset 0005E5B0 00004H bytes from E:\watcom\lib386\os2\clib3r.lib (amblksiz.c)
	at offset 0005E5B4 00051H bytes from F:\src\os2\uniaud32t\lib\Debug.ACP\ac97.lib (F:\src\os2\uniaud32t\alsa-kernel\pci\ac97\ac97_pcm.c)
	at offset 0005E608 00812H bytes from F:\src\os2\uniaud32t\lib\Debug.ACP\ac97.lib (F:\src\os2\uniaud32t\alsa-kernel\pci\ac97\ac97_codec.c)
	at offset 0005EE1C 00110H bytes from F:\src\os2\uniaud32t\lib\Debug.ACP\ac97.lib (F:\src\os2\uniaud32t\alsa-kernel\pci\ac97\ac97_proc.c)
	at offset 0005EF2C 00018H bytes from F:\src\os2\uniaud32t\lib\Debug.ACP\sequencer.lib (F:\src\os2\uniaud32t\alsa-kernel\core\seq\seq_midi_emul.c)
	at offset 0005EF44 00008H bytes from F:\src\os2\uniaud32t\lib\Debug.ACP\synth.lib (F:\src\os2\uniaud32t\alsa-kernel\synth\util_mem.c)

 0005:0006074C 000014E45H CONST                  DATA 32-bit
	at offset 00000000 00013H bytes from F:\src\os2\uniaud32t\drv32\bin\Debug.ACP\strategy.obj (F:\src\os2\uniaud32t\drv32\strategy.c)
	at offset 00000013 0003AH bytes from F:\src\os2\uniaud32t\drv32\bin\Debug.ACP\init.obj (F:\src\os2\uniaud32t\drv32\init.c)
	at offset 0000004D 00073H bytes from F:\src\os2\uniaud32t\drv32\bin\Debug.ACP\parse.obj (F:\src\os2\uniaud32t\drv32\parse.c)
	at offset 000000C0 00012H bytes from F:\src\os2\uniaud32t\drv32\bin\Debug.ACP\idc.obj (F:\src\os2\uniaud32t\drv32\idc.c)
	at offset 000000D2 00096H bytes from F:\src\os2\uniaud32t\drv32\bin\Debug.ACP\dispatch.obj (F:\src\os2\uniaud32t\drv32\dispatch.c)
	at offset 00000168 001CCH bytes from F:\src\os2\uniaud32t\drv32\bin\Debug.ACP\rmhelp.obj (F:\src\os2\uniaud32t\drv32\rmhelp.cpp)
	at offset 00000334 00081H bytes from F:\src\os2\uniaud32t\drv32\bin\Debug.ACP\irq.obj (F:\src\os2\uniaud32t\drv32\irq.cpp)
	at offset 000003B8 00029H bytes from F:\src\os2\uniaud32t\lib\Debug.ACP\linuxlib.lib (F:\src\os2\uniaud32t\lib32\vsprintf.c)
	at offset 000003E4 0001FH bytes from F:\src\os2\uniaud32t\lib\Debug.ACP\linuxlib.lib (F:\src\os2\uniaud32t\lib32\timer.c)
	at offset 00000404 00054H bytes from F:\src\os2\uniaud32t\lib\Debug.ACP\linuxlib.lib (F:\src\os2\uniaud32t\lib32\misc.c)
	at offset 00000458 000C2H bytes from F:\src\os2\uniaud32t\lib\Debug.ACP\linuxlib.lib (F:\src\os2\uniaud32t\lib32\ossidc.cpp)
	at offset 0000051C 001C8H bytes from F:\src\os2\uniaud32t\lib\Debug.ACP\linuxlib.lib (F:\src\os2\uniaud32t\lib32\soundmidi.c)
	at offset 000006E4 0028FH bytes from F:\src\os2\uniaud32t\lib\Debug.ACP\linuxlib.lib (F:\src\os2\uniaud32t\lib32\soundmixer.c)
	at offset 00000974 00809H bytes from F:\src\os2\uniaud32t\lib\Debug.ACP\linuxlib.lib (F:\src\os2\uniaud32t\lib32\sound.c)
	at offset 00001180 0002EH bytes from F:\src\os2\uniaud32t\lib\Debug.ACP\linuxlib.lib (F:\src\os2\uniaud32t\lib32\debug.c)
	at offset 000011AE 000DEH bytes from F:\src\os2\uniaud32t\lib\Debug.ACP\linuxlib.lib (F:\src\os2\uniaud32t\lib32\memory.cpp)
	at offset 0000128C 00195H bytes from F:\src\os2\uniaud32t\lib\Debug.ACP\linuxlib.lib (F:\src\os2\uniaud32t\lib32\ioctl.c)
	at offset 00001424 0009AH bytes from F:\src\os2\uniaud32t\lib\Debug.ACP\linuxlib.lib (F:\src\os2\uniaud32t\lib32\irq.c)
	at offset 000014C0 0032EH bytes from F:\src\os2\uniaud32t\lib\Debug.ACP\linuxlib.lib (F:\src\os2\uniaud32t\lib32\pci.c)
	at offset 000017EE 001FDH bytes from F:\src\os2\uniaud32t\lib\Debug.ACP\linuxlib.lib (F:\src\os2\uniaud32t\lib32\malloc.cpp)
	at offset 000019EC 0006AH bytes from F:\src\os2\uniaud32t\lib\Debug.ACP\linuxlib.lib (F:\src\os2\uniaud32t\lib32\waitqueue.c)
	at offset 00001A58 00109H bytes from F:\src\os2\uniaud32t\lib\Debug.ACP\core.lib (F:\src\os2\uniaud32t\alsa-kernel\core\hwdep.c)
	at offset 00001B64 00166H bytes from F:\src\os2\uniaud32t\lib\Debug.ACP\core.lib (F:\src\os2\uniaud32t\alsa-kernel\core\timer.c)
	at offset 00001CCC 002FEH bytes from F:\src\os2\uniaud32t\lib\Debug.ACP\core.lib (F:\src\os2\uniaud32t\alsa-kernel\core\rawmidi.c)
	at offset 00001FCC 000A9H bytes from F:\src\os2\uniaud32t\lib\Debug.ACP\core.lib (F:\src\os2\uniaud32t\alsa-kernel\core\pcm_lib.c)
	at offset 00002078 000CCH bytes from F:\src\os2\uniaud32t\lib\Debug.ACP\core.lib (F:\src\os2\uniaud32t\alsa-kernel\core\pcm.c)
	at offset 00002144 000DEH bytes from F:\src\os2\uniaud32t\lib\Debug.ACP\core.lib (F:\src\os2\uniaud32t\alsa-kernel\core\sound.c)
	at offset 00002224 000B4H bytes from F:\src\os2\uniaud32t\lib\Debug.ACP\core.lib (F:\src\os2\uniaud32t\alsa-kernel\core\info.c)
	at offset 000022D8 0006AH bytes from F:\src\os2\uniaud32t\lib\Debug.ACP\core.lib (F:\src\os2\uniaud32t\alsa-kernel\core\pcm_timer.c)
	at offset 00002344 000C4H bytes from F:\src\os2\uniaud32t\lib\Debug.ACP\core.lib (F:\src\os2\uniaud32t\alsa-kernel\core\pcm_native.c)
	at offset 00002408 000F2H bytes from F:\src\os2\uniaud32t\lib\Debug.ACP\core.lib (F:\src\os2\uniaud32t\alsa-kernel\core\info_oss.c)
	at offset 000024FC 00068H bytes from F:\src\os2\uniaud32t\lib\Debug.ACP\core.lib (F:\src\os2\uniaud32t\alsa-kernel\core\sound_oss.c)
	at offset 00002564 000BDH bytes from F:\src\os2\uniaud32t\lib\Debug.ACP\core.lib (F:\src\os2\uniaud32t\alsa-kernel\core\device.c)
	at offset 00002624 0011DH bytes from F:\src\os2\uniaud32t\lib\Debug.ACP\core.lib (F:\src\os2\uniaud32t\alsa-kernel\core\control.c)
	at offset 00002744 0007EH bytes from F:\src\os2\uniaud32t\lib\Debug.ACP\core.lib (F:\src\os2\uniaud32t\alsa-kernel\core\memalloc.c)
	at offset 000027C4 0022FH bytes from F:\src\os2\uniaud32t\lib\Debug.ACP\core.lib (F:\src\os2\uniaud32t\alsa-kernel\core\init.c)
	at offset 000029F4 00020H bytes from F:\src\os2\uniaud32t\lib\Debug.ACP\core.lib (F:\src\os2\uniaud32t\alsa-kernel\core\sgbuf.c)
	at offset 00002A14 00339H bytes from F:\src\os2\uniaud32t\lib\Debug.ACP\pci.lib (F:\src\os2\uniaud32t\alsa-kernel\pci\bt87x.c)
	at offset 00002D50 00103H bytes from F:\src\os2\uniaud32t\lib\Debug.ACP\pci.lib (F:\src\os2\uniaud32t\alsa-kernel\pci\als4000.c)
	at offset 00002E54 0055FH bytes from F:\src\os2\uniaud32t\lib\Debug.ACP\pci.lib (F:\src\os2\uniaud32t\alsa-kernel\pci\cmipci.c)
	at offset 000033B4 0027CH bytes from F:\src\os2\uniaud32t\lib\Debug.ACP\pci.lib (F:\src\os2\uniaud32t\alsa-kernel\pci\atiixp.c)
	at offset 00003630 00260H bytes from F:\src\os2\uniaud32t\lib\Debug.ACP\pci.lib (F:\src\os2\uniaud32t\alsa-kernel\pci\fm801.c)
	at offset 00003890 00653H bytes from F:\src\os2\uniaud32t\lib\Debug.ACP\pci.lib (F:\src\os2\uniaud32t\alsa-kernel\pci\via82xx.c)
	at offset 00003EE4 00267H bytes from F:\src\os2\uniaud32t\lib\Debug.ACP\pci.lib (F:\src\os2\uniaud32t\alsa-kernel\pci\maestro3.c)
	at offset 0000414C 00A6FH bytes from F:\src\os2\uniaud32t\lib\Debug.ACP\pci.lib (F:\src\os2\uniaud32t\alsa-kernel\pci\intel8x0.c)
	at offset 00004BBC 002FBH bytes from F:\src\os2\uniaud32t\lib\Debug.ACP\pci.lib (F:\src\os2\uniaud32t\alsa-kernel\pci\es1968.c)
	at offset 00004EB8 00428H bytes from F:\src\os2\uniaud32t\lib\Debug.ACP\pci.lib (F:\src\os2\uniaud32t\alsa-kernel\pci\es1938.c)
	at offset 000052E0 002CBH bytes from F:\src\os2\uniaud32t\lib\Debug.ACP\pci.lib (F:\src\os2\uniaud32t\alsa-kernel\pci\cs4281.c)
	at offset 000055AC 00266H bytes from F:\src\os2\uniaud32t\lib\Debug.ACP\pci.lib (F:\src\os2\uniaud32t\alsa-kernel\pci\ens1371.c)
	at offset 00005814 00301H bytes from F:\src\os2\uniaud32t\lib\Debug.ACP\ca0106.lib (F:\src\os2\uniaud32t\alsa-kernel\pci\ca0106\ca0106_main.c)
	at offset 00005B18 00045H bytes from F:\src\os2\uniaud32t\lib\Debug.ACP\ca0106.lib (F:\src\os2\uniaud32t\alsa-kernel\pci\ca0106\ca_midi.c)
	at offset 00005B60 00689H bytes from F:\src\os2\uniaud32t\lib\Debug.ACP\ca0106.lib (F:\src\os2\uniaud32t\alsa-kernel\pci\ca0106\ca0106_mixer.c)
	at offset 000061EC 003CCH bytes from F:\src\os2\uniaud32t\lib\Debug.ACP\ca0106.lib (F:\src\os2\uniaud32t\alsa-kernel\pci\ca0106\ca0106_proc.c)
	at offset 000065B8 003A0H bytes from F:\src\os2\uniaud32t\lib\Debug.ACP\hda.lib (F:\src\os2\uniaud32t\alsa-kernel\pci\hda\patch_via.c)
	at offset 00006958 005ECH bytes from F:\src\os2\uniaud32t\lib\Debug.ACP\hda.lib (F:\src\os2\uniaud32t\alsa-kernel\pci\hda\patch_conexant.c)
	at offset 00006F44 00048H bytes from F:\src\os2\uniaud32t\lib\Debug.ACP\hda.lib (F:\src\os2\uniaud32t\alsa-kernel\pci\hda\patch_atihdmi.c)
	at offset 00006F8C 00FCFH bytes from F:\src\os2\uniaud32t\lib\Debug.ACP\hda.lib (F:\src\os2\uniaud32t\alsa-kernel\pci\hda\patch_sigmatel.c)
	at offset 00007F5C 00A32H bytes from F:\src\os2\uniaud32t\lib\Debug.ACP\hda.lib (F:\src\os2\uniaud32t\alsa-kernel\pci\hda\patch_analog.c)
	at offset 00008990 001A6H bytes from F:\src\os2\uniaud32t\lib\Debug.ACP\hda.lib (F:\src\os2\uniaud32t\alsa-kernel\pci\hda\patch_cmedia.c)
	at offset 00008B38 01CB7H bytes from F:\src\os2\uniaud32t\lib\Debug.ACP\hda.lib (F:\src\os2\uniaud32t\alsa-kernel\pci\hda\patch_realtek.c)
	at offset 0000A7F0 00895H bytes from F:\src\os2\uniaud32t\lib\Debug.ACP\hda.lib (F:\src\os2\uniaud32t\alsa-kernel\pci\hda\hda_intel.c)
	at offset 0000B088 0097BH bytes from F:\src\os2\uniaud32t\lib\Debug.ACP\hda.lib (F:\src\os2\uniaud32t\alsa-kernel\pci\hda\hda_codec.c)
	at offset 0000BA04 0000DH bytes from F:\src\os2\uniaud32t\lib\Debug.ACP\hda.lib (F:\src\os2\uniaud32t\alsa-kernel\pci\hda\hda_hwdep.c)
	at offset 0000BA14 002C1H bytes from F:\src\os2\uniaud32t\lib\Debug.ACP\hda.lib (F:\src\os2\uniaud32t\alsa-kernel\pci\hda\hda_generic.c)
	at offset 0000BCD8 006EBH bytes from F:\src\os2\uniaud32t\lib\Debug.ACP\hda.lib (F:\src\os2\uniaud32t\alsa-kernel\pci\hda\hda_proc.c)
	at offset 0000C3C4 00163H bytes from F:\src\os2\uniaud32t\lib\Debug.ACP\sequencer.lib (F:\src\os2\uniaud32t\alsa-kernel\core\seq\seq_device.c)
	at offset 0000C528 00015H bytes from F:\src\os2\uniaud32t\lib\Debug.ACP\sequencer.lib (F:\src\os2\uniaud32t\alsa-kernel\core\seq\seq_info.c)
	at offset 0000C540 00016H bytes from F:\src\os2\uniaud32t\lib\Debug.ACP\sequencer.lib (F:\src\os2\uniaud32t\alsa-kernel\core\seq\seq_system.c)
	at offset 0000C558 00156H bytes from F:\src\os2\uniaud32t\lib\Debug.ACP\sequencer.lib (F:\src\os2\uniaud32t\alsa-kernel\core\seq\seq_queue.c)
	at offset 0000C6B0 0013AH bytes from F:\src\os2\uniaud32t\lib\Debug.ACP\sequencer.lib (F:\src\os2\uniaud32t\alsa-kernel\core\seq\seq_memory.c)
	at offset 0000C7EC 001FAH bytes from F:\src\os2\uniaud32t\lib\Debug.ACP\sequencer.lib (F:\src\os2\uniaud32t\alsa-kernel\core\seq\seq_clientmgr.c)
	at offset 0000C9E8 00060H bytes from F:\src\os2\uniaud32t\lib\Debug.ACP\sequencer.lib (F:\src\os2\uniaud32t\alsa-kernel\core\seq\seq_ports.c)
	at offset 0000CA48 00127H bytes from F:\src\os2\uniaud32t\lib\Debug.ACP\sequencer.lib (F:\src\os2\uniaud32t\alsa-kernel\core\seq\seq_timer.c)
	at offset 0000CB70 000C3H bytes from F:\src\os2\uniaud32t\lib\Debug.ACP\sequencer.lib (F:\src\os2\uniaud32t\alsa-kernel\core\seq\seq_prioq.c)
	at offset 0000CC34 00047H bytes from F:\src\os2\uniaud32t\lib\Debug.ACP\sequencer.lib (F:\src\os2\uniaud32t\alsa-kernel\core\seq\seq_fifo.c)
	at offset 0000CC7C 00028H bytes from F:\src\os2\uniaud32t\lib\Debug.ACP\opl3.lib (F:\src\os2\uniaud32t\alsa-kernel\drivers\opl3\opl3_seq.c)
	at offset 0000CCA4 0014DH bytes from F:\src\os2\uniaud32t\lib\Debug.ACP\opl3.lib (F:\src\os2\uniaud32t\alsa-kernel\drivers\opl3\opl3_lib.c)
	at offset 0000CDF4 0000FH bytes from F:\src\os2\uniaud32t\lib\Debug.ACP\opl3.lib (F:\src\os2\uniaud32t\alsa-kernel\drivers\opl3\opl3_synth.c)
	at offset 0000CE04 000E6H bytes from F:\src\os2\uniaud32t\lib\Debug.ACP\mpu401.lib (F:\src\os2\uniaud32t\alsa-kernel\drivers\mpu401\mpu401_uart.c)
	at offset 0000CEEC 00035H bytes from F:\src\os2\uniaud32t\lib\Debug.ACP\cs46xx.lib (F:\src\os2\uniaud32t\alsa-kernel\pci\cs46xx\cs46xx.c)
	at offset 0000CF24 005A3H bytes from F:\src\os2\uniaud32t\lib\Debug.ACP\cs46xx.lib (F:\src\os2\uniaud32t\alsa-kernel\pci\cs46xx\cs46xx_lib.c)
	at offset 0000D4C8 00129H bytes from F:\src\os2\uniaud32t\lib\Debug.ACP\cs5535audio.lib (F:\src\os2\uniaud32t\alsa-kernel\pci\cs5535audio\cs5535audio.c)
	at offset 0000D5F4 000C2H bytes from F:\src\os2\uniaud32t\lib\Debug.ACP\cs5535audio.lib (F:\src\os2\uniaud32t\alsa-kernel\pci\cs5535audio\cs5535audio_pm.c)
	at offset 0000D6B8 0005CH bytes from F:\src\os2\uniaud32t\lib\Debug.ACP\cs5535audio.lib (F:\src\os2\uniaud32t\alsa-kernel\pci\cs5535audio\cs5535audio_pcm.c)
	at offset 0000D714 000BBH bytes from F:\src\os2\uniaud32t\lib\Debug.ACP\emu10k1.lib (F:\src\os2\uniaud32t\alsa-kernel\pci\emu10k1\emu10k1.c)
	at offset 0000D7D0 00189H bytes from F:\src\os2\uniaud32t\lib\Debug.ACP\emu10k1.lib (F:\src\os2\uniaud32t\alsa-kernel\pci\emu10k1\p16v.c)
	at offset 0000D95C 00016H bytes from F:\src\os2\uniaud32t\lib\Debug.ACP\emu10k1.lib (F:\src\os2\uniaud32t\alsa-kernel\pci\emu10k1\timer.c)
	at offset 0000D974 00B47H bytes from F:\src\os2\uniaud32t\lib\Debug.ACP\emu10k1.lib (F:\src\os2\uniaud32t\alsa-kernel\pci\emu10k1\emufx.c)
	at offset 0000E4BC 01089H bytes from F:\src\os2\uniaud32t\lib\Debug.ACP\emu10k1.lib (F:\src\os2\uniaud32t\alsa-kernel\pci\emu10k1\emumixer.c)
	at offset 0000F548 000B8H bytes from F:\src\os2\uniaud32t\lib\Debug.ACP\emu10k1.lib (F:\src\os2\uniaud32t\alsa-kernel\pci\emu10k1\emupcm.c)
	at offset 0000F600 00082H bytes from F:\src\os2\uniaud32t\lib\Debug.ACP\emu10k1.lib (F:\src\os2\uniaud32t\alsa-kernel\pci\emu10k1\emumpu401.c)
	at offset 0000F684 007C9H bytes from F:\src\os2\uniaud32t\lib\Debug.ACP\emu10k1.lib (F:\src\os2\uniaud32t\alsa-kernel\pci\emu10k1\emu10k1_main.c)
	at offset 0000FE50 00831H bytes from F:\src\os2\uniaud32t\lib\Debug.ACP\emu10k1.lib (F:\src\os2\uniaud32t\alsa-kernel\pci\emu10k1\emuproc.c)
	at offset 00010684 0009CH bytes from F:\src\os2\uniaud32t\lib\Debug.ACP\emu10k1.lib (F:\src\os2\uniaud32t\alsa-kernel\pci\emu10k1\io.c)
	at offset 00010720 0008CH bytes from F:\src\os2\uniaud32t\lib\Debug.ACP\emu10k1.lib (F:\src\os2\uniaud32t\alsa-kernel\pci\emu10k1\memory.c)
	at offset 000107AC 000C9H bytes from F:\src\os2\uniaud32t\lib\Debug.ACP\emu10k1.lib (F:\src\os2\uniaud32t\alsa-kernel\pci\emu10k1\irq.c)
	at offset 00010878 00128H bytes from F:\src\os2\uniaud32t\lib\Debug.ACP\ymfpci.lib (F:\src\os2\uniaud32t\alsa-kernel\pci\ymfpci\ymfpci.c)
	at offset 000109A0 00374H bytes from F:\src\os2\uniaud32t\lib\Debug.ACP\ymfpci.lib (F:\src\os2\uniaud32t\alsa-kernel\pci\ymfpci\ymfpci_main.c)
	at offset 00010D14 0044CH bytes from F:\src\os2\uniaud32t\lib\Debug.ACP\ali5451.lib (F:\src\os2\uniaud32t\alsa-kernel\pci\ali5451\ali5451.c)
	at offset 00011160 00068H bytes from F:\src\os2\uniaud32t\lib\Debug.ACP\trident.lib (F:\src\os2\uniaud32t\alsa-kernel\pci\trident\trident.c)
	at offset 000111C8 00442H bytes from F:\src\os2\uniaud32t\lib\Debug.ACP\trident.lib (F:\src\os2\uniaud32t\alsa-kernel\pci\trident\trident_main.c)
	at offset 0001160C 00035H bytes from F:\src\os2\uniaud32t\lib\Debug.ACP\trident.lib (F:\src\os2\uniaud32t\alsa-kernel\pci\trident\trident_memory.c)
	at offset 00011644 0043FH bytes from F:\src\os2\uniaud32t\lib\Debug.ACP\nm256.lib (F:\src\os2\uniaud32t\alsa-kernel\pci\nm256\nm256.c)
	at offset 00011A84 00374H bytes from F:\src\os2\uniaud32t\lib\Debug.ACP\sb.lib (F:\src\os2\uniaud32t\alsa-kernel\isa\sb\sb_mixer.c)
	at offset 00011DF8 0017AH bytes from F:\src\os2\uniaud32t\lib\Debug.ACP\sb.lib (F:\src\os2\uniaud32t\alsa-kernel\isa\sb\sb_common.c)
	at offset 00011F74 00247H bytes from F:\src\os2\uniaud32t\lib\Debug.ACP\core_oss.lib (F:\src\os2\uniaud32t\alsa-kernel\core\oss\pcm_oss.c)
	at offset 000121BC 00025H bytes from E:\watcom\lib386\os2\clib3r.lib (alphabet.c)
	at offset 000121E4 000E3H bytes from F:\src\os2\uniaud32t\lib\Debug.ACP\linuxlib.lib (F:\src\os2\uniaud32t\lib32\semaphore.c)
	at offset 000122C8 0001AH bytes from F:\src\os2\uniaud32t\lib\Debug.ACP\core.lib (F:\src\os2\uniaud32t\alsa-kernel\core\vmaster.c)
	at offset 000122E4 0008CH bytes from F:\src\os2\uniaud32t\lib\Debug.ACP\ac97.lib (F:\src\os2\uniaud32t\alsa-kernel\pci\ac97\ac97_pcm.c)
	at offset 00012370 01E85H bytes from F:\src\os2\uniaud32t\lib\Debug.ACP\ac97.lib (F:\src\os2\uniaud32t\alsa-kernel\pci\ac97\ac97_codec.c)
	at offset 000141F8 00BFFH bytes from F:\src\os2\uniaud32t\lib\Debug.ACP\ac97.lib (F:\src\os2\uniaud32t\alsa-kernel\pci\ac97\ac97_proc.c)
	at offset 00014DF8 0004DH bytes from F:\src\os2\uniaud32t\lib\Debug.ACP\sequencer.lib (F:\src\os2\uniaud32t\alsa-kernel\core\seq\seq_midi_emul.c)

 0005:000755A0 0000055D6H CONST2                 DATA 32-bit
	at offset 00000000 0017BH bytes from F:\src\os2\uniaud32t\drv32\bin\Debug.ACP\init.obj (F:\src\os2\uniaud32t\drv32\init.c)
	at offset 0000017C 00040H bytes from F:\src\os2\uniaud32t\lib\Debug.ACP\core.lib (F:\src\os2\uniaud32t\alsa-kernel\core\info.c)
	at offset 000001BC 00004H bytes from F:\src\os2\uniaud32t\lib\Debug.ACP\core.lib (F:\src\os2\uniaud32t\alsa-kernel\core\pcm_memory.c)
	at offset 000001C0 0000CH bytes from F:\src\os2\uniaud32t\lib\Debug.ACP\core.lib (F:\src\os2\uniaud32t\alsa-kernel\core\pcm_native.c)
	at offset 000001CC 00028H bytes from F:\src\os2\uniaud32t\lib\Debug.ACP\pci.lib (F:\src\os2\uniaud32t\alsa-kernel\pci\als4000.c)
	at offset 000001F4 00020H bytes from F:\src\os2\uniaud32t\lib\Debug.ACP\pci.lib (F:\src\os2\uniaud32t\alsa-kernel\pci\cmipci.c)
	at offset 00000214 00010H bytes from F:\src\os2\uniaud32t\lib\Debug.ACP\pci.lib (F:\src\os2\uniaud32t\alsa-kernel\pci\fm801.c)
	at offset 00000224 00010H bytes from F:\src\os2\uniaud32t\lib\Debug.ACP\pci.lib (F:\src\os2\uniaud32t\alsa-kernel\pci\via82xx.c)
	at offset 00000234 000BCH bytes from F:\src\os2\uniaud32t\lib\Debug.ACP\pci.lib (F:\src\os2\uniaud32t\alsa-kernel\pci\maestro3.c)
	at offset 000002F0 00010H bytes from F:\src\os2\uniaud32t\lib\Debug.ACP\pci.lib (F:\src\os2\uniaud32t\alsa-kernel\pci\es1938.c)
	at offset 00000300 00010H bytes from F:\src\os2\uniaud32t\lib\Debug.ACP\pci.lib (F:\src\os2\uniaud32t\alsa-kernel\pci\cs4281.c)
	at offset 00000310 00010H bytes from F:\src\os2\uniaud32t\lib\Debug.ACP\pci.lib (F:\src\os2\uniaud32t\alsa-kernel\pci\ens1371.c)
	at offset 00000320 00020H bytes from F:\src\os2\uniaud32t\lib\Debug.ACP\ca0106.lib (F:\src\os2\uniaud32t\alsa-kernel\pci\ca0106\ca0106_main.c)
	at offset 00000340 00020H bytes from F:\src\os2\uniaud32t\lib\Debug.ACP\ca0106.lib (F:\src\os2\uniaud32t\alsa-kernel\pci\ca0106\ca0106_mixer.c)
	at offset 00000360 00084H bytes from F:\src\os2\uniaud32t\lib\Debug.ACP\hda.lib (F:\src\os2\uniaud32t\alsa-kernel\pci\hda\patch_conexant.c)
	at offset 000003E4 00010H bytes from F:\src\os2\uniaud32t\lib\Debug.ACP\emu10k1.lib (F:\src\os2\uniaud32t\alsa-kernel\pci\emu10k1\p16v.c)
	at offset 000003F4 00814H bytes from F:\src\os2\uniaud32t\lib\Debug.ACP\emu10k1.lib (F:\src\os2\uniaud32t\alsa-kernel\pci\emu10k1\emufx.c)
	at offset 00000C08 00010H bytes from F:\src\os2\uniaud32t\lib\Debug.ACP\emu10k1.lib (F:\src\os2\uniaud32t\alsa-kernel\pci\emu10k1\emumixer.c)
	at offset 00000C18 00010H bytes from F:\src\os2\uniaud32t\lib\Debug.ACP\ymfpci.lib (F:\src\os2\uniaud32t\alsa-kernel\pci\ymfpci\ymfpci_main.c)
	at offset 00000C28 00020H bytes from F:\src\os2\uniaud32t\lib\Debug.ACP\trident.lib (F:\src\os2\uniaud32t\alsa-kernel\pci\trident\trident_main.c)
	at offset 00000C48 00018H bytes from F:\src\os2\uniaud32t\lib\Debug.ACP\ac97.lib (F:\src\os2\uniaud32t\alsa-kernel\pci\ac97\ac97_pcm.c)
	at offset 00000C60 04976H bytes from F:\src\os2\uniaud32t\lib\Debug.ACP\ac97.lib (F:\src\os2\uniaud32t\alsa-kernel\pci\ac97\ac97_codec.c)

 0005:0007AB78 000000004H LASTDATA32             DATA 32-bit
	at offset 00000000 00004H bytes from F:\src\os2\uniaud32t\drv32\bin\Debug.ACP\end.obj (end.asm)

 0005:0007AB7C 000000000H XIB                    DATA 32-bit

 0005:0007AB7C 000000006H XI                     DATA 32-bit
	at offset 00000000 00006H bytes from E:\watcom\lib386\os2\clib3r.lib (mbislead.c)

 0005:0007AB82 000000000H XIE                    DATA 32-bit

 0005:0007AB82 000000000H TIB                    DATA 32-bit

 0005:0007AB82 000000000H TI                     DATA 32-bit

 0005:0007AB82 000000000H TIE                    DATA 32-bit

 0005:0007AB82 000000000H YIB                    DATA 32-bit

 0005:0007AB82 000000000H YI                     DATA 32-bit

 0005:0007AB82 000000000H YIE                    DATA 32-bit

 0005:0007AB82 000000000H DATA                   DATA 32-bit

 0005:0007AB84 000000000H CONST32                CONST 32-bit

 0005:0007AB84 000000045H CONST32_RO             CONST 32-bit
	at offset 00000000 00045H bytes from F:\acpi\lib\acpidrv.lib (acpi)

 0005:0007ABD0 000000004H _NULL                  BEGDATA 32-bit
	at offset 00000000 00004H bytes from E:\watcom\lib386\os2\clib3r.lib (segdefns)

 0005:0007ABD4 000000000H _AFTERNULL             BEGDATA 32-bit

 0005:0007ABE0 000010000H STACK                  STACK 32-bit
	at offset 00000000 10000H bytes from E:\watcom\lib386\os2\clib3r.lib (segdefns)


 Origin   Group
 0000:0   FLAT
 0003:0   CGROUP
 0005:0   DGROUP


 Address         Publics by Name
 0003:000CD800       ACPIFindPCIDevice
 0003:00009E2B       AddBaseAddress_
 0003:00003ED1       add_timer_
 0003:00010115       add_wait_queue_
 0003:00010131       add_wait_queue_exclusive_
 0003:0000A50F       alloc_pages_
 0003:00007445       ALSAToOSSDataType_
 0003:0000753A       ALSAToOSSRateFlags_
 0003:00003409       ALSA_FreeIrq_
 0003:00001672       ALSA_IDC
 0003:00003451       ALSA_Interrupt
 0003:00003326       ALSA_SetIrq_
 0003:00000656       ALSA_STRATEGY
 0003:00003D6C       ALSA_TIMER_
 0005:00001758       BootCode
 0003:00056B6C       ca_midi_init_
 0003:00009907       CharOut_
 0003:00089508       client_init_data_
 0003:00005820       ConvertVolume_
 0003:0000A75A       copy_from_user_
 0003:000CE8E4       copy_from_user_toio_
 0003:0000A6B5       copy_to_user_
 0003:000CE834       copy_to_user_fromio_
 0003:000042F6       create_proc_entry_
 0003:000046BD       create_workqueue_
 0003:00009DE1       DbgPrintIrq_
 0001:0000004C       DbgU32IntCnt
 0001:00000048       DbgU32TimerCnt
 0003:00009625       DecLongToASCII_
 0003:00003EEC       del_timer_
 0003:00004747       destroy_workqueue_
 0005:000017F4       DevHelp32
 0001:0000003C       DevHelpInit
 0003:00000010       DevHlp
 0003:00000030       DevHlp_ModifiedDS
 0003:0000445F       disable_dma_
 0003:0000CB12       disable_irq_
 0000:00000000  Imp  DOS32FLATDS          (DOSCALLS.370)
 0000:00000000  Imp  DOSCLOSE             (DOSCALLS.59)
 0000:00000000  Imp  DosExit              (DOSCALLS.234)
 0000:00000000  Imp  DOSIODELAYCNT        (DOSCALLS.427)
 0000:00000000  Imp  DOSOPEN              (DOSCALLS.70)
 0000:00000000  Imp  DosQueryCp           (DOSCALLS.291)
 0000:00000000  Imp  DosQueryDBCSEnv      (NLS.6)
 0000:00000000  Imp  DosQuerySysInfo      (DOSCALLS.348)
 0000:00000000  Imp  DOSWRITE             (DOSCALLS.138)
 0000:00000000  Imp  DosWrite             (DOSCALLS.282)
 0003:000CDC68       down_
 0003:000CDCCC       down_interruptible_
 0003:00003E85       do_gettimeofday_
 0003:00028056       dummy_get_unmapped_area_
 0003:00004444       enable_dma_
 0003:0000C96A       eoi_irq_
 0003:000043BE       fasync_helper_
 0001:0000046D       FileName
 0003:0000B3C0       FillCaps_
 0003:000CD990       FindAddress
 0003:00004650       flush_workqueue_
 0001:00000040       fOpen
 0003:00004429       free_dma_
 0003:0000C85F       free_irq_
 0003:0000A401       free_pages_
 0003:00009E8F       GetBaseAddress_
 0003:0000AD95       GetMaxChannels_
 0003:0000AC1B       GetNumberOfCards_
 0003:0000AC3E       GetNumberOfPcm_
 0003:00001513       GetParms_
 0003:0000ACB3       GetPcmForChannels_
 0003:00001624       GetTKSSBase
 0003:0000B704       GetUniaudCardInfo_
 0003:0000BCB6       GetUniaudControlInfo_
 0003:0000B850       GetUniaudControlNum_
 0003:0000BA45       GetUniaudControls_
 0003:0000BE27       GetUniaudControlValueGet_
 0003:0000BF98       GetUniaudControlValuePut_
 0003:0000AE7E       GetUniaudPcmCaps1_
 0003:0000B456       GetUniaudPcmCaps_
 0001:00000000       help_header
 0002:00000000       help_stub_strategy
 0003:00009792       HexLongToASCII_
 0003:0000425C       hweight32_
 0003:000000E0       IDC_
 0003:000CD8A2       InitACPICall
 0001:00000046       InitPktOff
 0001:00000044       InitPktSeg
 0003:000CDBFC       init_MUTEX_
 0003:000CDC32       init_MUTEX_LOCKED_
 0003:000101F8       init_waitqueue_entry_
 0003:000100FA       init_waitqueue_head_
 0003:0001019C       interruptible_sleep_on_
 0003:00010168       interruptible_sleep_on_timeout_
 0005:000017F8       intSwitchStack
 0003:0000CAEF       in_interrupt_
 0003:00001664       iodelay32_
 0003:000537B8       ioport_map_
 0003:000537F4       ioport_unmap_
 0003:0005365A       ioread16_
 0003:000536A8       ioread32_
 0003:0005360E       ioread8_
 0003:0000A610       iounmap_
 0003:00053730       iowrite16_
 0003:00053775       iowrite32_
 0003:000536ED       iowrite8_
 0003:0000A642       is_access_ok_
 0003:000E0760       itoa_
 0003:0000A95E       kcalloc_
 0000:00000000  Imp  KernLinToPageList    (KEE.64)
 0000:00000000  Imp  KernSelToFlat        (KEE.66)
 0000:00000000  Imp  KernThunkStackTo16   (KEE.40)
 0000:00000000  Imp  KernThunkStackTo32   (KEE.41)
 0000:00000000  Imp  KernVMAlloc          (KEE.60)
 0000:00000000  Imp  KernVMFree           (KEE.61)
 0000:00000000  Imp  KernVMLock           (KEE.62)
 0003:000043E6       kill_fasync_
 0003:0000476A       kstrdup_
 0003:0000A918       kzalloc_
 0003:000E06E0       lltoa_
 0003:000E0640       ltoa_
 0003:000E0510       mbtowc_
 0003:00003E51       mdelay_
 0003:00004960       memdup_user_
 0003:000DE380       memmove_
 0003:000DE360       memset_
 0003:000047DC       mod_firmware_load_
 0003:00003F11       mod_timer_
 0003:00003F2D       msleep_
 0003:00004E31       MyDevBlock_
 0002:000003DA       MY_DEVHELP_ATTACHDD
 0003:00003625       os2gettimemsec_
 0003:00003602       os2gettimesec_
 0003:0000F488       OSS32_APMResume_
 0003:0000F535       OSS32_APMSuspend_
 0003:00004E05       OSS32_CloseUNI16_
 0003:00004E83       OSS32_DebugString_
 0003:00004A47       OSS32_Initialize_
 0003:00005371       OSS32_MidiClose_
 0003:0000563D       OSS32_MidiCommand_
 0003:00004EBA       OSS32_MidiOpen_
 0003:00005605       OSS32_MidiQueryCaps_
 0003:00005551       OSS32_MidiRead_
 0003:00005519       OSS32_MidiWrite_
 0003:00005F55       OSS32_MixClose_
 0003:000069C7       OSS32_MixGetProperty_
 0003:00005FE5       OSS32_MixGetVolume_
 0003:0000586D       OSS32_MixOpen_
 0003:00006B97       OSS32_MixQueryCaps_
 0003:00006C7D       OSS32_MixQueryName_
 0003:00006521       OSS32_MixSetProperty_
 0003:00006036       OSS32_MixSetVolume_
 0003:00004DA9       OSS32_ProcessIRQ_
 0003:00004DD5       OSS32_ProcessMIDIIRQ_
 0003:00007629       OSS32_QueryDevCaps_
 0003:00006DDB       OSS32_QueryNames_
 0003:000040B6       OSS32_SetFileId_
 0003:00004D0C       OSS32_Shutdown_
 0003:00008F7D       OSS32_WaveAddBuffer_
 0003:00007EAE       OSS32_WaveClose_
 0003:0000941B       OSS32_WaveGetHwPtr_
 0003:0000928C       OSS32_WaveGetPosition_
 0003:0000936D       OSS32_WaveGetSpace_
 0003:000094C1       OSS32_WaveGetStatus_
 0003:00007BD1       OSS32_WaveOpen_
 0003:000081FB       OSS32_WavePause_
 0003:00008035       OSS32_WavePrepare_
 0003:00008289       OSS32_WaveResume_
 0003:0000831A       OSS32_WaveSetHwParams_
 0003:00009561       OSS32_WaveSetVolume_
 0003:000080DF       OSS32_WaveStart_
 0003:0000816D       OSS32_WaveStop_
 0003:00006A18       OSSToALSAVolume_
 0003:0000F5F5       PciAdjustInterrupts_
 0003:0000D633       pcibios_present_
 0003:0000CDE6       pcidev_activate_
 0003:0000CE1D       pcidev_deactivate_
 0003:0000CDAF       pcidev_prepare_
 0003:0000DE50       pci_alloc_consistent_
 0003:0000E2B1       pci_disable_device_
 0003:0000D69F       pci_dma_supported_
 0003:0000D958       pci_enable_device_
 0003:0000D6D3       pci_find_capability_
 0003:0000D355       pci_find_device_
 0003:0000D663       pci_find_slot_
 0003:0000DF7E       pci_free_consistent_
 0003:0000E017       pci_get_dma_mask_
 0003:0000DFDE       pci_get_driver_data_
 0003:0000D5E5       pci_get_flags_
 0003:0005380F       pci_iomap_
 0003:00053A3F       pci_iounmap_
 0003:0000F292       pci_match_device_
 0003:0000DBBC       pci_module_init_
 0003:0000E105       pci_orig_restore_state_
 0003:0000E0AD       pci_orig_save_state_
 0003:0000CB3F       pci_read_config_byte_
 0003:0000CC19       pci_read_config_dword_
 0003:0000CBAB       pci_read_config_word_
 0003:0000D9C0       pci_register_driver_
 0003:0000F257       pci_release_regions_
 0003:0000ED57       pci_release_region_
 0003:0000F1E8       pci_request_regions_
 0003:0000E2FB       pci_request_region_
 0003:0000E22D       pci_restore_state_
 0003:0000E1AC       pci_save_state_
 0003:0000DFB0       pci_set_driver_data_
 0003:0000E075       pci_set_latency_time_
 0003:0000DD52       pci_set_master_
 0003:0000D78B       pci_set_power_state_
 0003:0000DBFA       pci_unregister_driver_
 0003:0000CC7E       pci_write_config_byte_
 0003:0000CD4F       pci_write_config_dword_
 0003:0000CCE6       pci_write_config_word_
 0003:0001EB01       pcm_info_
 0003:0001EBE6       pcm_instances_
 0005:00001778       PDDName
 0001:00000466       pddname16
 0003:00009FAF       phys_to_virt_
 0003:0000DDAE       pm_register_
 0003:0000DDE3       pm_unregister_
 0003:00004218       poll_wait_
 0003:0000C996       process_interrupt_
 0003:00004372       proc_register_
 0003:00004398       proc_unregister_
 0003:0007D777       query_amp_caps_
 0003:000876A2       queueptr_
 0003:0000453B       queue_work_
 0003:00006FD1       register_chrdev_
 0003:0000447A       register_reboot_notifier_
 0003:00007148       register_sound_dsp_
 0003:000070F6       register_sound_midi_
 0003:000070A4       register_sound_mixer_
 0003:00007052       register_sound_special_
 0003:0000719A       register_sound_synth_
 0003:000CE77B       release_and_free_resource_
 0003:0000492C       release_firmware_
 0003:0000E050       release_resource_
 0003:0000A535       remap_page_range_
 0003:00004356       remove_proc_entry_
 0003:0001014C       remove_wait_queue_
 0003:00004403       request_dma_
 0003:00004882       request_firmware_
 0003:0000C686       request_irq_
 0005:0000177C       RMAllocResource1632
 0005:0000179C       RMCreateAdapter1632
 0005:00001794       RMCreateDevice1632
 0005:000017A4       RMCreateDriver1632
 0003:00002DB4       RMDeallocateIRQ_
 0005:0000178C       RMDeallocResource1632
 0005:000017AC       RMDestroyDriver1632
 0005:000017BC       RMDevIDToHandleList1632
 0003:00002E2D       RMDone_
 0005:000017B4       RMGetNodeInfo1632
 0005:000017C4       RMHandleToResourceHandleList1632
 0003:000028EC       RMInit_
 0005:00001784       RMModifyResources1632
 0003:00002A9B       RMRequestIO_
 0003:00002C6E       RMRequestIRQ_
 0003:00002B8B       RMRequestMem_
 0003:000032FA       RMSetHandles_
 0003:00004200       schedule_
 0003:00003DCA       schedule_timeout_
 0003:0000AC67       SetPCMInstance_
 0003:000D9229       snd_ac97_bus_
 0003:000DCB40       snd_ac97_bus_proc_done_
 0003:000DCAB6       snd_ac97_bus_proc_init_
 0003:000D8EEB       snd_ac97_get_name_
 0003:000D90C3       snd_ac97_get_short_name_
 0003:000D9315       snd_ac97_mixer_
 0003:000CF2F3       snd_ac97_pcm_assign_
 0003:000CFA9F       snd_ac97_pcm_close_
 0003:000CFC90       snd_ac97_pcm_double_rate_rules_
 0003:000CF744       snd_ac97_pcm_open_
 0003:000DCA71       snd_ac97_proc_done_
 0003:000DC8DC       snd_ac97_proc_init_
 0003:000D5CC5       snd_ac97_read_
 0003:000DA3E5       snd_ac97_resume_
 0003:000CEC8F       snd_ac97_set_rate_
 0003:000DA262       snd_ac97_suspend_
 0003:000DAF29       snd_ac97_tune_hardware_
 0003:000D5E39       snd_ac97_update_
 0003:000D5F08       snd_ac97_update_bits_
 0003:000D5F7D       snd_ac97_update_bits_nolock_
 0003:000D5C4B       snd_ac97_write_
 0003:000D5DAE       snd_ac97_write_cache_
 0003:0001F182       snd_add_device_sysfs_file_
 0003:0008240A       snd_array_free_
 0003:00082300       snd_array_new_
 0003:00053C96       snd_ca0106_i2c_write_
 0003:00057EA1       snd_ca0106_mixer_
 0003:00058196       snd_ca0106_mixer_resume_
 0003:00058137       snd_ca0106_mixer_suspend_
 0003:00058E4C       snd_ca0106_proc_init_
 0003:00053AB5       snd_ca0106_ptr_read_
 0003:00053B1B       snd_ca0106_ptr_write_
 0003:00053B79       snd_ca0106_spi_write_
 0003:0002C7EE       snd_card_create_
 0003:0002CDAB       snd_card_disconnect_
 0003:0002D899       snd_card_file_add_
 0003:0002D969       snd_card_file_remove_
 0003:0002D0D1       snd_card_free_
 0003:0002D013       snd_card_free_when_closed_
 0003:0002D75F       snd_card_info_done_
 0003:0002D6A6       snd_card_info_init_
 0003:0002D5B6       snd_card_info_read_oss_
 0003:0002CB61       snd_card_locked_
 0003:000209E0       snd_card_proc_new_
 0003:0002D414       snd_card_register_
 0003:0002D3CE       snd_card_set_id_
 0003:0002D795       snd_component_add_
 0003:00098DC3       snd_cs46xx_create_
 0003:0009595E       snd_cs46xx_download_
 0003:000959EB       snd_cs46xx_download_image_
 0003:00097C9F       snd_cs46xx_gameport_
 0003:00097BC0       snd_cs46xx_midi_
 0003:000974D1       snd_cs46xx_mixer_
 0003:000970A6       snd_cs46xx_pcm_
 0003:00098C6A       snd_cs46xx_resume_
 0003:000985DB       snd_cs46xx_start_dsp_
 0003:00098B16       snd_cs46xx_suspend_
 0003:0009AA28       snd_cs5535audio_pcm_
 0003:00099E52       snd_cs5535audio_resume_
 0003:00099D48       snd_cs5535audio_suspend_
 0003:00029A08       snd_ctl_add_
 0003:0002BEC7       snd_ctl_boolean_mono_info_
 0003:0002BF15       snd_ctl_boolean_stereo_info_
 0003:0002BE73       snd_ctl_create_
 0003:00029EDF       snd_ctl_find_id_
 0003:00029E52       snd_ctl_find_numid_
 0003:00029878       snd_ctl_free_one_
 0003:000CE659       snd_ctl_make_virtual_master_
 0003:0002970E       snd_ctl_new1_
 0003:000294FF       snd_ctl_notify_
 0003:0002BA91       snd_ctl_register_ioctl_
 0003:00029B9B       snd_ctl_remove_
 0003:00029C67       snd_ctl_remove_id_
 0003:00029DB8       snd_ctl_rename_id_
 0003:0002BB82       snd_ctl_unregister_ioctl_
 0003:00028C9C       snd_device_disconnect_
 0003:00028EF2       snd_device_disconnect_all_
 0003:00028B71       snd_device_free_
 0003:00028F77       snd_device_free_all_
 0003:00028AA4       snd_device_new_
 0003:00028D6F       snd_device_register_
 0003:00028E4B       snd_device_register_all_
 0003:0002C17A       snd_dma_alloc_pages_
 0003:0002C28B       snd_dma_alloc_pages_fallback_
 0003:0002C328       snd_dma_free_pages_
 0003:0002C3AE       snd_dma_get_reserved_buf_
 0003:0002C4D3       snd_dma_reserve_buf_
 0003:000B07A5       snd_emu1010_fpga_link_dst_src_write_
 0003:000B0704       snd_emu1010_fpga_read_
 0003:000B063E       snd_emu1010_fpga_write_
 0003:000B0E37       snd_emu10k1_ac97_read_
 0003:000B0EA0       snd_emu10k1_ac97_write_
 0003:000B1AFE       snd_emu10k1_alloc_pages_
 0003:000AC600       snd_emu10k1_audigy_midi_
 0003:000AE43D       snd_emu10k1_create_
 0003:000AD0D7       snd_emu10k1_done_
 0003:000A461B       snd_emu10k1_efx_alloc_pm_buffer_
 0003:000A4752       snd_emu10k1_efx_free_pm_buffer_
 0003:0009D155       snd_emu10k1_efx_read_
 0003:000A494A       snd_emu10k1_efx_resume_
 0003:000A47A5       snd_emu10k1_efx_suspend_
 0003:000A3937       snd_emu10k1_free_efx_
 0003:000B1CCB       snd_emu10k1_free_pages_
 0003:000A4545       snd_emu10k1_fx8010_new_
 0003:0009CDE8       snd_emu10k1_fx8010_register_irq_handler_
 0003:000A39A7       snd_emu10k1_fx8010_tram_setup_
 0003:0009CED6       snd_emu10k1_fx8010_unregister_irq_handler_
 0003:000B04CA       snd_emu10k1_i2c_write_
 0003:000A38C9       snd_emu10k1_init_efx_
 0003:000B231A       snd_emu10k1_interrupt_
 0003:000B0875       snd_emu10k1_intr_disable_
 0003:000B081B       snd_emu10k1_intr_enable_
 0003:000B19BE       snd_emu10k1_memblk_map_
 0003:000AC571       snd_emu10k1_midi_
 0003:000A71A1       snd_emu10k1_mixer_
 0003:000AABFE       snd_emu10k1_pcm_
 0003:000ABA37       snd_emu10k1_pcm_efx_
 0003:000AAEA2       snd_emu10k1_pcm_mic_
 0003:000AAD79       snd_emu10k1_pcm_multi_
 0003:000AFD4C       snd_emu10k1_proc_init_
 0003:000B029A       snd_emu10k1_ptr20_read_
 0003:000B0307       snd_emu10k1_ptr20_write_
 0003:000B004C       snd_emu10k1_ptr_read_
 0003:000B015D       snd_emu10k1_ptr_write_
 0003:000B0F01       snd_emu10k1_rate_to_pitch_
 0003:000AEF13       snd_emu10k1_resume_init_
 0003:000AEF9B       snd_emu10k1_resume_regs_
 0003:000B036C       snd_emu10k1_spi_write_
 0003:000AEE16       snd_emu10k1_suspend_regs_
 0003:000B1D16       snd_emu10k1_synth_alloc_
 0003:000B2196       snd_emu10k1_synth_bzero_
 0003:000B224C       snd_emu10k1_synth_copy_from_user_
 0003:000B1DBE       snd_emu10k1_synth_free_
 0003:0009C86A       snd_emu10k1_timer_
 0003:000B1182       snd_emu10k1_voice_alloc_
 0003:000B0D0F       snd_emu10k1_voice_clear_loop_stop_
 0003:000B12F0       snd_emu10k1_voice_free_
 0003:000B0BE7       snd_emu10k1_voice_half_loop_intr_ack_
 0003:000B0B41       snd_emu10k1_voice_half_loop_intr_disable_
 0003:000B0A9F       snd_emu10k1_voice_half_loop_intr_enable_
 0003:000AC6FF       snd_emu10k1_voice_init_
 0003:000B0A19       snd_emu10k1_voice_intr_ack_
 0003:000B0973       snd_emu10k1_voice_intr_disable_
 0003:000B08D1       snd_emu10k1_voice_intr_enable_
 0003:000B0C6D       snd_emu10k1_voice_set_loop_stop_
 0003:000B0DB5       snd_emu10k1_wait_
 0003:0002C117       snd_free_dev_pages_
 0003:0002C052       snd_free_pages_
 0003:0002DC18       snd_free_sgbuf_pages_
 0003:0007BA46       snd_hda_add_codec_preset_
 0003:00080DF9       snd_hda_add_new_ctls_
 0003:0007CBD4       snd_hda_add_pincfg_
 0003:0007E7D8       snd_hda_add_vmaster_
 0003:0007FD6D       snd_hda_build_controls_
 0003:00080ACF       snd_hda_build_pcms_
 0003:0007C44B       snd_hda_bus_new_
 0003:0007FE80       snd_hda_calc_stream_format_
 0003:00080CC6       snd_hda_check_board_codec_sid_config_
 0003:00080B37       snd_hda_check_board_config_
 0003:00080F3F       snd_hda_ch_mode_get_
 0003:00080EC2       snd_hda_ch_mode_info_
 0003:00080F9B       snd_hda_ch_mode_put_
 0003:0007DB40       snd_hda_codec_amp_read_
 0003:0007DCB1       snd_hda_codec_amp_stereo_
 0003:0007DBCF       snd_hda_codec_amp_update_
 0003:0007FE0C       snd_hda_codec_build_controls_
 0003:00080999       snd_hda_codec_build_pcms_
 0003:0007D58A       snd_hda_codec_cleanup_stream_
 0003:0007D3C0       snd_hda_codec_configure_
 0003:0007CCBA       snd_hda_codec_get_pincfg_
 0003:0007CF47       snd_hda_codec_new_
 0003:000860AC       snd_hda_codec_proc_new_
 0003:0007BDC2       snd_hda_codec_read_
 0003:0007E56D       snd_hda_codec_reset_
 0003:0007DD19       snd_hda_codec_resume_amp_
 0003:0007F9E4       snd_hda_codec_resume_cache_
 0003:0007D4FE       snd_hda_codec_setup_stream_
 0003:0007CC7D       snd_hda_codec_set_pincfg_
 0003:0007BE14       snd_hda_codec_write_
 0003:0007F933       snd_hda_codec_write_cache_
 0003:0008283B       snd_hda_create_hwdep_
 0003:0007F83F       snd_hda_create_spdif_in_ctls_
 0003:0007F490       snd_hda_create_spdif_out_ctls_
 0003:0007F64F       snd_hda_create_spdif_share_sw_
 0003:0007E45A       snd_hda_ctls_clear_
 0003:0007E3EF       snd_hda_ctl_add_
 0003:0007BAA7       snd_hda_delete_codec_preset_
 0003:0007E3C0       snd_hda_find_mixer_ctl_
 0003:0007BF33       snd_hda_get_connections_
 0003:0007BB9C       snd_hda_get_jack_connectivity_
 0003:0007BB11       snd_hda_get_jack_location_
 0003:0007BBCF       snd_hda_get_jack_type_
 0003:0007BECC       snd_hda_get_sub_nodes_
 0003:0008102D       snd_hda_input_mux_info_
 0003:000810CB       snd_hda_input_mux_put_
 0003:00080413       snd_hda_is_supported_format_
 0003:0007E9A6       snd_hda_mixer_amp_switch_get_
 0003:0007E934       snd_hda_mixer_amp_switch_info_
 0003:0007EA94       snd_hda_mixer_amp_switch_put_
 0003:0007E178       snd_hda_mixer_amp_tlv_
 0003:0007DFAB       snd_hda_mixer_amp_volume_get_
 0003:0007DDFF       snd_hda_mixer_amp_volume_info_
 0003:0007E086       snd_hda_mixer_amp_volume_put_
 0003:0007ED65       snd_hda_mixer_bind_ctls_get_
 0003:0007ECEF       snd_hda_mixer_bind_ctls_info_
 0003:0007EDDC       snd_hda_mixer_bind_ctls_put_
 0003:0007EBA5       snd_hda_mixer_bind_switch_get_
 0003:0007EC1B       snd_hda_mixer_bind_switch_put_
 0003:0007EE9C       snd_hda_mixer_bind_tlv_
 0003:000817C4       snd_hda_multi_out_analog_cleanup_
 0003:00081414       snd_hda_multi_out_analog_open_
 0003:000815C5       snd_hda_multi_out_analog_prepare_
 0003:00081379       snd_hda_multi_out_dig_cleanup_
 0003:000813CA       snd_hda_multi_out_dig_close_
 0003:000812BA       snd_hda_multi_out_dig_open_
 0003:0008131E       snd_hda_multi_out_dig_prepare_
 0003:0007D853       snd_hda_override_amp_caps_
 0003:0008482A       snd_hda_parse_generic_codec_
 0003:000819EA       snd_hda_parse_pin_def_config_
 0003:0007D98C       snd_hda_query_pin_caps_
 0003:0007C23B       snd_hda_queue_unsol_event_
 0003:000822A9       snd_hda_resume_
 0003:0007BE80       snd_hda_sequence_write_
 0003:0007FA6C       snd_hda_sequence_write_cache_
 0003:0007E2AF       snd_hda_set_vmaster_tlv_
 0003:00082252       snd_hda_suspend_
 0003:00010D85       snd_hwdep_new_
 0003:000202D7       snd_info_card_create_
 0003:00020461       snd_info_card_disconnect_
 0003:000204F3       snd_info_card_free_
 0003:000203F1       snd_info_card_id_change_
 0003:0002038B       snd_info_card_register_
 0003:0001F51B       snd_info_check_reserved_words_
 0003:00020858       snd_info_create_card_entry_
 0003:0002080F       snd_info_create_module_entry_
 0003:00020255       snd_info_done_
 0003:00020A69       snd_info_free_entry_
 0003:00020542       snd_info_get_line_
 0003:0002064C       snd_info_get_str_
 0003:00020149       snd_info_init_
 0003:00028319       snd_info_minor_register_
 0003:00028397       snd_info_minor_unregister_
 0003:00020AD5       snd_info_register_
 0003:0001A40A       snd_interval_div_
 0003:0001AEAA       snd_interval_list_
 0003:0001A55F       snd_interval_muldivk_
 0003:0001A69C       snd_interval_mulkdiv_
 0003:0001A2AE       snd_interval_mul_
 0003:0001A7F8       snd_interval_ratnum_
 0003:00019FCF       snd_interval_refine_
 0003:00009AD5       snd_iprintf_
 0003:0001ECBC       snd_lookup_minor_data_
 0003:000283CD       snd_lookup_oss_minor_data_
 0003:0002C0A2       snd_malloc_dev_pages_
 0003:0002BFE6       snd_malloc_pages_
 0003:0002DC94       snd_malloc_sgbuf_pages_
 0003:000DDB1D       snd_midi_channel_alloc_set_
 0003:000DDBBD       snd_midi_channel_free_set_
 0003:000DD3A9       snd_midi_channel_set_clear_
 0003:000DCB70       snd_midi_process_event_
 0003:0001F3A0       snd_minor_info_done_
 0003:0001F337       snd_minor_info_init_
 0003:00028A39       snd_minor_info_oss_done_
 0003:000289CC       snd_minor_info_oss_init_
 0003:00093D17       snd_mpu401_uart_interrupt_
 0003:00093D5A       snd_mpu401_uart_interrupt_tx_
 0003:00094735       snd_mpu401_uart_new_
 0003:00091BE5       snd_opl3_calc_volume_
 0003:000934BC       snd_opl3_clear_patches_
 0003:00092D13       snd_opl3_control_
 0003:00091338       snd_opl3_create_
 0003:00091AE5       snd_opl3_drum_switch_
 0003:000933D2       snd_opl3_find_patch_
 0003:00091589       snd_opl3_hwdep_new_
 0003:00091284       snd_opl3_init_
 0003:00091098       snd_opl3_interrupt_
 0003:00092E42       snd_opl3_ioctl_
 0003:00092B0D       snd_opl3_key_press_
 0003:00091A55       snd_opl3_load_drums_
 0003:000931D2       snd_opl3_load_patch_
 0003:000911C6       snd_opl3_new_
 0003:000929FA       snd_opl3_note_off_
 0003:000920F6       snd_opl3_note_on_
 0003:00092DD3       snd_opl3_nrpn_
 0003:00092E1C       snd_opl3_open_
 0003:0009307C       snd_opl3_release_
 0003:0009352C       snd_opl3_reset_
 0003:0009052F       snd_opl3_synth_cleanup_
 0003:00090428       snd_opl3_synth_setup_
 0003:000903F4       snd_opl3_synth_use_dec_
 0003:000903B3       snd_opl3_synth_use_inc_
 0003:00092DF6       snd_opl3_sysex_
 0003:00092B31       snd_opl3_terminate_note_
 0003:00091FA1       snd_opl3_timer_func_
 0003:00091503       snd_opl3_timer_new_
 0003:000930B6       snd_opl3_write_
 0003:00028080       snd_oss_info_register_
 0003:0009C5F9       snd_p16v_alloc_pm_buffer_
 0003:0009BE9D       snd_p16v_free_
 0003:0009C648       snd_p16v_free_pm_buffer_
 0003:0009C583       snd_p16v_mixer_
 0003:0009BED6       snd_p16v_pcm_
 0003:0009C6E1       snd_p16v_resume_
 0003:0009C671       snd_p16v_suspend_
 0003:0000F447       snd_pci_compat_get_pci_driver_
 0003:0000F390       snd_pci_dev_present_
 0003:000CE7AC       snd_pci_quirk_lookup_
 0003:0001E036       snd_pcm_attach_substream_
 0003:0001E451       snd_pcm_detach_substream_
 0003:00023BAF       snd_pcm_drain_done_
 0003:000185A1       snd_pcm_format_big_endian_
 0003:00018509       snd_pcm_format_linear_
 0003:00018549       snd_pcm_format_little_endian_
 0003:0001864B       snd_pcm_format_physical_width_
 0003:00018742       snd_pcm_format_set_silence_
 0003:0001845E       snd_pcm_format_signed_
 0003:000186E8       snd_pcm_format_silence_64_
 0003:000186A2       snd_pcm_format_size_
 0003:000184B6       snd_pcm_format_unsigned_
 0003:000185F4       snd_pcm_format_width_
 0003:00025D1E       snd_pcm_hw_constraints_complete_
 0003:0002577C       snd_pcm_hw_constraints_init_
 0003:0001B2F7       snd_pcm_hw_constraint_integer_
 0003:0001B45A       snd_pcm_hw_constraint_list_
 0003:0001B252       snd_pcm_hw_constraint_mask64_
 0003:0001B1D5       snd_pcm_hw_constraint_mask_
 0003:0001B34F       snd_pcm_hw_constraint_minmax_
 0003:0001B753       snd_pcm_hw_constraint_msbits_
 0003:0001B8C8       snd_pcm_hw_constraint_pow2_
 0003:0001B66E       snd_pcm_hw_constraint_ratdens_
 0003:0001B564       snd_pcm_hw_constraint_ratnums_
 0003:0001B811       snd_pcm_hw_constraint_step_
 0003:0001C089       snd_pcm_hw_params_choose_
 0003:0001BE66       snd_pcm_hw_param_first_
 0003:0001C004       snd_pcm_hw_param_last_
 0003:0001BAB9       snd_pcm_hw_param_value_
 0003:00021F2E       snd_pcm_hw_refine_
 0003:0001B05D       snd_pcm_hw_rule_add_
 0003:00021D76       snd_pcm_info_
 0003:00021EB1       snd_pcm_info_user_
 0003:00027A7C       snd_pcm_kernel_ioctl_
 0003:00021257       snd_pcm_lib_free_pages_
 0003:0001C381       snd_pcm_lib_ioctl_
 0003:00021112       snd_pcm_lib_malloc_pages_
 0003:00020E33       snd_pcm_lib_preallocate_free_
 0003:00020E60       snd_pcm_lib_preallocate_free_for_all_
 0003:00020F41       snd_pcm_lib_preallocate_pages_
 0003:00020F87       snd_pcm_lib_preallocate_pages_for_all_
 0003:0001D585       snd_pcm_lib_readv_
 0003:0001D32C       snd_pcm_lib_read_
 0003:0001CE50       snd_pcm_lib_writev_
 0003:0001CB8D       snd_pcm_lib_write_
 0003:00018902       snd_pcm_limit_hw_rates_
 0003:0001DD65       snd_pcm_new_
 0003:0001DAF0       snd_pcm_new_stream_
 0003:0001E87C       snd_pcm_notify_
 0003:00026087       snd_pcm_open_substream_
 0003:000CA34A       snd_pcm_oss_read3_
 0003:000CA543       snd_pcm_oss_readv3_
 0003:000CA279       snd_pcm_oss_write3_
 0003:000CA472       snd_pcm_oss_writev3_
 0003:0001C403       snd_pcm_period_elapsed_
 0003:00019330       snd_pcm_playback_silence_
 0003:000189B7       snd_pcm_rate_to_rate_bit_
 0003:00025FE6       snd_pcm_release_substream_
 0003:00019D57       snd_pcm_set_ops_
 0003:00019DA9       snd_pcm_set_sync_
 0003:0002106E       snd_pcm_sgbuf_get_chunk_size_
 0003:0002100D       snd_pcm_sgbuf_ops_page_
 0003:00023A31       snd_pcm_start_
 0003:00022FBF       snd_pcm_status_
 0003:00023B7D       snd_pcm_stop_
 0003:00023F0A       snd_pcm_suspend_
 0003:00023F80       snd_pcm_suspend_all_
 0003:0002167F       snd_pcm_timer_done_
 0003:00021564       snd_pcm_timer_init_
 0003:0002134D       snd_pcm_timer_resolution_change_
 0003:00019BCD       snd_pcm_update_hw_ptr_
 0003:0002DAC4       snd_power_wait_
 0003:000824C9       snd_print_pcm_bits_
 0003:0008244D       snd_print_pcm_rates_
 0003:000158C3       snd_rawmidi_drain_input_
 0003:000157EF       snd_rawmidi_drain_output_
 0003:00015776       snd_rawmidi_drop_output_
 0003:00016410       snd_rawmidi_info_select_
 0003:00016720       snd_rawmidi_input_params_
 0003:00015C0E       snd_rawmidi_kernel_open_
 0003:00016CE3       snd_rawmidi_kernel_read_
 0003:0001620D       snd_rawmidi_kernel_release_
 0003:00017467       snd_rawmidi_kernel_write_
 0003:00017AD4       snd_rawmidi_new_
 0003:000165D5       snd_rawmidi_output_params_
 0003:0001692B       snd_rawmidi_receive_
 0003:00018301       snd_rawmidi_set_ops_
 0003:000171FF       snd_rawmidi_transmit_
 0003:000170FE       snd_rawmidi_transmit_ack_
 0003:00016F0D       snd_rawmidi_transmit_empty_
 0003:00016F97       snd_rawmidi_transmit_peek_
 0003:0001EF3C       snd_register_device_for_dev_
 0003:000285DD       snd_register_oss_device_
 0003:000C6866       snd_sbdsp_command_
 0003:000C6CED       snd_sbdsp_create_
 0003:000C68E5       snd_sbdsp_get_byte_
 0003:000C6961       snd_sbdsp_reset_
 0003:000C6254       snd_sbmixer_add_ctl_
 0003:000C6406       snd_sbmixer_new_
 0003:000C547B       snd_sbmixer_read_
 0003:000C6799       snd_sbmixer_resume_
 0003:000C66CC       snd_sbmixer_suspend_
 0003:000C5430       snd_sbmixer_write_
 0003:0008D15D       snd_sequencer_device_done_
 0003:0008D0E4       snd_sequencer_device_init_
 0003:000891FD       snd_sequencer_memory_done_
 0003:000891DB       snd_sequencer_memory_init_
 0003:0008895F       snd_seq_cell_free_
 0003:0008776F       snd_seq_check_queue_
 0003:0008B10F       snd_seq_client_notify_subscription_
 0003:00089422       snd_seq_client_use_ptr_
 0003:00088368       snd_seq_control_queue_
 0003:0008C71F       snd_seq_create_kernel_client_
 0003:0008D439       snd_seq_create_port_
 0003:0008D9C5       snd_seq_delete_all_ports_
 0003:0008C861       snd_seq_delete_kernel_client_
 0003:0008D8D2       snd_seq_delete_port_
 0003:00086308       snd_seq_device_load_drivers_
 0003:00086320       snd_seq_device_new_
 0003:0008667B       snd_seq_device_register_driver_
 0003:00086868       snd_seq_device_unregister_driver_
 0003:0008A230       snd_seq_dispatch_event_
 0003:0008864D       snd_seq_dump_var_event_
 0003:000878F8       snd_seq_enqueue_event_
 0003:00088C04       snd_seq_event_dup_
 0003:0008E57D       snd_seq_event_port_attach_
 0003:0008E639       snd_seq_event_port_detach_
 0003:00088826       snd_seq_expand_var_event_
 0003:000900FC       snd_seq_fifo_cell_out_
 0003:0009020C       snd_seq_fifo_cell_putback_
 0003:0008FF50       snd_seq_fifo_clear_
 0003:0008FEAA       snd_seq_fifo_delete_
 0003:0008FFA9       snd_seq_fifo_event_in_
 0003:0008FDC7       snd_seq_fifo_new_
 0003:00090262       snd_seq_fifo_poll_wait_
 0003:000902B2       snd_seq_fifo_resize_
 0003:0008DC83       snd_seq_get_port_info_
 0003:0008CF0C       snd_seq_info_clients_read_
 0003:00086E5B       snd_seq_info_done_
 0003:00086DFD       snd_seq_info_init_
 0003:00089215       snd_seq_info_pool_
 0003:00088405       snd_seq_info_queues_read_
 0003:0008F271       snd_seq_info_timer_read_
 0003:0008CACF       snd_seq_kernel_client_ctl_
 0003:0008CA22       snd_seq_kernel_client_dispatch_
 0003:0008C9A6       snd_seq_kernel_client_enqueue_
 0003:0008C9E1       snd_seq_kernel_client_enqueue_blocking_
 0003:0008CB39       snd_seq_kernel_client_write_poll_
 0003:00089186       snd_seq_pool_delete_
 0003:00088FA9       snd_seq_pool_done_
 0003:00088E85       snd_seq_pool_init_
 0003:000890D9       snd_seq_pool_new_
 0003:00088E12       snd_seq_pool_poll_wait_
 0003:0008E007       snd_seq_port_connect_
 0003:0008E346       snd_seq_port_disconnect_
 0003:0008E4FD       snd_seq_port_get_subscription_
 0003:0008D2FB       snd_seq_port_query_nearest_
 0003:0008D24C       snd_seq_port_use_ptr_
 0003:0008F81B       snd_seq_prioq_avail_
 0003:0008F5F2       snd_seq_prioq_cell_in_
 0003:0008F783       snd_seq_prioq_cell_out_
 0003:0008F85F       snd_seq_prioq_cell_peek_
 0003:0008F438       snd_seq_prioq_delete_
 0003:0008F94C       snd_seq_prioq_leave_
 0003:0008F3C0       snd_seq_prioq_new_
 0003:0008FC71       snd_seq_prioq_remove_events_
 0003:00087578       snd_seq_queues_delete_
 0003:00087556       snd_seq_queues_init_
 0003:000875C5       snd_seq_queue_alloc_
 0003:00087AF7       snd_seq_queue_check_access_
 0003:00087F7B       snd_seq_queue_client_leave_
 0003:0008803E       snd_seq_queue_client_leave_cells_
 0003:00087EDD       snd_seq_queue_client_termination_
 0003:00087642       snd_seq_queue_delete_
 0003:00087705       snd_seq_queue_find_name_
 0003:00087284       snd_seq_queue_get_cur_queues_
 0003:00087E68       snd_seq_queue_is_used_
 0003:000880A1       snd_seq_queue_remove_cells_
 0003:00087B5D       snd_seq_queue_set_owner_
 0003:00087C75       snd_seq_queue_timer_close_
 0003:00087C03       snd_seq_queue_timer_open_
 0003:00087CCB       snd_seq_queue_timer_set_tempo_
 0003:00087D87       snd_seq_queue_use_
 0003:0008DB2D       snd_seq_set_port_info_
 0003:0008B983       snd_seq_set_queue_tempo_
 0003:00086F1B       snd_seq_system_broadcast_
 0003:00087170       snd_seq_system_client_done_
 0003:00086FFA       snd_seq_system_client_init_
 0003:00086F63       snd_seq_system_notify_
 0003:0008EEC7       snd_seq_timer_close_
 0003:0008F11D       snd_seq_timer_continue_
 0003:0008E88D       snd_seq_timer_defaults_
 0003:0008E82D       snd_seq_timer_delete_
 0003:0008F24A       snd_seq_timer_get_cur_tick_
 0003:0008F1AC       snd_seq_timer_get_cur_time_
 0003:0008E7C2       snd_seq_timer_new_
 0003:0008ED61       snd_seq_timer_open_
 0003:0008E941       snd_seq_timer_reset_
 0003:0008EBF5       snd_seq_timer_set_position_tick_
 0003:0008EC65       snd_seq_timer_set_position_time_
 0003:0008EB2C       snd_seq_timer_set_ppq_
 0003:0008ECD6       snd_seq_timer_set_skew_
 0003:0008EA95       snd_seq_timer_set_tempo_
 0003:0008F097       snd_seq_timer_start_
 0003:0008EF3C       snd_seq_timer_stop_
 0003:00011B24       snd_timer_close_
 0003:0001237B       snd_timer_continue_
 0003:000131C7       snd_timer_global_free_
 0003:00013172       snd_timer_global_new_
 0003:000131F0       snd_timer_global_register_
 0003:00012646       snd_timer_interrupt_
 0003:00012ADD       snd_timer_new_
 0003:00013033       snd_timer_notify_
 0003:000118A4       snd_timer_open_
 0003:00012445       snd_timer_pause_
 0003:00011DB7       snd_timer_resolution_
 0003:000120C7       snd_timer_start_
 0003:000122FB       snd_timer_stop_
 0003:000C29A7       snd_trident_alloc_pages_
 0003:000C1F27       snd_trident_alloc_voice_
 0003:000C1745       snd_trident_create_
 0003:000C0E19       snd_trident_create_gameport_
 0003:000BF3B6       snd_trident_foldback_pcm_
 0003:000C2A0B       snd_trident_free_pages_
 0003:000C207E       snd_trident_free_voice_
 0003:000BF200       snd_trident_pcm_
 0003:000C2384       snd_trident_resume_
 0003:000BF5CD       snd_trident_spdif_pcm_
 0003:000BCA64       snd_trident_start_voice_
 0003:000BCABD       snd_trident_stop_voice_
 0003:000C22B9       snd_trident_suspend_
 0003:000BCCC0       snd_trident_write_voice_regs_
 0003:0001F0FC       snd_unregister_device_
 0003:0002875C       snd_unregister_oss_device_
 0003:000DDCDC       snd_util_memhdr_free_
 0003:000DDC6C       snd_util_memhdr_new_
 0003:000DDEE9       snd_util_mem_alloc_
 0003:000DDFFD       snd_util_mem_avail_
 0003:000DDF98       snd_util_mem_free_
 0003:000B8763       snd_ymfpci_create_
 0003:000B286B       snd_ymfpci_free_gameport_
 0003:000B6DCB       snd_ymfpci_mixer_
 0003:000B595C       snd_ymfpci_pcm2_
 0003:000B5858       snd_ymfpci_pcm_
 0003:000B5B4C       snd_ymfpci_pcm_4ch_
 0003:000B5A5A       snd_ymfpci_pcm_spdif_
 0003:000B85D5       snd_ymfpci_resume_
 0003:000B844D       snd_ymfpci_suspend_
 0003:000B72B4       snd_ymfpci_timer_
 0003:000DE330       snprintf_
 0003:0001025D       spin_lock_
 0003:00010282       spin_lock_flag_
 0003:00010239       spin_lock_init_
 0003:000102A8       spin_trylock_
 0003:000102CD       spin_unlock_
 0003:00003D2D       sprintf_
 0003:000DE260       sscanf_
 0005:00001768       stackbase
 0005:0000176C       stacksel
 0003:00000080       STRATEGY_
 0003:00003F70       strcmp_
 0003:0000994D       StringOut_
 0003:000DE1A0       strlcpy_
 0003:000CD940       StrLen
 0003:000CD960       StrNCmp
 0003:00003FCD       strncmp_
 0003:00010093       strncpy_
 0003:000DE0F0       strstr_
 0003:000DE610       strtol_
 0003:000DE600       strtoul_
 0003:000E0340       strupr_
 0003:0000403C       tasklet_hi_schedule_
 0003:00004074       tasklet_init_
 0003:00000024       thunk1632_devhelp
 0003:00000044       thunk1632_devhelp_modified_ds
 0002:000001A0       thunk3216_devhelp
 0002:000001B2       thunk3216_devhelp_modified_ds
 0003:00000140       TIMER_
 0003:000E02E0       tolower_
 0003:000E0670       ulltoa_
 0003:000E05F0       ultoa_
 0003:0000C570       UniaudCloseAll_
 0003:0000B4CC       UniaudCtlGetPowerState_
 0003:0000B5E8       UniaudCtlSetPowerState_
 0003:0000C189       UniaudIoctlHWParamSet_
 0003:0000C109       UniaudIoctlHWRefine_
 0003:0000C50E       UniaudIoctlPCMDrop_
 0003:0000C3E6       UniaudIoctlPCMPrepare_
 0003:0000C374       UniaudIoctlPCMRead_
 0003:0000C448       UniaudIoctlPCMResume_
 0003:0000C4AC       UniaudIoctlPCMStart_
 0003:0000C289       UniaudIoctlPCMStatus_
 0003:0000C302       UniaudIoctlPCMWrite_
 0003:0000C209       UniaudIoctlSWParamSet_
 0001:0000001E       uniaud_header
 0003:0000A9B0       uniaud_set_interrupted_substream_
 0002:0000010A       uniaud_stub_idc
 0002:00000096       uniaud_stub_strategy
 0002:00000128       uniaud_stub_timer
 0003:000072C8       UNIXToOSSError_
 0003:00007011       unregister_chrdev_
 0003:0000449F       unregister_reboot_notifier_
 0003:00007270       unregister_sound_dsp_
 0003:00007244       unregister_sound_midi_
 0003:00007218       unregister_sound_mixer_
 0003:000071EC       unregister_sound_special_
 0003:0000729C       unregister_sound_synth_
 0003:000CDC9A       up_
 0003:000E0710       utoa_
 0003:0000A4CB       vfree_
 0003:00009F65       virt_to_phys_
 0003:0000A00E       VMAlloc_
 0003:0000A453       vmalloc_
 0003:0000A0D8       VMFree_
 0003:000DE2D0       vsnprintf_
 0003:00003947       vsprintf_
 0003:000DE230       vsscanf_
 0003:000035A5       W?$dln(pnv)v
 0003:0000357C       W?$nwn(ui)pnv
 0003:000035C8       W?$nwn(uipnv)pnv
 0005:00000554       W?acHeap$npnuc
 0003:000049DF       W?CallOSS16$n(ululul)ul
 0003:00001096       W?CheckCardName$n(pfa)v
 0003:0000FCBC       W?compact$n()v
 0005:00000030       W?deviceOwner$nul
 0003:0000084E       W?DevSaveMessage$n(pfai)v
 0003:00000A0D       W?DiscardableInit$n(pf$RPInit$$)ul
 0003:00001313       W?DoParm$n(apfa)i
 0003:0000F764       W?dumpheap$n()v
 0005:000000B0       W?fnCardExitCall$n[]pn()v
 0005:00001894       W?ForceCard$ni
 0003:0000FD84       W?free$n(pnv)v
 0003:0000F951       W?HeapCheck$n(pna)v
 0003:0000FFEB       W?HeapInit$n(ul)ul
 0003:0000FF95       W?IsHeapAddr$n(ul)ul
 0003:00000FC7       W?IsWhitespace$n(a)i
 0003:0000090D       W?LockSegments$n()i
 0003:0000FB5C       W?malloc$n(ul)pnv
 0003:00000E5D       W?mymemchr$n(pfaaus)pfa
 0003:0000FA69       W?npvAllocateBlock$n(pn$_MEMBLOCK$$ulpn$1$)pnv
 0005:00000034       W?numOS2Opens$nul
 0003:000016FC       W?OSS32IDC$n(ulpn$__6ikc0pIDC32_PACKET$$)ul
 0003:0000140E       W?ParseParm$n(pfai)i
 0005:0000054C       W?pmbFree$npn$_MEMBLOCK$$
 0005:00000548       W?pmbUsed$npn$_MEMBLOCK$$
 0003:0000FEE8       W?realloc$n(pnvul)pnv
 0003:0000FC53       W?remove$n(pn$_MEMBLOCK$$)v
 0005:00000060       W?RMFlags$nul
 0005:00000054       W?RM_Help$npn()i
 0005:00000058       W?RM_Help0$npn()i
 0005:0000005C       W?RM_Help3$npn()i
 0003:0000F8A7       W?SignatureCheck$n(pn$_MEMBLOCK$$pna)s
 0003:00001018       W?SkipWhite$n(pfa)pfa
 0003:0000288A       W?StratClose$n(pf$RP$$)ul
 0005:00001800       W?StratDispatch$n[]pn(pf$RP$$)ul
 0003:00000544       W?StratInit$n(pf$RP$$)ul
 0003:000005AE       W?StratInitComplete$n(pf$RP$$)ul
 0003:00001CB3       W?StratIOCtl$n(pf$RP$$)ul
 0003:000004DD       W?StratOpen$n(pf$RP$$)ul
 0003:000006D8       W?StratRead$n(pf$RP$$)ul
 0003:000005E9       W?StratShutdown$n(pf$RP$$)ul
 0003:00000EDC       W?sz2us$n(pfai)us
 0003:00000E1D       W?toupper$n(i)i
 0005:0000055C       W?ulcAlloc$nul
 0005:00000568       W?ulcFree$nul
 0005:0000E9E0       W?ulcTotalHeap$nul
 0005:00000558       W?ulnAlloc$nul
 0005:00000560       W?ulnAllocCalls$nul
 0005:00000570       W?ulnCompact$nul
 0005:00000564       W?ulnFree$nul
 0005:0000056C       W?ulnFreeCalls$nul
 0005:00000550       W?uMemFree$nui
 0003:0000FE86       W?_memfree$n()ui
 0003:0000FEA9       W?_msize$n(pnv)ui
 0003:0000AA16       WaitForControlChange_
 0003:0000AAAF       WaitForPCMInterrupt_
 0003:00010214       waitqueue_active_
 0003:000E04E0       wctomb_
 0005:00002144       _alsa_fops
 0005:00040A23       _auto_pin_cfg_labels
 0003:00000050       _CallPDD16
 0002:0000049A       _CallRM
 0005:00001D04       _cardcalls
 0005:0000A214       _card_id_changed
 0005:0000A210       _control_id_changed
 0005:000081D4       _CountWv
 0005:000018EC       _current
 0005:000018C8       _current_task
 0005:000000D8       _DbgInt
 0005:000000FC       _DebugLevel
 0005:0008ABE0       _edata
 0005:0008ABE0       _end
 0005:00000048       _fDebug
 0005:0000A21C       _fInInterrupt
 0005:0000D5DC       _fRewired
 0005:000000D4       _fStrategyInit
 0005:00000044       _fVerbose
 0005:000081DC       _hextab
 0005:0000004C       _idc16_PddHandler
 0005:00001CB4       _iLastError
 0005:00001A92       _iomem_resource
 0005:00001A76       _ioport_resource
 0003:000E05D0       _ismbblead_
 0005:000017D2       _ISR00
 0005:000017D6       _ISR01
 0005:000017DA       _ISR02
 0005:000017DE       _ISR03
 0005:000017E2       _ISR04
 0005:000017E6       _ISR05
 0005:000017EA       _ISR06
 0005:000017EE       _ISR07
 0005:000018C4       _jiffies
 0000:00000000  Imp  _KernSISData         (KEE.90)
 0005:000081D8       _LockAdd
 0005:000081ED       _MAGIC_COMM_PORT
 0005:00001AAE       _mem_map
 0001:00000060       _MESSAGE_STR
 0005:00001E0C       _midi_port
 0001:00000460       _MSG_TABLE16
 0005:00001774       _MSG_TABLE32
 0005:000000D0       _nrCardsDetected
 0005:00002158       _opened_handles
 0005:00040DC0       _opl3_ops
 0005:00002004       _oss_devices
 0005:0000AA9C       _pci_devices
 0005:000081F0       _pcmcaps
 0005:00002150       _pcm_device
 0005:00002148       _per_bytes
 0005:0000214C       _prev_size
 0003:00004177       _printk
 0005:00001CB8       _proc_root
 0003:0000A822       _put_user_
 0005:00000038       _rdOffset
 0003:0000024C       _RMAllocResource
 0002:00000204       _RMAllocResource16
 0002:000001C8       _RMAllocResourceOrg
 0003:00000358       _RMCreateAdapter
 0002:000002B6       _RMCreateAdapter16
 0002:0000027A       _RMCreateAdapterOrg
 0003:00000310       _RMCreateDevice
 0002:0000031E       _RMCreateDevice16
 0002:000002E2       _RMCreateDeviceOrg
 0003:000003A0       _RMCreateDriver
 0002:0000047A       _RMCreateDriver16
 0002:00000400       _RMCreateDriverOrg
 0003:000002D0       _RMDeallocResource
 0002:000003BA       _RMDeallocResource16
 0002:00000390       _RMDeallocResourceOrg
 0002:00000374       _RMDestroyDevice16
 0002:0000034A       _RMDestroyDeviceOrg
 0003:000003E0       _RMDestroyDriver
 0002:000004F8       _RMDestroyDriver16
 0002:000004CE       _RMDestroyDriverOrg
 0003:0000044C       _RMDevIDToHandleList
 0002:000005A8       _RMDevIDToHandleList16
 0001:0000005C       _RMFlags
 0003:0000040C       _RMGetNodeInfo
 0002:0000054C       _RMGetNodeInfo16
 0003:000004A0       _RMHandleToResourceHandleList
 0002:0000061C       _RMHandleToResourceHandleList16
 0003:0000028C       _RMModifyResources
 0002:00000252       _RMModifyResources16
 0002:00000228       _RMModifyResourcesOrg
 0001:00000050       _RM_Help0
 0001:00000054       _RM_Help1
 0001:00000058       _RM_Help3
 0005:00040BEC       _seq_client_load
 0005:00040C30       _seq_default_timer_card
 0005:00040C28       _seq_default_timer_class
 0005:00040C34       _seq_default_timer_device
 0005:00040C3C       _seq_default_timer_resolution
 0005:00040C2C       _seq_default_timer_sclass
 0005:00040C38       _seq_default_timer_subdevice
 0005:00000DA8       _snd_cards
 0003:000CE350       _snd_ctl_add_slave_
 0005:00000AA4       _snd_ecards_limit
 0005:00040797       _snd_hda_bind_sw
 0005:00040787       _snd_hda_bind_vol
 0005:00000AA8       _snd_major
 0005:00040FF0       _snd_opl3_regmap
 0005:00000AB8       _snd_oss_root
 0005:0000059C       _snd_pcm_devices_os2
 0005:0000F008       _snd_pcm_f_ops
 0003:0001BA42       _snd_pcm_hw_params_any_
 0003:0001BC10       _snd_pcm_hw_param_setempty_
 0003:000C8660       _snd_pcm_hw_param_set_
 0005:00075760       _snd_pcm_known_rates
 0005:0000EF44       _snd_pcm_link_rwlock
 0005:00000AB4       _snd_seq_root
 0005:00008210       _substream_int
 0005:000018F0       _system_utsname
 0005:00001BB2       _szLastALSAError1
 0005:00001C33       _szLastALSAError2
 0005:00001C32       _szOverrunTest1
 0005:00001CB3       _szOverrunTest2
 0005:00000040       _szprintBuf
 0005:00001F78       _szRecSources
 0005:00001AB2       _this_module
 0005:000017CC       _TimerHandler16
 0005:000017FC       _TKSSBase
 0005:00002154       _total
 0005:00000104       _ulget_free_pagesMemUsed
 0005:0000A218       _unlock_all
 0005:00040DBC       _use_internal_drums
 0005:0000003C       _wrOffset
 0005:0005FD38       __AccessFHeap
 0005:0005FD24       __AccessFileH
 0005:0005FD2C       __AccessIOB
 0005:0005FD34       __AccessNHeap
 0005:0005FD44       __AccessTDList
 0005:0005FDB0       __amblksiz
 0005:0005FD88       __ASTACKPTR
 0005:0005FD84       __ASTACKSIZ
 0003:000E0360       __Bits
 0005:0005FD8C       __cbyte
 0005:0005FD90       __cbyte2
 0003:00004235       __check_region_
 0005:0005FD94       __child
 0003:000E08C0       __CommonInit_
 0003:0000DE0C       __compat_get_order_
 0003:0000A669       __copy_user_
 0003:0000A719       __copy_user_zeroing_
 0005:0005FD60       __curbrk
 0000:00001234  Abs  __DOSseg__
 0005:0005FD5C       __dynend
 0005:0007AB82       __End_XI
 0005:0007AB82       __End_YI
 0003:000E0A00       __EnterWVIDEO_
 0005:0005FD9A       __Envptr
 0005:0005FD9E       __Envseg
 0003:000E0496       __exit_
 0003:000E0790       __exit_with_msg_
 0003:000E07E0       __fatal_runtime_error_
 0003:000E02F0       __FDFS
 0003:000E0860       __FiniRtns
 0003:00000000       __GETDS
 0003:0000A10F       __get_free_dma_pages_
 0003:0000A299       __get_free_pages_
 0003:0000A7BE       __get_user_
 0003:000DE0B5       __I8LS
 0003:000DE0D0       __I8M
 0003:000DE09A       __I8RS
 0003:000E0810       __InitRtns
 0003:0000A55D       __ioremap_
 0003:000DE620       __IsTable
 0003:0000A8D1       __kfree_
 0003:0000A866       __kmalloc_
 0005:0005FD64       __LpCmdLine
 0005:0005FD6C       __LpDllName
 0005:0005FD68       __LpPgmName
 0005:0005FD70       __LpwCmdLine
 0005:0005FD78       __LpwDllName
 0005:0005FD74       __LpwPgmName
 0003:000E0905       __mbinit_
 0005:0005FD98       __no87
 0005:0007ABD0       __nullarea
 0003:00000000       __OffBeginCS32
 0005:00000000       __OffBeginDS32
 0002:000006DB       __OffFinalCS16
 0003:000E0A28       __OffFinalCS32
 0001:0000048B       __OffFinalDS16
 0005:0007AB78       __OffFinalDS32
 0005:00001770       __OffsetFinalCS16
 0005:00001772       __OffsetFinalDS16
 0003:000E0479       __OS2Fini_
 0003:000E043B       __OS2Init_
 0003:000E03CC       __OS2MainInit_
 0005:0005FDA0       __osmajor
 0005:0005FDA1       __osminor
 0003:000DF5B0       __prtf_
 0005:0005FD40       __ReleaseFHeap
 0005:0005FD28       __ReleaseFileH
 0005:0005FD30       __ReleaseIOB
 0005:0005FD3C       __ReleaseNHeap
 0005:0005FD48       __ReleaseTDList
 0003:0000D56E       __release_region_
 0003:0000D45C       __request_region_
 0003:000DF340       __scnf_
 0003:000E02D1       __set_doserrno_
 0003:000E02A2       __set_EDOM_
 0003:000E02BE       __set_EINVAL_
 0003:000E02B0       __set_ERANGE_
 0003:000E0294       __set_errno_
 0003:000E0481       __shutdown_stack_checking_
 0003:000DDE31       __snd_util_memblk_new_
 0003:000DDD50       __snd_util_mem_alloc_
 0003:000DDF32       __snd_util_mem_free_
 0005:0005FD7C       __STACKLOW
 0005:0005FD80       __STACKTOP
 0005:0007AB7C       __Start_XI
 0005:0007AB82       __Start_YI
 0003:000DE730       __STOSB
 0003:000DE767       __STOSD
 0003:000E03C3       __threadid_
 0003:000E03BC       __threadstack_
 0005:0005FD54       __threadstksize
 0003:000DE0B5       __U8LS
 0003:000DE0D0       __U8M
 0003:000DE080       __U8RS
 0003:00003E1F       __udelay_
 0003:000101C5       __wake_up_
 0003:000034E6       __wcpp_2_pure_error__
 0003:000034B4       __wcpp_2_undefed_cdtor__
 0003:000034CD       __wcpp_2_undefined_member_function__
 0003:000034FF       __wcpp_2_undef_vfun__
 0003:0000354A       __wcpp_4_pure_error__
 0003:00003518       __wcpp_4_undefed_cdtor__
 0003:00003531       __wcpp_4_undefined_member_function__
 0003:00003563       __wcpp_4_undef_vfun__
 0005:00072908       ___Alphabet
 0004:00000003       ___begtext
 0005:0005FD14       ___EFG_printf
 0005:0005FD18       ___EFG_scanf
 0005:00060616       ___exitcall_alsa_ac97_exit
 0005:000527FC       ___exitcall_alsa_card_ali_exit
 0005:0000F714       ___exitcall_alsa_card_als4000_exit
 0005:00010920       ___exitcall_alsa_card_atiixp_exit
 0005:00040634       ___exitcall_alsa_card_azx_exit
 0005:0000F578       ___exitcall_alsa_card_bt87x_exit
 0005:00014318       ___exitcall_alsa_card_ca0106_exit
 0005:00010575       ___exitcall_alsa_card_cmipci_exit
 0005:00013990       ___exitcall_alsa_card_cs4281_exit
 0005:00041154       ___exitcall_alsa_card_cs46xx_exit
 0005:0004EE34       ___exitcall_alsa_card_cs5535audio_exit
 0005:0004F0A0       ___exitcall_alsa_card_emu10k1_exit
 0005:00013E2C       ___exitcall_alsa_card_ens137x_exit
 0005:000136BD       ___exitcall_alsa_card_es1938_exit
 0005:00012E24       ___exitcall_alsa_card_es1968_exit
 0005:00010DE0       ___exitcall_alsa_card_fm801_exit
 0005:00012B70       ___exitcall_alsa_card_intel8x0_exit
 0005:00011BDC       ___exitcall_alsa_card_m3_exit
 0005:0005F640       ___exitcall_alsa_card_nm256_exit
 0005:00052938       ___exitcall_alsa_card_trident_exit
 0005:00011498       ___exitcall_alsa_card_via82xx_exit
 0005:00051E3C       ___exitcall_alsa_card_ymfpci_exit
 0005:0000EA48       ___exitcall_alsa_hwdep_exit
 0005:00041038       ___exitcall_alsa_mpu401_uart_exit
 0005:00040E5C       ___exitcall_alsa_opl3_exit
 0005:00040DE8       ___exitcall_alsa_opl3_seq_exit
 0005:0000EE64       ___exitcall_alsa_pcm_exit
 0005:0005FC84       ___exitcall_alsa_pcm_oss_exit
 0005:0000EB84       ___exitcall_alsa_rawmidi_exit
 0005:0005FC04       ___exitcall_alsa_sb_common_exit
 0005:00040C6C       ___exitcall_alsa_seq_device_exit
 0005:00040C44       ___exitcall_alsa_seq_exit
 0005:00060740       ___exitcall_alsa_seq_midi_emul_exit
 0005:0000EEC0       ___exitcall_alsa_sound_exit
 0005:0000EAF4       ___exitcall_alsa_timer_exit
 0005:00060748       ___exitcall_alsa_util_mem_exit
 0005:0002275C       ___exitcall_patch_analog_exit
 0005:00018010       ___exitcall_patch_atihdmi_exit
 0005:00022EFC       ___exitcall_patch_cmedia_exit
 0005:00017EB4       ___exitcall_patch_conexant_exit
 0005:0003FFCD       ___exitcall_patch_realtek_exit
 0005:0001B176       ___exitcall_patch_sigmatel_exit
 0005:0001602C       ___exitcall_patch_via_exit
 0005:0000F118       ___exitcall_snd_mem_exit
 0005:0005FD1C       ___FirstThreadData
 0005:0005FDA2       ___FPE_handler
 0005:0005FD20       ___GetThreadPtr
 0005:00001734       ___hmodule
 0005:00060612       ___initcall_alsa_ac97_init
 0005:000527F8       ___initcall_alsa_card_ali_init
 0005:0000F710       ___initcall_alsa_card_als4000_init
 0005:0001091C       ___initcall_alsa_card_atiixp_init
 0005:00040630       ___initcall_alsa_card_azx_init
 0005:0000F574       ___initcall_alsa_card_bt87x_init
 0005:00014314       ___initcall_alsa_card_ca0106_init
 0005:00010571       ___initcall_alsa_card_cmipci_init
 0005:0001398C       ___initcall_alsa_card_cs4281_init
 0005:00041150       ___initcall_alsa_card_cs46xx_init
 0005:0004EE30       ___initcall_alsa_card_cs5535audio_init
 0005:0004F09C       ___initcall_alsa_card_emu10k1_init
 0005:00013E28       ___initcall_alsa_card_ens137x_init
 0005:000136B9       ___initcall_alsa_card_es1938_init
 0005:00012E20       ___initcall_alsa_card_es1968_init
 0005:00010DDC       ___initcall_alsa_card_fm801_init
 0005:00012B6C       ___initcall_alsa_card_intel8x0_init
 0005:00011BD8       ___initcall_alsa_card_m3_init
 0005:0005F63C       ___initcall_alsa_card_nm256_init
 0005:00052934       ___initcall_alsa_card_trident_init
 0005:00011494       ___initcall_alsa_card_via82xx_init
 0005:00051E38       ___initcall_alsa_card_ymfpci_init
 0005:0000EA44       ___initcall_alsa_hwdep_init
 0005:00041034       ___initcall_alsa_mpu401_uart_init
 0005:00040E58       ___initcall_alsa_opl3_init
 0005:00040DE4       ___initcall_alsa_opl3_seq_init
 0005:0000EE60       ___initcall_alsa_pcm_init
 0005:0005FC80       ___initcall_alsa_pcm_oss_init
 0005:0000EB80       ___initcall_alsa_rawmidi_init
 0005:0005FC00       ___initcall_alsa_sb_common_init
 0005:00040C68       ___initcall_alsa_seq_device_init
 0005:00040C40       ___initcall_alsa_seq_init
 0005:0006073C       ___initcall_alsa_seq_midi_emul_init
 0005:0000EEBC       ___initcall_alsa_sound_init
 0005:0000EAF0       ___initcall_alsa_timer_init
 0005:00060744       ___initcall_alsa_util_mem_init
 0005:00022758       ___initcall_patch_analog_init
 0005:0001800C       ___initcall_patch_atihdmi_init
 0005:00022EF8       ___initcall_patch_cmedia_init
 0005:00017EB0       ___initcall_patch_conexant_init
 0005:0003FFC9       ___initcall_patch_realtek_init
 0005:0001B172       ___initcall_patch_sigmatel_init
 0005:00016028       ___initcall_patch_via_init
 0005:0000F114       ___initcall_snd_mem_init
 0005:00001730       ___IsDBCS
 0005:00001524       ___Is_DLL
 0005:0005FDA8       ___MBCodePage
 0005:0000162C       ___MBCSIsTable
 0005:0005FD58       ___process_fini
 0005:00001528       ___saved_CS
 0005:0005FD50       ___sig_fini_rtn
 0005:0005FD4C       ___sig_init_rtn
 0005:0005FDAC       ___WD_Present


 Address         Publics by Value
 0000:00000000  Imp  DOSIODELAYCNT        (DOSCALLS.427)
 0000:00000000  Imp  DOSOPEN              (DOSCALLS.70)
 0000:00000000  Imp  _KernSISData         (KEE.90)
 0000:00000000  Imp  DosQueryCp           (DOSCALLS.291)
 0000:00000000  Imp  DosQueryDBCSEnv      (NLS.6)
 0000:00000000  Imp  KernVMAlloc          (KEE.60)
 0000:00000000  Imp  DOS32FLATDS          (DOSCALLS.370)
 0000:00000000  Imp  KernThunkStackTo32   (KEE.41)
 0000:00000000  Imp  DosQuerySysInfo      (DOSCALLS.348)
 0000:00000000  Imp  DOSWRITE             (DOSCALLS.138)
 0000:00000000  Imp  DosWrite             (DOSCALLS.282)
 0000:00000000  Imp  DOSCLOSE             (DOSCALLS.59)
 0000:00000000  Imp  KernThunkStackTo16   (KEE.40)
 0000:00000000  Imp  KernLinToPageList    (KEE.64)
 0000:00000000  Imp  KernVMLock           (KEE.62)
 0000:00000000  Imp  KernSelToFlat        (KEE.66)
 0000:00000000  Imp  DosExit              (DOSCALLS.234)
 0000:00000000  Imp  KernVMFree           (KEE.61)
 0000:00001234  Abs  __DOSseg__
 0001:00000000       help_header
 0001:0000001E       uniaud_header
 0001:0000003C       DevHelpInit
 0001:00000040       fOpen
 0001:00000044       InitPktSeg
 0001:00000046       InitPktOff
 0001:00000048       DbgU32TimerCnt
 0001:0000004C       DbgU32IntCnt
 0001:00000050       _RM_Help0
 0001:00000054       _RM_Help1
 0001:00000058       _RM_Help3
 0001:0000005C       _RMFlags
 0001:00000060       _MESSAGE_STR
 0001:00000460       _MSG_TABLE16
 0001:00000466       pddname16
 0001:0000046D       FileName
 0001:0000048B       __OffFinalDS16
 0002:00000000       help_stub_strategy
 0002:00000096       uniaud_stub_strategy
 0002:0000010A       uniaud_stub_idc
 0002:00000128       uniaud_stub_timer
 0002:000001A0       thunk3216_devhelp
 0002:000001B2       thunk3216_devhelp_modified_ds
 0002:000001C8       _RMAllocResourceOrg
 0002:00000204       _RMAllocResource16
 0002:00000228       _RMModifyResourcesOrg
 0002:00000252       _RMModifyResources16
 0002:0000027A       _RMCreateAdapterOrg
 0002:000002B6       _RMCreateAdapter16
 0002:000002E2       _RMCreateDeviceOrg
 0002:0000031E       _RMCreateDevice16
 0002:0000034A       _RMDestroyDeviceOrg
 0002:00000374       _RMDestroyDevice16
 0002:00000390       _RMDeallocResourceOrg
 0002:000003BA       _RMDeallocResource16
 0002:000003DA       MY_DEVHELP_ATTACHDD
 0002:00000400       _RMCreateDriverOrg
 0002:0000047A       _RMCreateDriver16
 0002:0000049A       _CallRM
 0002:000004CE       _RMDestroyDriverOrg
 0002:000004F8       _RMDestroyDriver16
 0002:0000054C       _RMGetNodeInfo16
 0002:000005A8       _RMDevIDToHandleList16
 0002:0000061C       _RMHandleToResourceHandleList16
 0002:000006DB       __OffFinalCS16
 0003:00000000       __OffBeginCS32
 0003:00000000       __GETDS
 0003:00000010       DevHlp
 0003:00000024       thunk1632_devhelp
 0003:00000030       DevHlp_ModifiedDS
 0003:00000044       thunk1632_devhelp_modified_ds
 0003:00000050       _CallPDD16
 0003:00000080       STRATEGY_
 0003:000000E0       IDC_
 0003:00000140       TIMER_
 0003:0000024C       _RMAllocResource
 0003:0000028C       _RMModifyResources
 0003:000002D0       _RMDeallocResource
 0003:00000310       _RMCreateDevice
 0003:00000358       _RMCreateAdapter
 0003:000003A0       _RMCreateDriver
 0003:000003E0       _RMDestroyDriver
 0003:0000040C       _RMGetNodeInfo
 0003:0000044C       _RMDevIDToHandleList
 0003:000004A0       _RMHandleToResourceHandleList
 0003:000004DD       W?StratOpen$n(pf$RP$$)ul
 0003:00000544       W?StratInit$n(pf$RP$$)ul
 0003:000005AE       W?StratInitComplete$n(pf$RP$$)ul
 0003:000005E9       W?StratShutdown$n(pf$RP$$)ul
 0003:00000656       ALSA_STRATEGY
 0003:000006D8       W?StratRead$n(pf$RP$$)ul
 0003:0000084E       W?DevSaveMessage$n(pfai)v
 0003:0000090D       W?LockSegments$n()i
 0003:00000A0D       W?DiscardableInit$n(pf$RPInit$$)ul
 0003:00000E1D       W?toupper$n(i)i
 0003:00000E5D       W?mymemchr$n(pfaaus)pfa
 0003:00000EDC       W?sz2us$n(pfai)us
 0003:00000FC7       W?IsWhitespace$n(a)i
 0003:00001018       W?SkipWhite$n(pfa)pfa
 0003:00001096       W?CheckCardName$n(pfa)v
 0003:00001313       W?DoParm$n(apfa)i
 0003:0000140E       W?ParseParm$n(pfai)i
 0003:00001513       GetParms_
 0003:00001624       GetTKSSBase
 0003:00001664       iodelay32_
 0003:00001672       ALSA_IDC
 0003:000016FC       W?OSS32IDC$n(ulpn$__6ikc0pIDC32_PACKET$$)ul
 0003:00001CB3       W?StratIOCtl$n(pf$RP$$)ul
 0003:0000288A       W?StratClose$n(pf$RP$$)ul
 0003:000028EC       RMInit_
 0003:00002A9B       RMRequestIO_
 0003:00002B8B       RMRequestMem_
 0003:00002C6E       RMRequestIRQ_
 0003:00002DB4       RMDeallocateIRQ_
 0003:00002E2D       RMDone_
 0003:000032FA       RMSetHandles_
 0003:00003326       ALSA_SetIrq_
 0003:00003409       ALSA_FreeIrq_
 0003:00003451       ALSA_Interrupt
 0003:000034B4       __wcpp_2_undefed_cdtor__
 0003:000034CD       __wcpp_2_undefined_member_function__
 0003:000034E6       __wcpp_2_pure_error__
 0003:000034FF       __wcpp_2_undef_vfun__
 0003:00003518       __wcpp_4_undefed_cdtor__
 0003:00003531       __wcpp_4_undefined_member_function__
 0003:0000354A       __wcpp_4_pure_error__
 0003:00003563       __wcpp_4_undef_vfun__
 0003:0000357C       W?$nwn(ui)pnv
 0003:000035A5       W?$dln(pnv)v
 0003:000035C8       W?$nwn(uipnv)pnv
 0003:00003602       os2gettimesec_
 0003:00003625       os2gettimemsec_
 0003:00003947       vsprintf_
 0003:00003D2D       sprintf_
 0003:00003D6C       ALSA_TIMER_
 0003:00003DCA       schedule_timeout_
 0003:00003E1F       __udelay_
 0003:00003E51       mdelay_
 0003:00003E85       do_gettimeofday_
 0003:00003ED1       add_timer_
 0003:00003EEC       del_timer_
 0003:00003F11       mod_timer_
 0003:00003F2D       msleep_
 0003:00003F70       strcmp_
 0003:00003FCD       strncmp_
 0003:0000403C       tasklet_hi_schedule_
 0003:00004074       tasklet_init_
 0003:000040B6       OSS32_SetFileId_
 0003:00004177       _printk
 0003:00004200       schedule_
 0003:00004218       poll_wait_
 0003:00004235       __check_region_
 0003:0000425C       hweight32_
 0003:000042F6       create_proc_entry_
 0003:00004356       remove_proc_entry_
 0003:00004372       proc_register_
 0003:00004398       proc_unregister_
 0003:000043BE       fasync_helper_
 0003:000043E6       kill_fasync_
 0003:00004403       request_dma_
 0003:00004429       free_dma_
 0003:00004444       enable_dma_
 0003:0000445F       disable_dma_
 0003:0000447A       register_reboot_notifier_
 0003:0000449F       unregister_reboot_notifier_
 0003:0000453B       queue_work_
 0003:00004650       flush_workqueue_
 0003:000046BD       create_workqueue_
 0003:00004747       destroy_workqueue_
 0003:0000476A       kstrdup_
 0003:000047DC       mod_firmware_load_
 0003:00004882       request_firmware_
 0003:0000492C       release_firmware_
 0003:00004960       memdup_user_
 0003:000049DF       W?CallOSS16$n(ululul)ul
 0003:00004A47       OSS32_Initialize_
 0003:00004D0C       OSS32_Shutdown_
 0003:00004DA9       OSS32_ProcessIRQ_
 0003:00004DD5       OSS32_ProcessMIDIIRQ_
 0003:00004E05       OSS32_CloseUNI16_
 0003:00004E31       MyDevBlock_
 0003:00004E83       OSS32_DebugString_
 0003:00004EBA       OSS32_MidiOpen_
 0003:00005371       OSS32_MidiClose_
 0003:00005519       OSS32_MidiWrite_
 0003:00005551       OSS32_MidiRead_
 0003:00005605       OSS32_MidiQueryCaps_
 0003:0000563D       OSS32_MidiCommand_
 0003:00005820       ConvertVolume_
 0003:0000586D       OSS32_MixOpen_
 0003:00005F55       OSS32_MixClose_
 0003:00005FE5       OSS32_MixGetVolume_
 0003:00006036       OSS32_MixSetVolume_
 0003:00006521       OSS32_MixSetProperty_
 0003:000069C7       OSS32_MixGetProperty_
 0003:00006A18       OSSToALSAVolume_
 0003:00006B97       OSS32_MixQueryCaps_
 0003:00006C7D       OSS32_MixQueryName_
 0003:00006DDB       OSS32_QueryNames_
 0003:00006FD1       register_chrdev_
 0003:00007011       unregister_chrdev_
 0003:00007052       register_sound_special_
 0003:000070A4       register_sound_mixer_
 0003:000070F6       register_sound_midi_
 0003:00007148       register_sound_dsp_
 0003:0000719A       register_sound_synth_
 0003:000071EC       unregister_sound_special_
 0003:00007218       unregister_sound_mixer_
 0003:00007244       unregister_sound_midi_
 0003:00007270       unregister_sound_dsp_
 0003:0000729C       unregister_sound_synth_
 0003:000072C8       UNIXToOSSError_
 0003:00007445       ALSAToOSSDataType_
 0003:0000753A       ALSAToOSSRateFlags_
 0003:00007629       OSS32_QueryDevCaps_
 0003:00007BD1       OSS32_WaveOpen_
 0003:00007EAE       OSS32_WaveClose_
 0003:00008035       OSS32_WavePrepare_
 0003:000080DF       OSS32_WaveStart_
 0003:0000816D       OSS32_WaveStop_
 0003:000081FB       OSS32_WavePause_
 0003:00008289       OSS32_WaveResume_
 0003:0000831A       OSS32_WaveSetHwParams_
 0003:00008F7D       OSS32_WaveAddBuffer_
 0003:0000928C       OSS32_WaveGetPosition_
 0003:0000936D       OSS32_WaveGetSpace_
 0003:0000941B       OSS32_WaveGetHwPtr_
 0003:000094C1       OSS32_WaveGetStatus_
 0003:00009561       OSS32_WaveSetVolume_
 0003:00009625       DecLongToASCII_
 0003:00009792       HexLongToASCII_
 0003:00009907       CharOut_
 0003:0000994D       StringOut_
 0003:00009AD5       snd_iprintf_
 0003:00009DE1       DbgPrintIrq_
 0003:00009E2B       AddBaseAddress_
 0003:00009E8F       GetBaseAddress_
 0003:00009F65       virt_to_phys_
 0003:00009FAF       phys_to_virt_
 0003:0000A00E       VMAlloc_
 0003:0000A0D8       VMFree_
 0003:0000A10F       __get_free_dma_pages_
 0003:0000A299       __get_free_pages_
 0003:0000A401       free_pages_
 0003:0000A453       vmalloc_
 0003:0000A4CB       vfree_
 0003:0000A50F       alloc_pages_
 0003:0000A535       remap_page_range_
 0003:0000A55D       __ioremap_
 0003:0000A610       iounmap_
 0003:0000A642       is_access_ok_
 0003:0000A669       __copy_user_
 0003:0000A6B5       copy_to_user_
 0003:0000A719       __copy_user_zeroing_
 0003:0000A75A       copy_from_user_
 0003:0000A7BE       __get_user_
 0003:0000A822       _put_user_
 0003:0000A866       __kmalloc_
 0003:0000A8D1       __kfree_
 0003:0000A918       kzalloc_
 0003:0000A95E       kcalloc_
 0003:0000A9B0       uniaud_set_interrupted_substream_
 0003:0000AA16       WaitForControlChange_
 0003:0000AAAF       WaitForPCMInterrupt_
 0003:0000AC1B       GetNumberOfCards_
 0003:0000AC3E       GetNumberOfPcm_
 0003:0000AC67       SetPCMInstance_
 0003:0000ACB3       GetPcmForChannels_
 0003:0000AD95       GetMaxChannels_
 0003:0000AE7E       GetUniaudPcmCaps1_
 0003:0000B3C0       FillCaps_
 0003:0000B456       GetUniaudPcmCaps_
 0003:0000B4CC       UniaudCtlGetPowerState_
 0003:0000B5E8       UniaudCtlSetPowerState_
 0003:0000B704       GetUniaudCardInfo_
 0003:0000B850       GetUniaudControlNum_
 0003:0000BA45       GetUniaudControls_
 0003:0000BCB6       GetUniaudControlInfo_
 0003:0000BE27       GetUniaudControlValueGet_
 0003:0000BF98       GetUniaudControlValuePut_
 0003:0000C109       UniaudIoctlHWRefine_
 0003:0000C189       UniaudIoctlHWParamSet_
 0003:0000C209       UniaudIoctlSWParamSet_
 0003:0000C289       UniaudIoctlPCMStatus_
 0003:0000C302       UniaudIoctlPCMWrite_
 0003:0000C374       UniaudIoctlPCMRead_
 0003:0000C3E6       UniaudIoctlPCMPrepare_
 0003:0000C448       UniaudIoctlPCMResume_
 0003:0000C4AC       UniaudIoctlPCMStart_
 0003:0000C50E       UniaudIoctlPCMDrop_
 0003:0000C570       UniaudCloseAll_
 0003:0000C686       request_irq_
 0003:0000C85F       free_irq_
 0003:0000C96A       eoi_irq_
 0003:0000C996       process_interrupt_
 0003:0000CAEF       in_interrupt_
 0003:0000CB12       disable_irq_
 0003:0000CB3F       pci_read_config_byte_
 0003:0000CBAB       pci_read_config_word_
 0003:0000CC19       pci_read_config_dword_
 0003:0000CC7E       pci_write_config_byte_
 0003:0000CCE6       pci_write_config_word_
 0003:0000CD4F       pci_write_config_dword_
 0003:0000CDAF       pcidev_prepare_
 0003:0000CDE6       pcidev_activate_
 0003:0000CE1D       pcidev_deactivate_
 0003:0000D355       pci_find_device_
 0003:0000D45C       __request_region_
 0003:0000D56E       __release_region_
 0003:0000D5E5       pci_get_flags_
 0003:0000D633       pcibios_present_
 0003:0000D663       pci_find_slot_
 0003:0000D69F       pci_dma_supported_
 0003:0000D6D3       pci_find_capability_
 0003:0000D78B       pci_set_power_state_
 0003:0000D958       pci_enable_device_
 0003:0000D9C0       pci_register_driver_
 0003:0000DBBC       pci_module_init_
 0003:0000DBFA       pci_unregister_driver_
 0003:0000DD52       pci_set_master_
 0003:0000DDAE       pm_register_
 0003:0000DDE3       pm_unregister_
 0003:0000DE0C       __compat_get_order_
 0003:0000DE50       pci_alloc_consistent_
 0003:0000DF7E       pci_free_consistent_
 0003:0000DFB0       pci_set_driver_data_
 0003:0000DFDE       pci_get_driver_data_
 0003:0000E017       pci_get_dma_mask_
 0003:0000E050       release_resource_
 0003:0000E075       pci_set_latency_time_
 0003:0000E0AD       pci_orig_save_state_
 0003:0000E105       pci_orig_restore_state_
 0003:0000E1AC       pci_save_state_
 0003:0000E22D       pci_restore_state_
 0003:0000E2B1       pci_disable_device_
 0003:0000E2FB       pci_request_region_
 0003:0000ED57       pci_release_region_
 0003:0000F1E8       pci_request_regions_
 0003:0000F257       pci_release_regions_
 0003:0000F292       pci_match_device_
 0003:0000F390       snd_pci_dev_present_
 0003:0000F447       snd_pci_compat_get_pci_driver_
 0003:0000F488       OSS32_APMResume_
 0003:0000F535       OSS32_APMSuspend_
 0003:0000F5F5       PciAdjustInterrupts_
 0003:0000F764       W?dumpheap$n()v
 0003:0000F8A7       W?SignatureCheck$n(pn$_MEMBLOCK$$pna)s
 0003:0000F951       W?HeapCheck$n(pna)v
 0003:0000FA69       W?npvAllocateBlock$n(pn$_MEMBLOCK$$ulpn$1$)pnv
 0003:0000FB5C       W?malloc$n(ul)pnv
 0003:0000FC53       W?remove$n(pn$_MEMBLOCK$$)v
 0003:0000FCBC       W?compact$n()v
 0003:0000FD84       W?free$n(pnv)v
 0003:0000FE86       W?_memfree$n()ui
 0003:0000FEA9       W?_msize$n(pnv)ui
 0003:0000FEE8       W?realloc$n(pnvul)pnv
 0003:0000FF95       W?IsHeapAddr$n(ul)ul
 0003:0000FFEB       W?HeapInit$n(ul)ul
 0003:00010093       strncpy_
 0003:000100FA       init_waitqueue_head_
 0003:00010115       add_wait_queue_
 0003:00010131       add_wait_queue_exclusive_
 0003:0001014C       remove_wait_queue_
 0003:00010168       interruptible_sleep_on_timeout_
 0003:0001019C       interruptible_sleep_on_
 0003:000101C5       __wake_up_
 0003:000101F8       init_waitqueue_entry_
 0003:00010214       waitqueue_active_
 0003:00010239       spin_lock_init_
 0003:0001025D       spin_lock_
 0003:00010282       spin_lock_flag_
 0003:000102A8       spin_trylock_
 0003:000102CD       spin_unlock_
 0003:00010D85       snd_hwdep_new_
 0003:000118A4       snd_timer_open_
 0003:00011B24       snd_timer_close_
 0003:00011DB7       snd_timer_resolution_
 0003:000120C7       snd_timer_start_
 0003:000122FB       snd_timer_stop_
 0003:0001237B       snd_timer_continue_
 0003:00012445       snd_timer_pause_
 0003:00012646       snd_timer_interrupt_
 0003:00012ADD       snd_timer_new_
 0003:00013033       snd_timer_notify_
 0003:00013172       snd_timer_global_new_
 0003:000131C7       snd_timer_global_free_
 0003:000131F0       snd_timer_global_register_
 0003:00015776       snd_rawmidi_drop_output_
 0003:000157EF       snd_rawmidi_drain_output_
 0003:000158C3       snd_rawmidi_drain_input_
 0003:00015C0E       snd_rawmidi_kernel_open_
 0003:0001620D       snd_rawmidi_kernel_release_
 0003:00016410       snd_rawmidi_info_select_
 0003:000165D5       snd_rawmidi_output_params_
 0003:00016720       snd_rawmidi_input_params_
 0003:0001692B       snd_rawmidi_receive_
 0003:00016CE3       snd_rawmidi_kernel_read_
 0003:00016F0D       snd_rawmidi_transmit_empty_
 0003:00016F97       snd_rawmidi_transmit_peek_
 0003:000170FE       snd_rawmidi_transmit_ack_
 0003:000171FF       snd_rawmidi_transmit_
 0003:00017467       snd_rawmidi_kernel_write_
 0003:00017AD4       snd_rawmidi_new_
 0003:00018301       snd_rawmidi_set_ops_
 0003:0001845E       snd_pcm_format_signed_
 0003:000184B6       snd_pcm_format_unsigned_
 0003:00018509       snd_pcm_format_linear_
 0003:00018549       snd_pcm_format_little_endian_
 0003:000185A1       snd_pcm_format_big_endian_
 0003:000185F4       snd_pcm_format_width_
 0003:0001864B       snd_pcm_format_physical_width_
 0003:000186A2       snd_pcm_format_size_
 0003:000186E8       snd_pcm_format_silence_64_
 0003:00018742       snd_pcm_format_set_silence_
 0003:00018902       snd_pcm_limit_hw_rates_
 0003:000189B7       snd_pcm_rate_to_rate_bit_
 0003:00019330       snd_pcm_playback_silence_
 0003:00019BCD       snd_pcm_update_hw_ptr_
 0003:00019D57       snd_pcm_set_ops_
 0003:00019DA9       snd_pcm_set_sync_
 0003:00019FCF       snd_interval_refine_
 0003:0001A2AE       snd_interval_mul_
 0003:0001A40A       snd_interval_div_
 0003:0001A55F       snd_interval_muldivk_
 0003:0001A69C       snd_interval_mulkdiv_
 0003:0001A7F8       snd_interval_ratnum_
 0003:0001AEAA       snd_interval_list_
 0003:0001B05D       snd_pcm_hw_rule_add_
 0003:0001B1D5       snd_pcm_hw_constraint_mask_
 0003:0001B252       snd_pcm_hw_constraint_mask64_
 0003:0001B2F7       snd_pcm_hw_constraint_integer_
 0003:0001B34F       snd_pcm_hw_constraint_minmax_
 0003:0001B45A       snd_pcm_hw_constraint_list_
 0003:0001B564       snd_pcm_hw_constraint_ratnums_
 0003:0001B66E       snd_pcm_hw_constraint_ratdens_
 0003:0001B753       snd_pcm_hw_constraint_msbits_
 0003:0001B811       snd_pcm_hw_constraint_step_
 0003:0001B8C8       snd_pcm_hw_constraint_pow2_
 0003:0001BA42       _snd_pcm_hw_params_any_
 0003:0001BAB9       snd_pcm_hw_param_value_
 0003:0001BC10       _snd_pcm_hw_param_setempty_
 0003:0001BE66       snd_pcm_hw_param_first_
 0003:0001C004       snd_pcm_hw_param_last_
 0003:0001C089       snd_pcm_hw_params_choose_
 0003:0001C381       snd_pcm_lib_ioctl_
 0003:0001C403       snd_pcm_period_elapsed_
 0003:0001CB8D       snd_pcm_lib_write_
 0003:0001CE50       snd_pcm_lib_writev_
 0003:0001D32C       snd_pcm_lib_read_
 0003:0001D585       snd_pcm_lib_readv_
 0003:0001DAF0       snd_pcm_new_stream_
 0003:0001DD65       snd_pcm_new_
 0003:0001E036       snd_pcm_attach_substream_
 0003:0001E451       snd_pcm_detach_substream_
 0003:0001E87C       snd_pcm_notify_
 0003:0001EB01       pcm_info_
 0003:0001EBE6       pcm_instances_
 0003:0001ECBC       snd_lookup_minor_data_
 0003:0001EF3C       snd_register_device_for_dev_
 0003:0001F0FC       snd_unregister_device_
 0003:0001F182       snd_add_device_sysfs_file_
 0003:0001F337       snd_minor_info_init_
 0003:0001F3A0       snd_minor_info_done_
 0003:0001F51B       snd_info_check_reserved_words_
 0003:00020149       snd_info_init_
 0003:00020255       snd_info_done_
 0003:000202D7       snd_info_card_create_
 0003:0002038B       snd_info_card_register_
 0003:000203F1       snd_info_card_id_change_
 0003:00020461       snd_info_card_disconnect_
 0003:000204F3       snd_info_card_free_
 0003:00020542       snd_info_get_line_
 0003:0002064C       snd_info_get_str_
 0003:0002080F       snd_info_create_module_entry_
 0003:00020858       snd_info_create_card_entry_
 0003:000209E0       snd_card_proc_new_
 0003:00020A69       snd_info_free_entry_
 0003:00020AD5       snd_info_register_
 0003:00020E33       snd_pcm_lib_preallocate_free_
 0003:00020E60       snd_pcm_lib_preallocate_free_for_all_
 0003:00020F41       snd_pcm_lib_preallocate_pages_
 0003:00020F87       snd_pcm_lib_preallocate_pages_for_all_
 0003:0002100D       snd_pcm_sgbuf_ops_page_
 0003:0002106E       snd_pcm_sgbuf_get_chunk_size_
 0003:00021112       snd_pcm_lib_malloc_pages_
 0003:00021257       snd_pcm_lib_free_pages_
 0003:0002134D       snd_pcm_timer_resolution_change_
 0003:00021564       snd_pcm_timer_init_
 0003:0002167F       snd_pcm_timer_done_
 0003:00021D76       snd_pcm_info_
 0003:00021EB1       snd_pcm_info_user_
 0003:00021F2E       snd_pcm_hw_refine_
 0003:00022FBF       snd_pcm_status_
 0003:00023A31       snd_pcm_start_
 0003:00023B7D       snd_pcm_stop_
 0003:00023BAF       snd_pcm_drain_done_
 0003:00023F0A       snd_pcm_suspend_
 0003:00023F80       snd_pcm_suspend_all_
 0003:0002577C       snd_pcm_hw_constraints_init_
 0003:00025D1E       snd_pcm_hw_constraints_complete_
 0003:00025FE6       snd_pcm_release_substream_
 0003:00026087       snd_pcm_open_substream_
 0003:00027A7C       snd_pcm_kernel_ioctl_
 0003:00028056       dummy_get_unmapped_area_
 0003:00028080       snd_oss_info_register_
 0003:00028319       snd_info_minor_register_
 0003:00028397       snd_info_minor_unregister_
 0003:000283CD       snd_lookup_oss_minor_data_
 0003:000285DD       snd_register_oss_device_
 0003:0002875C       snd_unregister_oss_device_
 0003:000289CC       snd_minor_info_oss_init_
 0003:00028A39       snd_minor_info_oss_done_
 0003:00028AA4       snd_device_new_
 0003:00028B71       snd_device_free_
 0003:00028C9C       snd_device_disconnect_
 0003:00028D6F       snd_device_register_
 0003:00028E4B       snd_device_register_all_
 0003:00028EF2       snd_device_disconnect_all_
 0003:00028F77       snd_device_free_all_
 0003:000294FF       snd_ctl_notify_
 0003:0002970E       snd_ctl_new1_
 0003:00029878       snd_ctl_free_one_
 0003:00029A08       snd_ctl_add_
 0003:00029B9B       snd_ctl_remove_
 0003:00029C67       snd_ctl_remove_id_
 0003:00029DB8       snd_ctl_rename_id_
 0003:00029E52       snd_ctl_find_numid_
 0003:00029EDF       snd_ctl_find_id_
 0003:0002BA91       snd_ctl_register_ioctl_
 0003:0002BB82       snd_ctl_unregister_ioctl_
 0003:0002BE73       snd_ctl_create_
 0003:0002BEC7       snd_ctl_boolean_mono_info_
 0003:0002BF15       snd_ctl_boolean_stereo_info_
 0003:0002BFE6       snd_malloc_pages_
 0003:0002C052       snd_free_pages_
 0003:0002C0A2       snd_malloc_dev_pages_
 0003:0002C117       snd_free_dev_pages_
 0003:0002C17A       snd_dma_alloc_pages_
 0003:0002C28B       snd_dma_alloc_pages_fallback_
 0003:0002C328       snd_dma_free_pages_
 0003:0002C3AE       snd_dma_get_reserved_buf_
 0003:0002C4D3       snd_dma_reserve_buf_
 0003:0002C7EE       snd_card_create_
 0003:0002CB61       snd_card_locked_
 0003:0002CDAB       snd_card_disconnect_
 0003:0002D013       snd_card_free_when_closed_
 0003:0002D0D1       snd_card_free_
 0003:0002D3CE       snd_card_set_id_
 0003:0002D414       snd_card_register_
 0003:0002D5B6       snd_card_info_read_oss_
 0003:0002D6A6       snd_card_info_init_
 0003:0002D75F       snd_card_info_done_
 0003:0002D795       snd_component_add_
 0003:0002D899       snd_card_file_add_
 0003:0002D969       snd_card_file_remove_
 0003:0002DAC4       snd_power_wait_
 0003:0002DC18       snd_free_sgbuf_pages_
 0003:0002DC94       snd_malloc_sgbuf_pages_
 0003:0005360E       ioread8_
 0003:0005365A       ioread16_
 0003:000536A8       ioread32_
 0003:000536ED       iowrite8_
 0003:00053730       iowrite16_
 0003:00053775       iowrite32_
 0003:000537B8       ioport_map_
 0003:000537F4       ioport_unmap_
 0003:0005380F       pci_iomap_
 0003:00053A3F       pci_iounmap_
 0003:00053AB5       snd_ca0106_ptr_read_
 0003:00053B1B       snd_ca0106_ptr_write_
 0003:00053B79       snd_ca0106_spi_write_
 0003:00053C96       snd_ca0106_i2c_write_
 0003:00056B6C       ca_midi_init_
 0003:00057EA1       snd_ca0106_mixer_
 0003:00058137       snd_ca0106_mixer_suspend_
 0003:00058196       snd_ca0106_mixer_resume_
 0003:00058E4C       snd_ca0106_proc_init_
 0003:0007BA46       snd_hda_add_codec_preset_
 0003:0007BAA7       snd_hda_delete_codec_preset_
 0003:0007BB11       snd_hda_get_jack_location_
 0003:0007BB9C       snd_hda_get_jack_connectivity_
 0003:0007BBCF       snd_hda_get_jack_type_
 0003:0007BDC2       snd_hda_codec_read_
 0003:0007BE14       snd_hda_codec_write_
 0003:0007BE80       snd_hda_sequence_write_
 0003:0007BECC       snd_hda_get_sub_nodes_
 0003:0007BF33       snd_hda_get_connections_
 0003:0007C23B       snd_hda_queue_unsol_event_
 0003:0007C44B       snd_hda_bus_new_
 0003:0007CBD4       snd_hda_add_pincfg_
 0003:0007CC7D       snd_hda_codec_set_pincfg_
 0003:0007CCBA       snd_hda_codec_get_pincfg_
 0003:0007CF47       snd_hda_codec_new_
 0003:0007D3C0       snd_hda_codec_configure_
 0003:0007D4FE       snd_hda_codec_setup_stream_
 0003:0007D58A       snd_hda_codec_cleanup_stream_
 0003:0007D777       query_amp_caps_
 0003:0007D853       snd_hda_override_amp_caps_
 0003:0007D98C       snd_hda_query_pin_caps_
 0003:0007DB40       snd_hda_codec_amp_read_
 0003:0007DBCF       snd_hda_codec_amp_update_
 0003:0007DCB1       snd_hda_codec_amp_stereo_
 0003:0007DD19       snd_hda_codec_resume_amp_
 0003:0007DDFF       snd_hda_mixer_amp_volume_info_
 0003:0007DFAB       snd_hda_mixer_amp_volume_get_
 0003:0007E086       snd_hda_mixer_amp_volume_put_
 0003:0007E178       snd_hda_mixer_amp_tlv_
 0003:0007E2AF       snd_hda_set_vmaster_tlv_
 0003:0007E3C0       snd_hda_find_mixer_ctl_
 0003:0007E3EF       snd_hda_ctl_add_
 0003:0007E45A       snd_hda_ctls_clear_
 0003:0007E56D       snd_hda_codec_reset_
 0003:0007E7D8       snd_hda_add_vmaster_
 0003:0007E934       snd_hda_mixer_amp_switch_info_
 0003:0007E9A6       snd_hda_mixer_amp_switch_get_
 0003:0007EA94       snd_hda_mixer_amp_switch_put_
 0003:0007EBA5       snd_hda_mixer_bind_switch_get_
 0003:0007EC1B       snd_hda_mixer_bind_switch_put_
 0003:0007ECEF       snd_hda_mixer_bind_ctls_info_
 0003:0007ED65       snd_hda_mixer_bind_ctls_get_
 0003:0007EDDC       snd_hda_mixer_bind_ctls_put_
 0003:0007EE9C       snd_hda_mixer_bind_tlv_
 0003:0007F490       snd_hda_create_spdif_out_ctls_
 0003:0007F64F       snd_hda_create_spdif_share_sw_
 0003:0007F83F       snd_hda_create_spdif_in_ctls_
 0003:0007F933       snd_hda_codec_write_cache_
 0003:0007F9E4       snd_hda_codec_resume_cache_
 0003:0007FA6C       snd_hda_sequence_write_cache_
 0003:0007FD6D       snd_hda_build_controls_
 0003:0007FE0C       snd_hda_codec_build_controls_
 0003:0007FE80       snd_hda_calc_stream_format_
 0003:00080413       snd_hda_is_supported_format_
 0003:00080999       snd_hda_codec_build_pcms_
 0003:00080ACF       snd_hda_build_pcms_
 0003:00080B37       snd_hda_check_board_config_
 0003:00080CC6       snd_hda_check_board_codec_sid_config_
 0003:00080DF9       snd_hda_add_new_ctls_
 0003:00080EC2       snd_hda_ch_mode_info_
 0003:00080F3F       snd_hda_ch_mode_get_
 0003:00080F9B       snd_hda_ch_mode_put_
 0003:0008102D       snd_hda_input_mux_info_
 0003:000810CB       snd_hda_input_mux_put_
 0003:000812BA       snd_hda_multi_out_dig_open_
 0003:0008131E       snd_hda_multi_out_dig_prepare_
 0003:00081379       snd_hda_multi_out_dig_cleanup_
 0003:000813CA       snd_hda_multi_out_dig_close_
 0003:00081414       snd_hda_multi_out_analog_open_
 0003:000815C5       snd_hda_multi_out_analog_prepare_
 0003:000817C4       snd_hda_multi_out_analog_cleanup_
 0003:000819EA       snd_hda_parse_pin_def_config_
 0003:00082252       snd_hda_suspend_
 0003:000822A9       snd_hda_resume_
 0003:00082300       snd_array_new_
 0003:0008240A       snd_array_free_
 0003:0008244D       snd_print_pcm_rates_
 0003:000824C9       snd_print_pcm_bits_
 0003:0008283B       snd_hda_create_hwdep_
 0003:0008482A       snd_hda_parse_generic_codec_
 0003:000860AC       snd_hda_codec_proc_new_
 0003:00086308       snd_seq_device_load_drivers_
 0003:00086320       snd_seq_device_new_
 0003:0008667B       snd_seq_device_register_driver_
 0003:00086868       snd_seq_device_unregister_driver_
 0003:00086DFD       snd_seq_info_init_
 0003:00086E5B       snd_seq_info_done_
 0003:00086F1B       snd_seq_system_broadcast_
 0003:00086F63       snd_seq_system_notify_
 0003:00086FFA       snd_seq_system_client_init_
 0003:00087170       snd_seq_system_client_done_
 0003:00087284       snd_seq_queue_get_cur_queues_
 0003:00087556       snd_seq_queues_init_
 0003:00087578       snd_seq_queues_delete_
 0003:000875C5       snd_seq_queue_alloc_
 0003:00087642       snd_seq_queue_delete_
 0003:000876A2       queueptr_
 0003:00087705       snd_seq_queue_find_name_
 0003:0008776F       snd_seq_check_queue_
 0003:000878F8       snd_seq_enqueue_event_
 0003:00087AF7       snd_seq_queue_check_access_
 0003:00087B5D       snd_seq_queue_set_owner_
 0003:00087C03       snd_seq_queue_timer_open_
 0003:00087C75       snd_seq_queue_timer_close_
 0003:00087CCB       snd_seq_queue_timer_set_tempo_
 0003:00087D87       snd_seq_queue_use_
 0003:00087E68       snd_seq_queue_is_used_
 0003:00087EDD       snd_seq_queue_client_termination_
 0003:00087F7B       snd_seq_queue_client_leave_
 0003:0008803E       snd_seq_queue_client_leave_cells_
 0003:000880A1       snd_seq_queue_remove_cells_
 0003:00088368       snd_seq_control_queue_
 0003:00088405       snd_seq_info_queues_read_
 0003:0008864D       snd_seq_dump_var_event_
 0003:00088826       snd_seq_expand_var_event_
 0003:0008895F       snd_seq_cell_free_
 0003:00088C04       snd_seq_event_dup_
 0003:00088E12       snd_seq_pool_poll_wait_
 0003:00088E85       snd_seq_pool_init_
 0003:00088FA9       snd_seq_pool_done_
 0003:000890D9       snd_seq_pool_new_
 0003:00089186       snd_seq_pool_delete_
 0003:000891DB       snd_sequencer_memory_init_
 0003:000891FD       snd_sequencer_memory_done_
 0003:00089215       snd_seq_info_pool_
 0003:00089422       snd_seq_client_use_ptr_
 0003:00089508       client_init_data_
 0003:0008A230       snd_seq_dispatch_event_
 0003:0008B10F       snd_seq_client_notify_subscription_
 0003:0008B983       snd_seq_set_queue_tempo_
 0003:0008C71F       snd_seq_create_kernel_client_
 0003:0008C861       snd_seq_delete_kernel_client_
 0003:0008C9A6       snd_seq_kernel_client_enqueue_
 0003:0008C9E1       snd_seq_kernel_client_enqueue_blocking_
 0003:0008CA22       snd_seq_kernel_client_dispatch_
 0003:0008CACF       snd_seq_kernel_client_ctl_
 0003:0008CB39       snd_seq_kernel_client_write_poll_
 0003:0008CF0C       snd_seq_info_clients_read_
 0003:0008D0E4       snd_sequencer_device_init_
 0003:0008D15D       snd_sequencer_device_done_
 0003:0008D24C       snd_seq_port_use_ptr_
 0003:0008D2FB       snd_seq_port_query_nearest_
 0003:0008D439       snd_seq_create_port_
 0003:0008D8D2       snd_seq_delete_port_
 0003:0008D9C5       snd_seq_delete_all_ports_
 0003:0008DB2D       snd_seq_set_port_info_
 0003:0008DC83       snd_seq_get_port_info_
 0003:0008E007       snd_seq_port_connect_
 0003:0008E346       snd_seq_port_disconnect_
 0003:0008E4FD       snd_seq_port_get_subscription_
 0003:0008E57D       snd_seq_event_port_attach_
 0003:0008E639       snd_seq_event_port_detach_
 0003:0008E7C2       snd_seq_timer_new_
 0003:0008E82D       snd_seq_timer_delete_
 0003:0008E88D       snd_seq_timer_defaults_
 0003:0008E941       snd_seq_timer_reset_
 0003:0008EA95       snd_seq_timer_set_tempo_
 0003:0008EB2C       snd_seq_timer_set_ppq_
 0003:0008EBF5       snd_seq_timer_set_position_tick_
 0003:0008EC65       snd_seq_timer_set_position_time_
 0003:0008ECD6       snd_seq_timer_set_skew_
 0003:0008ED61       snd_seq_timer_open_
 0003:0008EEC7       snd_seq_timer_close_
 0003:0008EF3C       snd_seq_timer_stop_
 0003:0008F097       snd_seq_timer_start_
 0003:0008F11D       snd_seq_timer_continue_
 0003:0008F1AC       snd_seq_timer_get_cur_time_
 0003:0008F24A       snd_seq_timer_get_cur_tick_
 0003:0008F271       snd_seq_info_timer_read_
 0003:0008F3C0       snd_seq_prioq_new_
 0003:0008F438       snd_seq_prioq_delete_
 0003:0008F5F2       snd_seq_prioq_cell_in_
 0003:0008F783       snd_seq_prioq_cell_out_
 0003:0008F81B       snd_seq_prioq_avail_
 0003:0008F85F       snd_seq_prioq_cell_peek_
 0003:0008F94C       snd_seq_prioq_leave_
 0003:0008FC71       snd_seq_prioq_remove_events_
 0003:0008FDC7       snd_seq_fifo_new_
 0003:0008FEAA       snd_seq_fifo_delete_
 0003:0008FF50       snd_seq_fifo_clear_
 0003:0008FFA9       snd_seq_fifo_event_in_
 0003:000900FC       snd_seq_fifo_cell_out_
 0003:0009020C       snd_seq_fifo_cell_putback_
 0003:00090262       snd_seq_fifo_poll_wait_
 0003:000902B2       snd_seq_fifo_resize_
 0003:000903B3       snd_opl3_synth_use_inc_
 0003:000903F4       snd_opl3_synth_use_dec_
 0003:00090428       snd_opl3_synth_setup_
 0003:0009052F       snd_opl3_synth_cleanup_
 0003:00091098       snd_opl3_interrupt_
 0003:000911C6       snd_opl3_new_
 0003:00091284       snd_opl3_init_
 0003:00091338       snd_opl3_create_
 0003:00091503       snd_opl3_timer_new_
 0003:00091589       snd_opl3_hwdep_new_
 0003:00091A55       snd_opl3_load_drums_
 0003:00091AE5       snd_opl3_drum_switch_
 0003:00091BE5       snd_opl3_calc_volume_
 0003:00091FA1       snd_opl3_timer_func_
 0003:000920F6       snd_opl3_note_on_
 0003:000929FA       snd_opl3_note_off_
 0003:00092B0D       snd_opl3_key_press_
 0003:00092B31       snd_opl3_terminate_note_
 0003:00092D13       snd_opl3_control_
 0003:00092DD3       snd_opl3_nrpn_
 0003:00092DF6       snd_opl3_sysex_
 0003:00092E1C       snd_opl3_open_
 0003:00092E42       snd_opl3_ioctl_
 0003:0009307C       snd_opl3_release_
 0003:000930B6       snd_opl3_write_
 0003:000931D2       snd_opl3_load_patch_
 0003:000933D2       snd_opl3_find_patch_
 0003:000934BC       snd_opl3_clear_patches_
 0003:0009352C       snd_opl3_reset_
 0003:00093D17       snd_mpu401_uart_interrupt_
 0003:00093D5A       snd_mpu401_uart_interrupt_tx_
 0003:00094735       snd_mpu401_uart_new_
 0003:0009595E       snd_cs46xx_download_
 0003:000959EB       snd_cs46xx_download_image_
 0003:000970A6       snd_cs46xx_pcm_
 0003:000974D1       snd_cs46xx_mixer_
 0003:00097BC0       snd_cs46xx_midi_
 0003:00097C9F       snd_cs46xx_gameport_
 0003:000985DB       snd_cs46xx_start_dsp_
 0003:00098B16       snd_cs46xx_suspend_
 0003:00098C6A       snd_cs46xx_resume_
 0003:00098DC3       snd_cs46xx_create_
 0003:00099D48       snd_cs5535audio_suspend_
 0003:00099E52       snd_cs5535audio_resume_
 0003:0009AA28       snd_cs5535audio_pcm_
 0003:0009BE9D       snd_p16v_free_
 0003:0009BED6       snd_p16v_pcm_
 0003:0009C583       snd_p16v_mixer_
 0003:0009C5F9       snd_p16v_alloc_pm_buffer_
 0003:0009C648       snd_p16v_free_pm_buffer_
 0003:0009C671       snd_p16v_suspend_
 0003:0009C6E1       snd_p16v_resume_
 0003:0009C86A       snd_emu10k1_timer_
 0003:0009CDE8       snd_emu10k1_fx8010_register_irq_handler_
 0003:0009CED6       snd_emu10k1_fx8010_unregister_irq_handler_
 0003:0009D155       snd_emu10k1_efx_read_
 0003:000A38C9       snd_emu10k1_init_efx_
 0003:000A3937       snd_emu10k1_free_efx_
 0003:000A39A7       snd_emu10k1_fx8010_tram_setup_
 0003:000A4545       snd_emu10k1_fx8010_new_
 0003:000A461B       snd_emu10k1_efx_alloc_pm_buffer_
 0003:000A4752       snd_emu10k1_efx_free_pm_buffer_
 0003:000A47A5       snd_emu10k1_efx_suspend_
 0003:000A494A       snd_emu10k1_efx_resume_
 0003:000A71A1       snd_emu10k1_mixer_
 0003:000AABFE       snd_emu10k1_pcm_
 0003:000AAD79       snd_emu10k1_pcm_multi_
 0003:000AAEA2       snd_emu10k1_pcm_mic_
 0003:000ABA37       snd_emu10k1_pcm_efx_
 0003:000AC571       snd_emu10k1_midi_
 0003:000AC600       snd_emu10k1_audigy_midi_
 0003:000AC6FF       snd_emu10k1_voice_init_
 0003:000AD0D7       snd_emu10k1_done_
 0003:000AE43D       snd_emu10k1_create_
 0003:000AEE16       snd_emu10k1_suspend_regs_
 0003:000AEF13       snd_emu10k1_resume_init_
 0003:000AEF9B       snd_emu10k1_resume_regs_
 0003:000AFD4C       snd_emu10k1_proc_init_
 0003:000B004C       snd_emu10k1_ptr_read_
 0003:000B015D       snd_emu10k1_ptr_write_
 0003:000B029A       snd_emu10k1_ptr20_read_
 0003:000B0307       snd_emu10k1_ptr20_write_
 0003:000B036C       snd_emu10k1_spi_write_
 0003:000B04CA       snd_emu10k1_i2c_write_
 0003:000B063E       snd_emu1010_fpga_write_
 0003:000B0704       snd_emu1010_fpga_read_
 0003:000B07A5       snd_emu1010_fpga_link_dst_src_write_
 0003:000B081B       snd_emu10k1_intr_enable_
 0003:000B0875       snd_emu10k1_intr_disable_
 0003:000B08D1       snd_emu10k1_voice_intr_enable_
 0003:000B0973       snd_emu10k1_voice_intr_disable_
 0003:000B0A19       snd_emu10k1_voice_intr_ack_
 0003:000B0A9F       snd_emu10k1_voice_half_loop_intr_enable_
 0003:000B0B41       snd_emu10k1_voice_half_loop_intr_disable_
 0003:000B0BE7       snd_emu10k1_voice_half_loop_intr_ack_
 0003:000B0C6D       snd_emu10k1_voice_set_loop_stop_
 0003:000B0D0F       snd_emu10k1_voice_clear_loop_stop_
 0003:000B0DB5       snd_emu10k1_wait_
 0003:000B0E37       snd_emu10k1_ac97_read_
 0003:000B0EA0       snd_emu10k1_ac97_write_
 0003:000B0F01       snd_emu10k1_rate_to_pitch_
 0003:000B1182       snd_emu10k1_voice_alloc_
 0003:000B12F0       snd_emu10k1_voice_free_
 0003:000B19BE       snd_emu10k1_memblk_map_
 0003:000B1AFE       snd_emu10k1_alloc_pages_
 0003:000B1CCB       snd_emu10k1_free_pages_
 0003:000B1D16       snd_emu10k1_synth_alloc_
 0003:000B1DBE       snd_emu10k1_synth_free_
 0003:000B2196       snd_emu10k1_synth_bzero_
 0003:000B224C       snd_emu10k1_synth_copy_from_user_
 0003:000B231A       snd_emu10k1_interrupt_
 0003:000B286B       snd_ymfpci_free_gameport_
 0003:000B5858       snd_ymfpci_pcm_
 0003:000B595C       snd_ymfpci_pcm2_
 0003:000B5A5A       snd_ymfpci_pcm_spdif_
 0003:000B5B4C       snd_ymfpci_pcm_4ch_
 0003:000B6DCB       snd_ymfpci_mixer_
 0003:000B72B4       snd_ymfpci_timer_
 0003:000B844D       snd_ymfpci_suspend_
 0003:000B85D5       snd_ymfpci_resume_
 0003:000B8763       snd_ymfpci_create_
 0003:000BCA64       snd_trident_start_voice_
 0003:000BCABD       snd_trident_stop_voice_
 0003:000BCCC0       snd_trident_write_voice_regs_
 0003:000BF200       snd_trident_pcm_
 0003:000BF3B6       snd_trident_foldback_pcm_
 0003:000BF5CD       snd_trident_spdif_pcm_
 0003:000C0E19       snd_trident_create_gameport_
 0003:000C1745       snd_trident_create_
 0003:000C1F27       snd_trident_alloc_voice_
 0003:000C207E       snd_trident_free_voice_
 0003:000C22B9       snd_trident_suspend_
 0003:000C2384       snd_trident_resume_
 0003:000C29A7       snd_trident_alloc_pages_
 0003:000C2A0B       snd_trident_free_pages_
 0003:000C5430       snd_sbmixer_write_
 0003:000C547B       snd_sbmixer_read_
 0003:000C6254       snd_sbmixer_add_ctl_
 0003:000C6406       snd_sbmixer_new_
 0003:000C66CC       snd_sbmixer_suspend_
 0003:000C6799       snd_sbmixer_resume_
 0003:000C6866       snd_sbdsp_command_
 0003:000C68E5       snd_sbdsp_get_byte_
 0003:000C6961       snd_sbdsp_reset_
 0003:000C6CED       snd_sbdsp_create_
 0003:000C8660       _snd_pcm_hw_param_set_
 0003:000CA279       snd_pcm_oss_write3_
 0003:000CA34A       snd_pcm_oss_read3_
 0003:000CA472       snd_pcm_oss_writev3_
 0003:000CA543       snd_pcm_oss_readv3_
 0003:000CD800       ACPIFindPCIDevice
 0003:000CD8A2       InitACPICall
 0003:000CD940       StrLen
 0003:000CD960       StrNCmp
 0003:000CD990       FindAddress
 0003:000CDBFC       init_MUTEX_
 0003:000CDC32       init_MUTEX_LOCKED_
 0003:000CDC68       down_
 0003:000CDC9A       up_
 0003:000CDCCC       down_interruptible_
 0003:000CE350       _snd_ctl_add_slave_
 0003:000CE659       snd_ctl_make_virtual_master_
 0003:000CE77B       release_and_free_resource_
 0003:000CE7AC       snd_pci_quirk_lookup_
 0003:000CE834       copy_to_user_fromio_
 0003:000CE8E4       copy_from_user_toio_
 0003:000CEC8F       snd_ac97_set_rate_
 0003:000CF2F3       snd_ac97_pcm_assign_
 0003:000CF744       snd_ac97_pcm_open_
 0003:000CFA9F       snd_ac97_pcm_close_
 0003:000CFC90       snd_ac97_pcm_double_rate_rules_
 0003:000D5C4B       snd_ac97_write_
 0003:000D5CC5       snd_ac97_read_
 0003:000D5DAE       snd_ac97_write_cache_
 0003:000D5E39       snd_ac97_update_
 0003:000D5F08       snd_ac97_update_bits_
 0003:000D5F7D       snd_ac97_update_bits_nolock_
 0003:000D8EEB       snd_ac97_get_name_
 0003:000D90C3       snd_ac97_get_short_name_
 0003:000D9229       snd_ac97_bus_
 0003:000D9315       snd_ac97_mixer_
 0003:000DA262       snd_ac97_suspend_
 0003:000DA3E5       snd_ac97_resume_
 0003:000DAF29       snd_ac97_tune_hardware_
 0003:000DC8DC       snd_ac97_proc_init_
 0003:000DCA71       snd_ac97_proc_done_
 0003:000DCAB6       snd_ac97_bus_proc_init_
 0003:000DCB40       snd_ac97_bus_proc_done_
 0003:000DCB70       snd_midi_process_event_
 0003:000DD3A9       snd_midi_channel_set_clear_
 0003:000DDB1D       snd_midi_channel_alloc_set_
 0003:000DDBBD       snd_midi_channel_free_set_
 0003:000DDC6C       snd_util_memhdr_new_
 0003:000DDCDC       snd_util_memhdr_free_
 0003:000DDD50       __snd_util_mem_alloc_
 0003:000DDE31       __snd_util_memblk_new_
 0003:000DDEE9       snd_util_mem_alloc_
 0003:000DDF32       __snd_util_mem_free_
 0003:000DDF98       snd_util_mem_free_
 0003:000DDFFD       snd_util_mem_avail_
 0003:000DE080       __U8RS
 0003:000DE09A       __I8RS
 0003:000DE0B5       __I8LS
 0003:000DE0B5       __U8LS
 0003:000DE0D0       __I8M
 0003:000DE0D0       __U8M
 0003:000DE0F0       strstr_
 0003:000DE1A0       strlcpy_
 0003:000DE230       vsscanf_
 0003:000DE260       sscanf_
 0003:000DE2D0       vsnprintf_
 0003:000DE330       snprintf_
 0003:000DE360       memset_
 0003:000DE380       memmove_
 0003:000DE600       strtoul_
 0003:000DE610       strtol_
 0003:000DE620       __IsTable
 0003:000DE730       __STOSB
 0003:000DE767       __STOSD
 0003:000DF340       __scnf_
 0003:000DF5B0       __prtf_
 0003:000E0294       __set_errno_
 0003:000E02A2       __set_EDOM_
 0003:000E02B0       __set_ERANGE_
 0003:000E02BE       __set_EINVAL_
 0003:000E02D1       __set_doserrno_
 0003:000E02E0       tolower_
 0003:000E02F0       __FDFS
 0003:000E0340       strupr_
 0003:000E0360       __Bits
 0003:000E03BC       __threadstack_
 0003:000E03C3       __threadid_
 0003:000E03CC       __OS2MainInit_
 0003:000E043B       __OS2Init_
 0003:000E0479       __OS2Fini_
 0003:000E0481       __shutdown_stack_checking_
 0003:000E0496       __exit_
 0003:000E04E0       wctomb_
 0003:000E0510       mbtowc_
 0003:000E05D0       _ismbblead_
 0003:000E05F0       ultoa_
 0003:000E0640       ltoa_
 0003:000E0670       ulltoa_
 0003:000E06E0       lltoa_
 0003:000E0710       utoa_
 0003:000E0760       itoa_
 0003:000E0790       __exit_with_msg_
 0003:000E07E0       __fatal_runtime_error_
 0003:000E0810       __InitRtns
 0003:000E0860       __FiniRtns
 0003:000E08C0       __CommonInit_
 0003:000E0905       __mbinit_
 0003:000E0A00       __EnterWVIDEO_
 0003:000E0A28       __OffFinalCS32
 0004:00000003       ___begtext
 0005:00000000       __OffBeginDS32
 0005:00000030       W?deviceOwner$nul
 0005:00000034       W?numOS2Opens$nul
 0005:00000038       _rdOffset
 0005:0000003C       _wrOffset
 0005:00000040       _szprintBuf
 0005:00000044       _fVerbose
 0005:00000048       _fDebug
 0005:0000004C       _idc16_PddHandler
 0005:00000054       W?RM_Help$npn()i
 0005:00000058       W?RM_Help0$npn()i
 0005:0000005C       W?RM_Help3$npn()i
 0005:00000060       W?RMFlags$nul
 0005:000000B0       W?fnCardExitCall$n[]pn()v
 0005:000000D0       _nrCardsDetected
 0005:000000D4       _fStrategyInit
 0005:000000D8       _DbgInt
 0005:000000FC       _DebugLevel
 0005:00000104       _ulget_free_pagesMemUsed
 0005:00000548       W?pmbUsed$npn$_MEMBLOCK$$
 0005:0000054C       W?pmbFree$npn$_MEMBLOCK$$
 0005:00000550       W?uMemFree$nui
 0005:00000554       W?acHeap$npnuc
 0005:00000558       W?ulnAlloc$nul
 0005:0000055C       W?ulcAlloc$nul
 0005:00000560       W?ulnAllocCalls$nul
 0005:00000564       W?ulnFree$nul
 0005:00000568       W?ulcFree$nul
 0005:0000056C       W?ulnFreeCalls$nul
 0005:00000570       W?ulnCompact$nul
 0005:0000059C       _snd_pcm_devices_os2
 0005:00000AA4       _snd_ecards_limit
 0005:00000AA8       _snd_major
 0005:00000AB4       _snd_seq_root
 0005:00000AB8       _snd_oss_root
 0005:00000DA8       _snd_cards
 0005:00001524       ___Is_DLL
 0005:00001528       ___saved_CS
 0005:0000162C       ___MBCSIsTable
 0005:00001730       ___IsDBCS
 0005:00001734       ___hmodule
 0005:00001758       BootCode
 0005:00001768       stackbase
 0005:0000176C       stacksel
 0005:00001770       __OffsetFinalCS16
 0005:00001772       __OffsetFinalDS16
 0005:00001774       _MSG_TABLE32
 0005:00001778       PDDName
 0005:0000177C       RMAllocResource1632
 0005:00001784       RMModifyResources1632
 0005:0000178C       RMDeallocResource1632
 0005:00001794       RMCreateDevice1632
 0005:0000179C       RMCreateAdapter1632
 0005:000017A4       RMCreateDriver1632
 0005:000017AC       RMDestroyDriver1632
 0005:000017B4       RMGetNodeInfo1632
 0005:000017BC       RMDevIDToHandleList1632
 0005:000017C4       RMHandleToResourceHandleList1632
 0005:000017CC       _TimerHandler16
 0005:000017D2       _ISR00
 0005:000017D6       _ISR01
 0005:000017DA       _ISR02
 0005:000017DE       _ISR03
 0005:000017E2       _ISR04
 0005:000017E6       _ISR05
 0005:000017EA       _ISR06
 0005:000017EE       _ISR07
 0005:000017F4       DevHelp32
 0005:000017F8       intSwitchStack
 0005:000017FC       _TKSSBase
 0005:00001800       W?StratDispatch$n[]pn(pf$RP$$)ul
 0005:00001894       W?ForceCard$ni
 0005:000018C4       _jiffies
 0005:000018C8       _current_task
 0005:000018EC       _current
 0005:000018F0       _system_utsname
 0005:00001A76       _ioport_resource
 0005:00001A92       _iomem_resource
 0005:00001AAE       _mem_map
 0005:00001AB2       _this_module
 0005:00001BB2       _szLastALSAError1
 0005:00001C32       _szOverrunTest1
 0005:00001C33       _szLastALSAError2
 0005:00001CB3       _szOverrunTest2
 0005:00001CB4       _iLastError
 0005:00001CB8       _proc_root
 0005:00001D04       _cardcalls
 0005:00001E0C       _midi_port
 0005:00001F78       _szRecSources
 0005:00002004       _oss_devices
 0005:00002144       _alsa_fops
 0005:00002148       _per_bytes
 0005:0000214C       _prev_size
 0005:00002150       _pcm_device
 0005:00002154       _total
 0005:00002158       _opened_handles
 0005:000081D4       _CountWv
 0005:000081D8       _LockAdd
 0005:000081DC       _hextab
 0005:000081ED       _MAGIC_COMM_PORT
 0005:000081F0       _pcmcaps
 0005:00008210       _substream_int
 0005:0000A210       _control_id_changed
 0005:0000A214       _card_id_changed
 0005:0000A218       _unlock_all
 0005:0000A21C       _fInInterrupt
 0005:0000AA9C       _pci_devices
 0005:0000D5DC       _fRewired
 0005:0000E9E0       W?ulcTotalHeap$nul
 0005:0000EA44       ___initcall_alsa_hwdep_init
 0005:0000EA48       ___exitcall_alsa_hwdep_exit
 0005:0000EAF0       ___initcall_alsa_timer_init
 0005:0000EAF4       ___exitcall_alsa_timer_exit
 0005:0000EB80       ___initcall_alsa_rawmidi_init
 0005:0000EB84       ___exitcall_alsa_rawmidi_exit
 0005:0000EE60       ___initcall_alsa_pcm_init
 0005:0000EE64       ___exitcall_alsa_pcm_exit
 0005:0000EEBC       ___initcall_alsa_sound_init
 0005:0000EEC0       ___exitcall_alsa_sound_exit
 0005:0000EF44       _snd_pcm_link_rwlock
 0005:0000F008       _snd_pcm_f_ops
 0005:0000F114       ___initcall_snd_mem_init
 0005:0000F118       ___exitcall_snd_mem_exit
 0005:0000F574       ___initcall_alsa_card_bt87x_init
 0005:0000F578       ___exitcall_alsa_card_bt87x_exit
 0005:0000F710       ___initcall_alsa_card_als4000_init
 0005:0000F714       ___exitcall_alsa_card_als4000_exit
 0005:00010571       ___initcall_alsa_card_cmipci_init
 0005:00010575       ___exitcall_alsa_card_cmipci_exit
 0005:0001091C       ___initcall_alsa_card_atiixp_init
 0005:00010920       ___exitcall_alsa_card_atiixp_exit
 0005:00010DDC       ___initcall_alsa_card_fm801_init
 0005:00010DE0       ___exitcall_alsa_card_fm801_exit
 0005:00011494       ___initcall_alsa_card_via82xx_init
 0005:00011498       ___exitcall_alsa_card_via82xx_exit
 0005:00011BD8       ___initcall_alsa_card_m3_init
 0005:00011BDC       ___exitcall_alsa_card_m3_exit
 0005:00012B6C       ___initcall_alsa_card_intel8x0_init
 0005:00012B70       ___exitcall_alsa_card_intel8x0_exit
 0005:00012E20       ___initcall_alsa_card_es1968_init
 0005:00012E24       ___exitcall_alsa_card_es1968_exit
 0005:000136B9       ___initcall_alsa_card_es1938_init
 0005:000136BD       ___exitcall_alsa_card_es1938_exit
 0005:0001398C       ___initcall_alsa_card_cs4281_init
 0005:00013990       ___exitcall_alsa_card_cs4281_exit
 0005:00013E28       ___initcall_alsa_card_ens137x_init
 0005:00013E2C       ___exitcall_alsa_card_ens137x_exit
 0005:00014314       ___initcall_alsa_card_ca0106_init
 0005:00014318       ___exitcall_alsa_card_ca0106_exit
 0005:00016028       ___initcall_patch_via_init
 0005:0001602C       ___exitcall_patch_via_exit
 0005:00017EB0       ___initcall_patch_conexant_init
 0005:00017EB4       ___exitcall_patch_conexant_exit
 0005:0001800C       ___initcall_patch_atihdmi_init
 0005:00018010       ___exitcall_patch_atihdmi_exit
 0005:0001B172       ___initcall_patch_sigmatel_init
 0005:0001B176       ___exitcall_patch_sigmatel_exit
 0005:00022758       ___initcall_patch_analog_init
 0005:0002275C       ___exitcall_patch_analog_exit
 0005:00022EF8       ___initcall_patch_cmedia_init
 0005:00022EFC       ___exitcall_patch_cmedia_exit
 0005:0003FFC9       ___initcall_patch_realtek_init
 0005:0003FFCD       ___exitcall_patch_realtek_exit
 0005:00040630       ___initcall_alsa_card_azx_init
 0005:00040634       ___exitcall_alsa_card_azx_exit
 0005:00040787       _snd_hda_bind_vol
 0005:00040797       _snd_hda_bind_sw
 0005:00040A23       _auto_pin_cfg_labels
 0005:00040BEC       _seq_client_load
 0005:00040C28       _seq_default_timer_class
 0005:00040C2C       _seq_default_timer_sclass
 0005:00040C30       _seq_default_timer_card
 0005:00040C34       _seq_default_timer_device
 0005:00040C38       _seq_default_timer_subdevice
 0005:00040C3C       _seq_default_timer_resolution
 0005:00040C40       ___initcall_alsa_seq_init
 0005:00040C44       ___exitcall_alsa_seq_exit
 0005:00040C68       ___initcall_alsa_seq_device_init
 0005:00040C6C       ___exitcall_alsa_seq_device_exit
 0005:00040DBC       _use_internal_drums
 0005:00040DC0       _opl3_ops
 0005:00040DE4       ___initcall_alsa_opl3_seq_init
 0005:00040DE8       ___exitcall_alsa_opl3_seq_exit
 0005:00040E58       ___initcall_alsa_opl3_init
 0005:00040E5C       ___exitcall_alsa_opl3_exit
 0005:00040FF0       _snd_opl3_regmap
 0005:00041034       ___initcall_alsa_mpu401_uart_init
 0005:00041038       ___exitcall_alsa_mpu401_uart_exit
 0005:00041150       ___initcall_alsa_card_cs46xx_init
 0005:00041154       ___exitcall_alsa_card_cs46xx_exit
 0005:0004EE30       ___initcall_alsa_card_cs5535audio_init
 0005:0004EE34       ___exitcall_alsa_card_cs5535audio_exit
 0005:0004F09C       ___initcall_alsa_card_emu10k1_init
 0005:0004F0A0       ___exitcall_alsa_card_emu10k1_exit
 0005:00051E38       ___initcall_alsa_card_ymfpci_init
 0005:00051E3C       ___exitcall_alsa_card_ymfpci_exit
 0005:000527F8       ___initcall_alsa_card_ali_init
 0005:000527FC       ___exitcall_alsa_card_ali_exit
 0005:00052934       ___initcall_alsa_card_trident_init
 0005:00052938       ___exitcall_alsa_card_trident_exit
 0005:0005F63C       ___initcall_alsa_card_nm256_init
 0005:0005F640       ___exitcall_alsa_card_nm256_exit
 0005:0005FC00       ___initcall_alsa_sb_common_init
 0005:0005FC04       ___exitcall_alsa_sb_common_exit
 0005:0005FC80       ___initcall_alsa_pcm_oss_init
 0005:0005FC84       ___exitcall_alsa_pcm_oss_exit
 0005:0005FD14       ___EFG_printf
 0005:0005FD18       ___EFG_scanf
 0005:0005FD1C       ___FirstThreadData
 0005:0005FD20       ___GetThreadPtr
 0005:0005FD24       __AccessFileH
 0005:0005FD28       __ReleaseFileH
 0005:0005FD2C       __AccessIOB
 0005:0005FD30       __ReleaseIOB
 0005:0005FD34       __AccessNHeap
 0005:0005FD38       __AccessFHeap
 0005:0005FD3C       __ReleaseNHeap
 0005:0005FD40       __ReleaseFHeap
 0005:0005FD44       __AccessTDList
 0005:0005FD48       __ReleaseTDList
 0005:0005FD4C       ___sig_init_rtn
 0005:0005FD50       ___sig_fini_rtn
 0005:0005FD54       __threadstksize
 0005:0005FD58       ___process_fini
 0005:0005FD5C       __dynend
 0005:0005FD60       __curbrk
 0005:0005FD64       __LpCmdLine
 0005:0005FD68       __LpPgmName
 0005:0005FD6C       __LpDllName
 0005:0005FD70       __LpwCmdLine
 0005:0005FD74       __LpwPgmName
 0005:0005FD78       __LpwDllName
 0005:0005FD7C       __STACKLOW
 0005:0005FD80       __STACKTOP
 0005:0005FD84       __ASTACKSIZ
 0005:0005FD88       __ASTACKPTR
 0005:0005FD8C       __cbyte
 0005:0005FD90       __cbyte2
 0005:0005FD94       __child
 0005:0005FD98       __no87
 0005:0005FD9A       __Envptr
 0005:0005FD9E       __Envseg
 0005:0005FDA0       __osmajor
 0005:0005FDA1       __osminor
 0005:0005FDA2       ___FPE_handler
 0005:0005FDA8       ___MBCodePage
 0005:0005FDAC       ___WD_Present
 0005:0005FDB0       __amblksiz
 0005:00060612       ___initcall_alsa_ac97_init
 0005:00060616       ___exitcall_alsa_ac97_exit
 0005:0006073C       ___initcall_alsa_seq_midi_emul_init
 0005:00060740       ___exitcall_alsa_seq_midi_emul_exit
 0005:00060744       ___initcall_alsa_util_mem_init
 0005:00060748       ___exitcall_alsa_util_mem_exit
 0005:00072908       ___Alphabet
 0005:00075760       _snd_pcm_known_rates
 0005:0007AB78       __OffFinalDS32
 0005:0007AB7C       __Start_XI
 0005:0007AB82       __Start_YI
 0005:0007AB82       __End_XI
 0005:0007AB82       __End_YI
 0005:0007ABD0       __nullarea
 0005:0008ABE0       _edata
 0005:0008ABE0       _end
